:020000040000FA
:10000000900A002045110000673D00009510000097
:10001000951000009510000095100000951000004C
:10002000951000009510000095100000850F00004D
:100030009510000095100000310F0000693C000091
:100040000511000005110000051100000511000058
:100050000511000005110000051100000511000048
:100060000511000005110000051100000511000038
:100070000511000005110000051100000511000028
:100080000511000005110000051100000511000018
:100090000511000005110000051100000511000008
:1000A00005110000051100000511000005110000F8
:1000B00005110000051100000511000005110000E8
:1000C00005110000051100000511000005110000D8
:1000D00005110000051100000511000005110000C8
:1000E00005110000051100000511000005110000B8
:1000F00005110000051100000511000005110000A8
:100100000511000005110000051100000511000097
:100110000511000005110000051100000511000087
:100120000511000005110000051100000511000077
:100130000511000005110000051100000511000067
:100140000511000000000000000000000000000099
:10015000000000000000000000000000000000009F
:10016000000000000000000000000000000000008F
:10017000000000000000000000000000000000007F
:10018000000000000000000000000000000000006F
:10019000000000000000000000000000000000005F
:1001A000000000000000000000000000000000004F
:1001B000000000000000000000000000000000003F
:1001C000000000000000000000000000000000002F
:1001D000000000000000000000000000000000001F
:1001E000000000000000000000000000000000000F
:1001F00000000000000000000000000000000000FF
:10020000DEE61E284CBBCE8F025B00003C000000E7
:10021000008000000100000000000000000000005D
:10022000FFFF02910000000000000000000000003D
:1002300000000000000000000000000053B94AB9AF
:10024000002908BF00281CBF4FF0FF314FF0FF30DE
:1002500000F07CB9ADF1080C6DE904CE00F006F8B1
:10026000DDF804E0DDE9022304B070472DE9F04732
:100270008C46089D04468A46002B4AD18A4217467E
:1002800062D9B2FA82F64EB1C6F1200E01FA06F337
:10029000B740B44020FA0EFE4EEA030A4FEA174870
:1002A000230C1FFA87F9BAFBF8FE08FB1EAA0EFB07
:1002B00009F243EA0A439A420BD9FB180EF1FF31C7
:1002C0002CBF012000209A4202D9002800F02A8188
:1002D0008E469A1AA3B2B2FBF8F008FB102200FB7C
:1002E00009F943EA0244A14507D93C1900F1FF335B
:1002F00002D2A14500F210811846A4EB090440EA9D
:100300000E4000211DB1F4400023C5E90043BDE8C3
:10031000F0878B4208D9002D00F0F2800021C5E95A
:10032000000C0846BDE8F087B3FA83F100294ED1EE
:100330006345C0F0E880824240F2E5800846002D27
:10034000E5D0C5E9004AE2E702B9FFDEB2FA82F67B
:10035000002E40F099808B1A4FEA124E1FFA82F855
:1003600001214FEA144CB3FBFEF20EFB123008FBE6
:1003700002F94CEA004CE14508D917EB0C0C02F1EC
:10038000FF3302D2E14500F2CA801A46ACEB090CF9
:10039000A3B2BCFBFEF00EFB10CC08FB00F843EA56
:1003A0000C44A0450ED93C1900F1FF332CBF4FF08F
:1003B000010C4FF0000CA04503D9BCF1000F00F078
:1003C000A8801846A4EB080440EA02409AE7C1F16D
:1003D00020048B4002FA01FE0CFA01F6E24020FAFA
:1003E00004F72CFA04FC00FA01F813433E431F0CF7
:1003F000320C1FFA83F9BCFBF7F007FB10CC00FBB3
:1004000009FA42EA0C4CE24508D913EB0C0C00F156
:10041000FF3202D2E24500F289801046ACEB0A0CB2
:10042000B6B2BCFBF7FA07FB1ACC0AFB09F946EA9D
:100430000C42914506D99A180AF1FF3601D291452E
:100440007AD8B2464AEA0040A2EB0902A0FB0E6746
:10045000BA42B446B94602D307D1B04505D2B6EB8D
:100460000E0C67EB030301389946002D6BD0B8EBF7
:100470000C0362EB090202FA04F4CB40CA400021EB
:100480001C43C5E9004242E7B740C6F1200201FA29
:1004900006F3B44021FA02FC4FEA174E20FA02F2AA
:1004A0001FFA87F8BCFBFEF11A430EFB11CC01FBCF
:1004B00008F0130C43EA0C4C604507D917EB0C0C01
:1004C00001F1FF3301D2604533D81946ACEB000C83
:1004D00092B2BCFBFEF00EFB10CC00FB08F342EA2C
:1004E0000C4C634507D917EB0C0C00F1FF3201D21D
:1004F000634525D81046ACEB030340EA014130E7E1
:100500002946284603E7841A6CEB030301209A4628
:1005100015E702383C4455E702383C44EDE6023A20
:10052000BC4433E7AEF1020E3B44D2E602389C44B1
:1005300074E70239BC44C9E7AAF1020A1A4481E708
:100540000238BC44D7E72946E1E600BF704700BF48
:100550002DE9E04F2746A046A146A246A346A44661
:100560002DED108B4FF0000545EC185B45EC195A4A
:1005700045EC1A5A45EC1B5A45EC1C5A45EC1D5AE1
:1005800045EC1E5A45EC1F5AF1EE105A4FF66076B4
:10059000C0F6FF763540E1EE105A84F30088254618
:1005A0002646A447BDEC108BBDE8E08F0B680133F5
:1005B0000B60014B1B681847D01300202DE9F04F4A
:1005C00085B00E9C9B46012CB8BF0124012B0CBFAB
:1005D0003023202316468246884601250A2700221A
:1005E000DFF86C900293B6FBF9F301930AB9B145B9
:1005F0001CD8019B414603F13000D0470122013550
:10060000019B013F09FB13660A23012FB9FBF3F994
:10061000E9D1414606F13000D047BBF1030F02D1CA
:10062000641B002C0EDC05B0BDE8F08FBC42E7DB9C
:10063000BBF1020FE4D84146029803920135D0473E
:10064000039ADDE741462020D047013CE9E700BF9F
:1006500000CA9A3B014B1860704700BFD0130020BE
:10066000002313B502AC44F8043D02460B46034890
:10067000214603F070F802B010BD00BFAD050000C8
:100680004FF02002EFF3118382F31188BFF36F8FD5
:100690000121044AC2F8401583F31188BFF36F8F1C
:1006A00000207047009003500A2838B50446074DD3
:1006B00004D1286843680D215B689847286843681F
:1006C000E1B25B689847204638BD00BF08000020B3
:1006D00010B5044C204601F095F82046BDE81040C6
:1006E000FFF7B8BFA906000008B5044801F0AEFA4C
:1006F000034B1860FFF7ECFF002008BDC84700005F
:100700000800002008B5114B1A686AB14FF050225A
:10071000D2F80423D10707D500220D481A60836858
:10072000597A09B903F0F0F90A4B1A686AB14FF027
:100730005022D2F80423920707D5002201211A6023
:100740000348BDE8084003F0DFB908BD0051005080
:10075000801400200451005000220D4BC3F84021AA
:100760004FF02002EFF3118182F31188BFF36F8FF6
:10077000084AD3F804051368C01A20F07F400344E8
:10078000136081F31188BFF36F8F02F031B800BF9F
:10079000005001502400002070B5154801F056FAB1
:1007A00010B3436801211B689847002401264FF4C9
:1007B00080334FF400120F4D3146C5F80845C5F897
:1007C0004065C5F804330C4B15201C600B4BC3F877
:1007D0008021224600F0F6FB152000F0E3FB2046C6
:1007E000074B1E602E6070BD4FF0FF30FBE700BF6F
:1007F0009D490000005001504051015000E100E0CF
:100800000850015070B5264EB0F1FF3F08BF30468A
:100810004FF02003EFF3118483F31188BFF36F8F40
:10082000204BD3F80455204B1B68EA1A22F07F4274
:10083000B2F5000F1AD2411E21EAE171B142A8BF00
:100840003146501C0844B04294BF18189819451BF3
:1008500025F07F45134A20F07F43022DC2F8403532
:1008600006D984F31188BFF36F8F70BD0021E8E7CC
:10087000D2F804350D49C31A23F07F435D1E8D4223
:1008800005D94FF400120A4BC3F80021E9E7012B08
:1008900002BF023020F07F40C2F84005E1E700BF10
:1008A000FEFFFF000050015024000020FEFF7F00EB
:1008B00000E100E04FF02002EFF3118382F3118892
:1008C000BFF36F8F064AD2F80405064A1268801AF1
:1008D00020F07F4083F31188BFF36F8F704700BF14
:1008E000005001502400002008B543B2002B0CDB5F
:1008F000012200F01F018A405B091049203341F8B2
:100900002320BFF34F8FBFF36F8F830003F1A0430A
:1009100003F540533128D3F8002806D0002A07DA1F
:1009200002F00302023A012A02D8054AC3F800285D
:10093000002103F0E9F9002008BD00BF00E100E05C
:100940000001008030B54FF440444CF2040585B0FE
:100950004FF440412C4803F074F821682B4803F011
:1009600070F829682A4803F06CF8102200216846C4
:1009700003F094FA236868460093029400F0CCFEDA
:10098000012000F0F9FE002000F0E2FE002000F05F
:1009900007FF0121002000F021FF00F015FF2C6867
:1009A0001C4803F04EF80820FFF79EFF24F00104D6
:1009B000BFF34F8FBFF36F8F64086400204621465A
:1009C000224623469FED140ADFED130A9FED121A0B
:1009D000DFED111A9FED102ADFED0F2A9FED0E3A81
:1009E000DFED0D3A9FED0C4ADFED0B4A9FED0A5A01
:1009F000DFED095A9FED086ADFED076A9FED067A81
:100A0000DFED057AFFF7A4FD1D4900003449000021
:100A10004949000067490000000000002DE9F84343
:100A20006E4803F00EF80021DFF8FC816C4F6D4D2D
:100A300058F82140CA0301F5C07347F823406A48BB
:100A400002F500434E1C02F0FCFF684B14F0100F3F
:100A50006749684808BF194602F0F3FF14F0040F15
:100A600014BF72212D21284602F0EBFF14F0020F73
:100A700014BF77212D21284602F0E3FF14F0010F67
:100A800014BF78212D21284602F0DBFF14F4807F6B
:100A900014BF6C212D21284602F0D3FF564802F0E6
:100AA000D0FF202E3146C3D1544B4D4AC3F3C4313D
:100AB000C3F30E03C3F50043C3F34313C2F8001599
:100AC000C2F80435D2F80015D2F804254C4852017A
:100AD00002F0B7FF484802F0B4FF03F0C7F8014640
:100AE00010B1484802F0ADFF434802F0AAFF464863
:100AF00002F0A7FF0021DFF83481394F394D58F853
:100B000021404A0301F5E07347F823403F4802F5CE
:100B100000534E1C02F095FF344B14F0100F344973
:100B2000344808BF194602F08CFF14F0040F14BFBC
:100B300072212D21284602F084FF14F0020F14BF09
:100B400077212D21284602F07CFF14F0010F14BFFD
:100B500078212D21284602F074FF14F4807F14BF01
:100B60006C212D21284602F06CFF234802F069FF1A
:100B7000202E3146C3D10024194D1F4802F061FFD9
:100B8000C5F88044224802F05CFFDFF8A480C5F875
:100B9000C044DFF8A0901F4D05EBC406777955F8E7
:100BA0003420002F14BF43464B4621461A4802F01A
:100BB00048FF57B91948013402F043FF1A2CEBD112
:100BC0000D48BDE8F84302F03CBF3079FFF78CFEDA
:100BD00008B11348EFE71348EDE700BFF9470000FD
:100BE00000300050314800001C480000E24700007F
:100BF000D9470000064900002D4B0000E07F0000AF
:100C0000344800007A480000AA480000CC480000A0
:100C1000E0480000EC440000FC48000009490000E6
:100C200010490000184900006C440000BC45000059
:100C3000EE470000E647000010B500284BD0002A20
:100C400049D0264B99423CD9541803F61D239C42A7
:100C50003AD803F0F6F80020BDE81040714672461D
:100C60007346B7EE000AF7EE000AB7EE001AF7EE89
:100C7000001AB7EE002AF7EE002AB7EE003AF7EEB8
:100C8000003AB7EE004AF7EE004AB7EE005AF7EE28
:100C9000005AB7EE006AF7EE006AB7EE007AF7EE98
:100CA000007A8EF3008C10B4F1EE10CA4FF6607427
:100CB000C0F6FF740CEA040CE1EE10CA10BCF44656
:100CC0007447074B994203D9064B54189C42C0D92C
:100CD0004FF0FF30C0E76FF01500BDE70302FF00E3
:100CE0002F01FF003801FF002DE9F04F824685B04B
:100CF0008946002951D00026DFF8B0B0DFF8B08077
:100D000001AF5BF8264098E80700544487E80700E5
:100D10000C223946204603F06DF8054608B9002C30
:100D20003ED10136052EECD16FF00D05284605B0F9
:100D3000B7EE000AF7EE000AB7EE001AF7EE001A57
:100D4000B7EE002AF7EE002AB7EE003AF7EE003AC7
:100D5000B7EE004AF7EE004AB7EE005AF7EE005A37
:100D6000B7EE006AF7EE006AB7EE007ABDE8F04F22
:100D7000714672467346F7EE007A8EF3008C10B41B
:100D8000F1EE10CA4FF66074C0F6FF740CEA040C62
:100D9000E1EE10CA10BCF44674476FF01505C5E7C4
:100DA0003C222146484603F04CF8BFE73C46000091
:100DB0001C440000014801F089BF00BF50460000FC
:100DC00008B530B143683BB1006801F03FF900203D
:100DD00008BD6FF4E040FBE70048F9E7EA8FFFFF4A
:100DE00008B558B1436863B100684FF0FF3101F0B6
:100DF000BBF80028044808BF002008BD6FF4E0409D
:100E0000FBE70248F9E700BFE98FFFFFEA8FFFFF2A
:100E100038B5044618B90B4B0B485B6898476568B2
:100E200055B115F00205206807D10146074801F0C9
:100E30006DF825600023636038BD1422002103F0A3
:100E40002DF8F7E7241400208E4A00002800002027
:100E500010B5044618B9134B13485B68984763688C
:100E6000BBB92368ABB94FF0FF3221460F4801F000
:100E70001FF808B923681BB90A4B0D485B689847EF
:100E800014220021206803F009F8636843F002038C
:100E90006360206803F098F8636843F001036360BF
:100EA00010BD00BF241400208E4A0000280000203E
:100EB000B44A000008B5064940231422054803F04F
:100EC00068F8BDE808400449044801F037BF00BF96
:100ED000440000202800002068460000584600001A
:100EE00004488168406A884203D003494FF0805229
:100EF0000A6070473006002004ED00E0094A0A4904
:100F0000936809685866996608494B6843F08053AE
:100F10004B60002383F31188BFF36F8F9368986E43
:100F2000704700BF30060020D446000000ED00E00E
:100F300012498A684FF028001044EFF3098C80E8CA
:100F4000F01F202080F31188BFF36F8F0C4F4FF0FC
:100F500000664A6A8A603E60506E0023536680F3E2
:100F6000118804B5104602F005FFBDE8044002F107
:100F7000280090E8F01F8CF30988704730060020A5
:100F800004ED00E01EF0040F0CBFEFF30880EFF358
:100F90000980816911F8021C0229FFD001B502F015
:100FA000DEFE01BD43B2002B08DB012200F01F0072
:100FB00002FA00F0024A5B0942F82300704700BFC2
:100FC00000E100E043B2002B01F10101A8BF03F1F1
:100FD00060434FEA4111B8BF054BC9B2ABBF03F53F
:100FE000614300F00F0083F800131954704700BFED
:100FF00014ED00E073B51E460A9B05460093099B5D
:101000008C1803F076F80B4AA4F1200323F00703B1
:1010100022F001029A61069A1E605A60079A9A604D
:10102000089ADA604FF08072DA61AB6400236B6675
:1010300002B070BD5D3A0000F8B51E4605460C468C
:1010400017460023E1EE103A00F0D6F90A4B3C4473
:1010500028469D6024F0070402F08CFE304684F39D
:101060000988002163B681F31188BFF36F8F0022D6
:10107000002302F0F3FC00BF3006002001491022DB
:101080000A60704710ED00E0404080F3118830BFE7
:10109000704700BFEFF30880EFF30981724601B596
:1010A00000F0D2F801BD00BF30BFFFF7FDBF00BFA9
:1010B000114A08B5114B22F07F029A60BFF34F8F9F
:1010C000BFF36F8FD3F8882042F4A002C3F88820C2
:1010D0000B4A536823F040435360BFF34F8FBFF375
:1010E0006F8F0023E1EE103A00F0F0FD00F0F8FD04
:1010F00000F050F900F032FE0000000000ED00E0CA
:1011000030EF00E001B572B60B4A106A00281EBF2E
:101110000021116202F03BFF62B6EFF30580A0F1FF
:1011200010004FEAC0000549014409C99847BDE8CD
:101130000140034908470000300600209C410000A0
:10114000E10E000002F095FC202080F31188084891
:101150004FF40061401880F30988EFF314800221F6
:10116000084380F31488BFF36F8FFFF7A1FF0000DF
:10117000D00B00200C4B9A6A9A6A9A6A920708D59B
:101180005A6B9A6A120604D518B19A6A22F0800244
:101190009A6200209A6A9A6A9A6A9A6A42F0FF02F0
:1011A0009A620870704700BF00ED00E00D4B9A6A2C
:1011B0009A6A9A6A920508D59A6B9A6A120404D5BB
:1011C00018B19A6A22F400429A6200209A6A9A6AD6
:1011D000D205044A58BF9B6A936A43F47F439362E3
:1011E0000870704700ED00E0074B00209A6A9A6A89
:1011F0009A6A9A6A9A6A9A6A9A6A9A6A6FEA02423A
:101200006FEA12429A62704700ED00E00D4B9A6956
:101210005A695A69D0070FD45A6991070CD45A6990
:10122000520709D45A69100706D45A69D10603D463
:101230005A69920658BF5A695A6942F0FF025A61C8
:10124000704700BFD0ED00E0F0B5414B8BB05B685C
:101250000025C3F3080385F31188BFF36F8F02F0F5
:101260007F44B4F17F4F1FD112F001041BD056060A
:1012700002F0080468D482F00402C2F3800564B16D
:10128000EFF389860022033B8DF80720042B4CD80E
:10129000DFE803F00C4D51424900EFF38886F1E797
:1012A00006460125EEE725462E46EBE7284BDA6A8F
:1012B00092073AD4DC6A14F0804408D028331B78B3
:1012C000EBB101200DF10701FFF754FF04469DF833
:1012D000073093B92022314602A802F0B2FD099BE3
:1012E0006DB3C3F3080222B96FEA53236FEA4323B5
:1012F000099302A9204602F030FD0BB0F0BD154B5A
:101300001B782BB101200DF10701FFF74FFFDDE73F
:10131000114B1C88A7B217B1FFF766FFD6E70F4B3A
:101320005C69002CD3D0FFF771FF0024CFE70DF1EB
:1013300007010020C8E70DF107010020E5E723F4CD
:10134000FF7323F00103D3E7002CA9D00E4699E7E1
:1013500000ED00E029ED00E02AED00E0D0ED00E036
:10136000024A536943F010035361704700ED00E0F7
:10137000BFF34F8F0549064BCA6802F4E06213437E
:10138000CB60BFF34F8F00BFFDE700BF00ED00E073
:101390000400FA05002320210348C2180133412B21
:1013A00082F80013F9D1704700E100E038B5054636
:1013B0004FF02003EFF3118483F31188BFF36F8F95
:1013C00000F0E8FF0A4B9B68AB420BD1094B5A680F
:1013D000C2F3080212B92046FFF790FD5A6842F0A6
:1013E00080525A602046BDE8384002F008BE00BF77
:1013F0003006002000ED00E010B50E4B88B00293DF
:101400000D4B0E4C03930E4B08A8049302AB40F80F
:101410001C3D0C4A2346012100F002F900230793EA
:10142000094B0121E41A05A80593069400F002F97E
:1014300008B010BD000000200000000000000120E6
:1014400006000100000000200000002010B50B681D
:101450000C7A23F01F0304F01F021A43CB686409BF
:1014600023F01F03044943F0010343EA4403886067
:10147000CA600B6110BD00BF90ED00E02DE9F04F98
:101480008046894614460027484D85B04F4507DA07
:1014900058F827305E68C6B31F2E05D86FF01504C4
:1014A000204605B0BDE8F08FF206F7D1D3F800A0D2
:1014B0001AF01F0FF2D1504602F086FC834606EB6D
:1014C0000A00013802F080FC8345E7D11BF1160FBA
:1014D000E4D0631E5B45E1DBC5F808B0E86858F866
:1014E0002710C5F808B02E6920F01F00D1E900329E
:1014F0001A44984246F01F0602F1FF3A18D15645A9
:1015000005D15FFA8BF002F03DFC0137BEE7C5F86C
:1015100008B0EB6822F01F0203F01F031A43EA60D1
:10152000E0B202F02FFC10F1160FB7D0441CECE72C
:10153000C5F808B02A69013B23F01F0302F01F021F
:1015400013435645E0B22B61EBD002F01BFC10F1C7
:10155000160FA3D0C5F808B0EA689DF80830013E20
:1015600062F304038DF808302B699DF808205B08AE
:1015700063F347128DF8082058F827200130D2E98C
:1015800000321344009323F01F031E44A6EB0A0607
:10159000C4B226F01F060F2C03963FF67FAF2046FD
:1015A0006946FFF753FF0134AFE700BF90ED00E05D
:1015B0000522034B5A60BFF34F8FBFF36F8F704705
:1015C00090ED00E0BFF35F8F0022014B5A6070473F
:1015D00090ED00E070B50E4D2E68102E15D8002449
:1015E000FFF7F0FF0B4B0C4A1A63A64205D10B4BD9
:1015F0001E70FFF7DDFF002070BD6968204601EB1B
:101600000411FFF723FF0134EFE74FF0FF30F3E75A
:101610007C46000090ED00E0AAFF44008C0600200C
:1016200010B5034C2278FFF729FF207010BD00BFD2
:101630008C0600202DE9F74F894607460026DFF883
:101640009080DFF890A0214C4E4519DAD7F804B00D
:10165000BBF1000F36D03B681846019302F0B4FB93
:10166000019B05460BEB0300013802F0ADFB142390
:10167000854203FB06F306D06FF0150248F80320FD
:1016800003B0BDE8F08F15F1160F48F80350F7D0FE
:101690009AF80020AA42F3DDA5604344A560E06803
:1016A000197B60F3040119732169187B490861F300
:1016B00047101873E26822F01F025A60226922F074
:1016C0001F021A6101360C37BEE700BF90ED00E043
:1016D000440500208C06002070B50C4B0E461C788B
:1016E0000546234600210A4A0F2B0BDD094B191D25
:1016F0001868FFF7ABFE224631462846BDE8704029
:10170000FFF7BCBE936011610133EDE78C0600204A
:1017100090ED00E04405002082680C4B9A6003685D
:1017200083F38888436883F38988027B02F0010190
:10173000EFF3948323F00303920748BF43F00203BF
:1017400009B143F0010383F39488704700ED02E090
:10175000084AD36848B123F400531B041B0C43F020
:10176000BF6343F40033D36070479BB243F400532C
:10177000F5E700BF00ED00E0084AD36840B19BB236
:1017800043F4804343F0BF6343F40033D3607047B6
:1017900023F480431B041B0CF4E700BF00ED00E0C2
:1017A000084AD36840B19BB243F0080343F0BF63DB
:1017B00043F40033D360704723F008031B041B0C71
:1017C000F4E700BF00ED00E0034AD2F88C3043F4A8
:1017D0004063C2F88C30704700ED00E0084B1A6897
:1017E00018B142F001021A60704722F001021A603B
:1017F0001A6811B142F00202F5E722F00202F2E7A4
:10180000D0ED00E0014B1860704700BFF4130020DA
:10181000F0B54B79012B29D0032B24D110268B79DD
:10182000032B20D1CC792CB1012C1CD103689B68EF
:101830001B79C3B10A7912B1022A14D10E2247F6DC
:10184000122703689B681D680B68BB426FD029D8BC
:10185000B3F5965F65D014D8B3F5167F4FD007D88F
:10186000B3F5967F78D06FF0220056E00026D6E7D9
:10187000B3F5966F52D0B3F5166FF4D14FF41D2324
:101880003FE0B3F5615F4ED004D8B3F5165FEAD1FF
:10189000334B36E0B3F5964F47D0B3F5E14FE2D185
:1018A000304B2EE0B3F5E13F4AD012D84DF6C027B9
:1018B000BB423FD005D8B3F5164FD4D14FF41D032A
:1018C0001FE0B3F5614F38D0B3F5963FCBD1264B2F
:1018D00017E0B3F5E12F39D008D8B3F5613F32D026
:1018E000224FBB42BFD14FF080630AE0B3F5612FB6
:1018F0002FD01F4FBB42B6D14FF0805301E04FF4C1
:101900001C33C5F8243544EA06031343C5F86C3587
:10191000836803C983E803000020F0BD4FF49E23D1
:10192000EFE7144BEDE7144BEBE7144BE9E74FF40B
:101930000003E6E74FF46503E3E74FF46B03E0E7EA
:101940004FF0EB73DDE74FF06C73DAE74FF0E863CD
:10195000D7E74FF07063D4E74FF4A033D1E700BF6F
:101960000050270000C0750000903A0190D003009D
:1019700040420F0000B0130000F03A0000A04E00FB
:10198000026870B59268184B14684FF00052856871
:1019900003219A601D260022C3F87412C3F8702236
:1019A000C4F80C651C26C4F814654FF000669E60F0
:1019B000C3F86C12C3F868221B23C4F808351A2335
:1019C0002946C4F81035FFF723FF58B90823C4F897
:1019D00000351D440123C4F81001C4F83455C4F87F
:1019E0003835236070BD00BF002584502DE9F043D9
:1019F00000261E4C85B054F8049C1D4F01ADB14526
:101A000003D8002005B0BDE8F083636A97E80700BB
:101A1000D3F8008085E807000C222946404602F0F2
:101A2000E9F9A0B9B8F1000F11D0636A21691B6808
:101A30001A6991420BD19A69A169914207D8E1696B
:101A4000914204D962695B6932EA030307D0236AD1
:101A50004BB1404080F311884FF0040002DFE3688F
:101A600001361C44CBE7626A1360F8E73C020000D1
:101A700028440000064B1868043B1B68092B05D15D
:101A8000013801288CBF00200120704700207047DA
:101A90003401FF00054B1868043B1B68092B03D178
:101AA000431E584258417047002070473401FF00E0
:101AB0004E4A08B5136843F002031360FFF7DAFFDC
:101AC00030B14FF050230022C3F81421C3F818217D
:101AD000FFF7E0FF30B10123454A1360A2F6382238
:101AE000C2F87835434B1B68092B07D1424B1B6862
:101AF000022B02BF0122414BC3F87825FFF7CAFF32
:101B000010B10E223E4B1A60FFF7B4FF20B1002245
:101B10003C4B1A6001225A600022D30003F57F0378
:101B2000D3F80013013108D0D3F800130132D3F8F1
:101B30000433B2F5807F0B60EFD1334BDA69D10704
:101B40003BD5324B1946D3F80024012AFBD1C3F808
:101B50000425D1F80034012BFBD12B4BDA69D207D5
:101B600008D5DA69294922F00102DA61D1F80024A6
:101B7000012AFBD11A6A01320AD11A6A22F0FF0245
:101B800042F020021A62214AD2F80034012BFBD124
:101B900000221E4BC3F80425D3F80024012AFBD1F0
:101BA000BFF34F8F1A491B4BCA6802F4E06213431C
:101BB000CB60BFF34F8F00BFFDE71B6A0133C0D07E
:101BC000134BD3F88C2042F44062C3F88C20D3F836
:101BD000882042F47002C3F88820BFF34F8FBFF310
:101BE0006F8F0D4B0D4A1A6008BD00BFD0ED00E0AD
:101BF000384A00503001FF003401FF00004000501F
:101C0000E4AE03500C4700500080FF0000900350EA
:101C100000ED00E00400FA05041400200090D00359
:101C200070B50026084B53F82040013053F820507F
:101C3000A54200D870BD236820465B68984700B174
:101C400066600C34F4E700BFC0460000104B70B56E
:101C500005461E460F4C9C4204D10E4CB44209D19D
:101C6000002412E062681AB122681268AA420CD0FD
:101C70000C34F0E763680BB90C34EFE723682846AF
:101C8000196802F0AAF80028F6D1204670BD00BFFE
:101C9000C81400205014002008B50B4D4FF020024E
:101CA000EFF3118382F31188BFF36F8F02F046FACE
:101CB000012104460228D8BF084602F04FFA2C62E0
:101CC000FFF7E2F9EAE700BF300600200248034AC6
:101CD0000021121A02F0E2B8000000209006002055
:101CE00008B50648064A0749121A02F0AAF8BDE8E4
:101CF0000840054A0549064802F0A3B8D013002061
:101D00002C150020404B000000000000404B00005C
:101D100000000020012208B50B4B02201A70FFF7CB
:101D20007FFF0A4A0A490B4801F08BFE0320FFF7A8
:101D300077FF00F083FC01F0ABFC074A137B23F034
:101D40000103137308BD00BF8D060020E1470000AA
:101D5000FB4A0000084B0000C405002080B5374B4B
:101D6000A2B083F308880025E023354C012784F8CE
:101D70002230E57725766576A576E576636A314E7D
:101D800043F4E0236362636A43F400236362A56360
:101D9000FFF7E6FAFFF772F94FF0FF33A362E36251
:101DA00007AB6C222946184602F078F8264C8DF8CD
:101DB0002970A0602846FFF733FF3846FFF730FF51
:101DC00000F0ECFB214B66624FF48062CDE90473B6
:101DD000CDE902551E4BCDE900551E49304600F0B5
:101DE00013FC737B23F0040213F01B0F727304D1F6
:101DF000B36913B9304600F01BFA174B0122059363
:101E00000F23CDE903320023144DCDE901330093B4
:101E10004FF4A072124B1349284600F0F5FB6B7B80
:101E2000E56023F004036B730F4B4FF48062C4E949
:101E300006330849064B0348FFF7FEF8D01300208D
:101E400000ED00E0C4050020300600202F4B00000C
:101E5000151D000090060020344B0000580500209E
:101E6000991C0000900A00204806002070B50E4B17
:101E70000E4CA34201D3002070BDD3E9030141EA17
:101E8000000212F003020BD19D685A61AA4201D1EF
:101E90001C33EEE75E6901320E6059610144F5E7DB
:101EA0006FF01500E8E700BFC8140020C814002038
:101EB00010B513460C464FF02002EFF3118182F368
:101EC0001188BFF36F8F426962B1226043691B685A
:101ED0004361836901338361002081F31188BFF37B
:101EE0006F8F0DE01BB923606FF00B00F5E7024622
:101EF000044800F0FDFA18B9034B9B685B69236046
:101F000010BD00BF8E0600203006002070B50446CC
:101F10000D464FF02003EFF3118683F31188BFF3D2
:101F20006F8F02F0B9F880B100212A6881664261A2
:101F3000427BD20603D183690BB900F079F93146AF
:101F4000BDE87040074802F04FB82B6862691A601C
:101F50002B686361A369013BA36186F31188BFF31A
:101F60006F8F70BD8E060020F8B504460F464FF007
:101F70002003EFF3118583F31188BFF36F8FC268DD
:101F800030495AB180688E68B04215D0B7B985F330
:101F90001188BFF36F8F6FF00F000CE08B6893F91F
:101FA0000E3023618B680132E260A36085F31188F3
:101FB000BFF36F8F0020F8BD2369F2E790F90E3070
:101FC00096F90E109942A8BF194621EAE17199428B
:101FD0002BDA00F0A1FA06463B46224629461A486B
:101FE00000F086FA0028E6D04FF02003EFF31185C9
:101FF00083F31188BFF36F8F236821699C4207D058
:1020000033B193F90E309942A8BF194621EAE17124
:10201000A06890F90E30994209D16EB129460A485C
:1020200001F0E2FF6FF00A00C5E70026D4E700F0F8
:1020300073FA0028F2D1F0E785F31188BFF36F8FB0
:10204000F0E700BF300600208E06002038B5836818
:102050000446002B3BD0214A926893423AD1DA7B66
:10206000013ADA73C368012B05D0013BC36000F06D
:10207000C3F8002038BD4FF02003EFF3118583F340
:102080001188BFF36F8F0169806890F90E30994213
:1020900001D000F041FA204601F0FEFFA06080B1BF
:1020A00090F90E20226100228266427BD20603D183
:1020B00083690BB900F0BCF82946094801F094FF88
:1020C000D5E7E06085F31188BFF36F8FCFE76FF03E
:1020D0001500CFE74FF0FF30CCE700BF30060020FF
:1020E0008E06002010B5084C23685BB1FEF7E2FBBA
:1020F0002368064A184410610021BDE810401846C4
:1021000002F02CB810BD00BF680600203006002089
:10211000F8B50D464FF02003EFF3118483F31188D7
:10212000BFF36F8F4FF4004140F2E73600270022E3
:10213000E1FB0067094B30461A6139464FF47A7269
:102140000023FEF77BF8064B1860064B1D60FFF777
:10215000C9FF84F31188BFF36F8FF8BD30060020EC
:1021600068060020640600204FF02003EFF3118181
:1021700083F31188BFF36F8F044B9A68D37B013BC5
:10218000D37381F31188BFF36F8F7047300600203F
:10219000094B03F12802824205D19B688B4202D190
:1021A0004B7BDB0607D1D1E900231A600A68536034
:1021B0000023C1E9003370473006002038B50D4CCC
:1021C000024604F1280001F030FF054600B9E56839
:1021D000A3684AB95A7BD20606D1AA6922B9DA891C
:1021E0007F2A01D9636238BD9D4201D0FFF77AFF93
:1021F0006562F8E73006002010B54FF02003EFF3DA
:10220000118483F31188BFF36F8F084B00209A6805
:10221000D37B0133D373FFF7D1FF84F31188BFF36E
:102220006F8FBDE8104001F0F6BE00BF3006002001
:10223000F8B54FF02003EFF3118483F31188BFF357
:102240006F8F164A114651F8283F8B420CD05BB174
:10225000D66A90F90E5093F90E70AF420BDCB34280
:1022600002D01B68002BF6D1D36A01604360D36AA9
:102270001860D06205E05A68C0E900325A68106000
:102280005860437B63F07F0343730020FFF796FFA2
:1022900084F31188BFF36F8FF8BD00BF30060020B4
:1022A000F8B504464FF02003EFF3118583F311884E
:1022B000BFF36F8F90F90D30002B03DA01461848F9
:1022C000FFF766FF174A02F12801D2E90A308B4274
:1022D0000BD053B194F90E6093F90E70B7420ADC3B
:1022E000834202D01B68002BF6D1C4E90010D36AE8
:1022F0001C60D46205E05968C4E9003159680C607B
:102300005C60637B906863F07F036373031B5842D8
:102310005841FFF753FF85F31188BFF36F8FF8BD66
:102320005806002030060020154A164938B50C68BA
:102330009368A342144603D1BDE83840FFF7D2BEEC
:1023400000250D6010490968B9B1D9897F2914D8D1
:102350000E4993F90E5009688D420EDB0C498B42F1
:102360000BD0996949B91169814203DC1846FFF71E
:1023700097FFE1E7091A116138BD00232361FBE7EC
:102380003006002060060020680600206406002059
:1023900058050020036D70B5044603B1984704F159
:1023A000180001F0B5FE4FF02003EFF3118583F321
:1023B0001188BFF36F8F204601F00DFE0646D8B19D
:1023C00094F90D30002B07DA21461248FFF7E0FEA2
:1023D000637B03F07F0363730F4B9868021B5042CB
:1023E0005041FFF7EBFE637B43F00803637385F313
:1023F0001188BFF36F8F70BD637B9B07F3D52146B8
:10240000A068FFF7C5FE637BA66023F00203637339
:10241000E9E700BF580600203006002038B5044622
:102420004FF02003EFF3118583F31188BFF36F8F13
:1024300090F90D30002B07DA01460948FFF7A8FE96
:10244000637B03F07F036373064B9868031B58425A
:102450005841FFF7B3FE85F31188BFF36F8F38BD86
:10246000580600203006002070B504460D4616467A
:10247000FFF7D4FF637B43F002036373EDB12B6876
:10248000A5609D420CD05BB194F90E2093F90E101B
:1024900091420CDC69688B4202D01B68002BF5D19D
:1024A0006B68256063606B681C606C6005E05A684F
:1024B000C4E900325A6814605C60731C15D04FF494
:1024C000004540F2E730002126EAE6764FF47A72C2
:1024D000C5FB06010023FDF7B1FE0449421C04F1CF
:1024E0001800BDE8704000F03FB970BD37400000F3
:1024F00010B50C461146064A9068064A10601A4606
:10250000FFF7B2FF2046BDE81040FEF7F7BC00BF62
:1025100030060020600600202DE9F84304464FF005
:102520002003EFF3118983F31188BFF36F8F01F05C
:1025300052FD4EB2804668B3174D214605F128077B
:102540003846FFF725FEAB6AA673BB422A460AD07F
:102550004BB1E96A93F90E00B0420BDC994202D00C
:102560001B68002BF6D1D36A27606360D36A1C60B6
:10257000D46205E05A68C4E900325A6814605C60AD
:102580000120FFF71BFE89F31188BFF36F8F4046D0
:10259000BDE8F883A673F6E7300600200021044B5F
:1025A000084603F12802C3E90A22FFF7B1BD00BFC4
:1025B00030060020014B9868704700BF30060020AD
:1025C00010B54FF02002EFF3118482F31188BFF3AE
:1025D0006F8F427B510704D484F31188BFF36F8F50
:1025E00010BD22F0040112F01B0F417303D1836967
:1025F0000BB9FFF71DFE2146BDE81040014801F070
:10260000F3BC00BF8E06002030B587B00E9D044697
:1026100004950D9D03950C9D02950B9D01950A9DBA
:102620000095FEF7E7FC044B9B6813B9236607B0DF
:1026300030BD1B6EFAE700BF300600202DE9F04FD9
:10264000284E294DB04687B0B54205F1300410D36D
:10265000FFF78AFD4FF4004940F2E7360027224C8D
:10266000DFF888A0444521D307B0BDE8F04FFFF75D
:10267000C3BD54F8043C059354F8103C049354F83B
:10268000143C039354F8183C029354F81C3C0193F7
:1026900054F8203C009354E90A2354E90C01FFF755
:1026A000B3FF54F8303CDD642546CDE7616A4B1C2E
:1026B00004D0256821B92846FFF782FF3034D1E7DE
:1026C000B346BC46E9FB01BC4FF47A72002358467E
:1026D0006146FDF7B3FD5146421C05F1180000F0BC
:1026E00043F8EBE7C8140020C8140020374000006E
:1026F000034B1B680BB9FEF7DDB80020704700BF25
:102700006C060020036840B1084A5268904204D029
:102710001BB19A6881680A449A6042681360036832
:102720005A600023C0E90033704700BF081400203E
:102730000B4B10B51C689C4208BF0024FFF7D8FF64
:1027400054B1A368181A20EAE070064B1B6913B154
:102750009842A8BF184610BD6FF00040F5E700BFD3
:10276000081400203006002070B504461646C160EB
:102770004FF02003EFF3118583F31188BFF36F8FC0
:10278000FFF7B6FF012EACBF80190130174BA060D8
:102790001A689A4201D05E6832B95A682360626052
:1027A0005A6814605C600BE09068A168884216DD8E
:1027B000411A91605168C4E9002151680C6054606D
:1027C0001A689A4206D0944204D1FFF7B1FF002163
:1027D000FEF718F885F31188BFF36F8F70BD091AE3
:1027E0009642A160D9D01268D6E700BF0814002035
:1027F0002DE9F04B0446FFF797FD4FF02003EFF370
:10280000118583F31188BFF36F8F214F214EB84696
:10281000DFF884903460D9F8004032684C45D7E93D
:1028200000BC05D024B1A368934214DD9B1AA360B9
:1028300000241BEB02004CEBE271C8E9000134609C
:10284000FFF776FF2146FDF7DDFF85F31188BFF323
:102850006F8FBDE8F08B1BEB03004CEBE371D31AD9
:1028600033600023C7E90001A3602046FFF74AFF59
:1028700085F31188BFF36F8FE36898474FF020030B
:10288000EFF3118583F31188BFF36F8FC3E700BFA8
:10289000000000206C0600200814002038B5074C0A
:1028A000074DAC4201D3002038BD04F1140320468B
:1028B000C4E9053300F0F3FE1C34F2E7C81400202D
:1028C000C814002001F0A6BA0A46002101F0E6BAB9
:1028D00010B5114800F048F800B110BD0F4800F0E5
:1028E00043F80028F9D10E4C204600F03DF80028AE
:1028F000F3D10C4B0C481C6000F036F80146002860
:10290000EBD100F02DF8044608B1204610BD00F0D0
:1029100051F82046FAE700BF1C14002010140020D4
:1029200018140020201400201414002008B50848B2
:1029300000F024F8074800F021F8074800F01EF8DE
:10294000064800F01BF8BDE8084000F00BB800BFD7
:102950001C1400201014002018140020141400204F
:1029600000207047704700BF08B5034B02681B6822
:1029700010689847002008BD2C14002008B5034BB0
:1029800002685B6810689847002008BD2C1400207E
:102990000268024B10689B68184700BF2C14002087
:1029A00008B5034B0268DB6810689847002008BD33
:1029B0002C14002070B5094C094D2069AB6898476C
:1029C00018B1084B08485B6898470021074AEB6834
:1029D00011602069BDE87040184700BF3C1400201A
:1029E0002C14002024140020D8460000700600207B
:1029F000F8B51A4C1A4D0746AB6820699847E8B9F4
:102A0000184E33687FB93BB90120174A1749C2F8FD
:102A100000050A68002AFCD101333360EB682069A5
:102A200098470020F8BD002BF8D0012B08D0013BBF
:102A300033602069EB6898470020F3E70C48F8BD45
:102A40000A4A1368002BFCD1074A6FF07E40C2F897
:102A5000003500F021F83368E9E700BF3C1400209E
:102A60002C1400207006002000008450101984509F
:102A7000E98FFFFF0020704700207047430503D512
:102A80004FF0FF32024B1A60024B1860704700BFD4
:102A900008118450081A8450014B1860704700BF19
:102AA000041A845008B100F003B84FF47500704761
:102AB0000246074803681342FCD021B1054B064883
:102AC0001B680B600360054B00201A60704700BF55
:102AD000001A84500411845008118450081A84503C
:102AE00000F0A0B830B129B10023014403700130D7
:102AF0008142FBD1704700BF2DE9F041ADF51A7D51
:102B00000F4605920021144612A84FF408721E4683
:102B100001F0C4F9002308A819462822069301F001
:102B2000BDF9002F3CD0002E3AD0002C38D0042123
:102B300006A8FFF7C9FE08A82821FFF7C5FE08A8C8
:102B400000F032F878B14FF0FF3512A84FF4087159
:102B5000FFF7C8FF06A80421FFF7C4FF28460DF5BC
:102B60001A7DBDE8F08112AB0DF11C080390CDE990
:102B70000163024605AB08A9CDF8008006A800F065
:102B8000E9FC0028DFD13368A342DCD3D8F8001079
:102B90000546083138462246FFF794FE3460D4E7F4
:102BA0004FF0FF35DAE700BF1C2330B583B002A930
:102BB00041F8043D044600F0B1F90546D8B9019B3F
:102BC0001C2B1BD1D4E9003201210033E16118BF75
:102BD00001230AB143F00203A26832B9E268AAB93C
:102BE000C4E908323BB90D4D09E0E26843F0040343
:102BF00062B9C4E90832284603B030BD084D20460A
:102C00001C21FFF761FE284603B030BD0022284694
:102C100043F00803C4E9083203B030BD0E0CF000E5
:102C2000370CF00010B50C4C236813B10B4B1B682C
:102C30006BB900F031F938B10138062896BF084B5E
:102C4000084853F8200010BD0122044B1A600123EC
:102C50000020236010BD00BF74060020780600200D
:102C6000F8460000FE8FFFFF10B5094C23681BB12A
:102C700001230020236010BD00F07CF80028F7D06D
:102C80000138062896BF034B034853F8200010BDB7
:102C900074060020F8460000FE8FFFFFBFF34F8F41
:102CA0000549064BCA6802F4E0621343CB60BFF3E8
:102CB0004F8F00BFFDE700BF00ED00E00400FA0504
:102CC000014B5B68184700BF24140020024BD0E979
:102CD0000012C3E90012704724140020704700BF9F
:102CE00010B5044620B1BFF35F8F0020206010BDF7
:102CF0000348FFF7E5FFBFF35F8F0020206010BDA2
:102D00003847000010B5044610B10023236010BD01
:102D10000248FFF7D5FF0023236010BD14470000D1
:102D200050B10122D0E8EF3FC0E8E12F0029F9D1EE
:102D3000012BF7D0BFF35F8F0020704770B40B4BAF
:102D40000668C268D0E90154C3E90242C3E90065DC
:102D5000D1E903020E68064BD1E90154C3E90065CD
:102D6000C3E902401A6170BC704700BF2C140020F8
:102D70003C14002010B5FFF77DFE70B9FFF7A8FDE9
:102D800080B9FFF735FE80B9114B1B681B0EF02B85
:102D90000DD00624FFF770FE00E00324FFF7C6FD08
:102DA000204610BD0424204610BD0024F2E7094A45
:102DB000094B12689A4201D00724EBE70120FFF784
:102DC00017FE0028F1D1054B04461860E8E700BF64
:102DD00028198450241A84500000E0200C1A8450D2
:102DE00030B5ADF5157D4FF4087200210CA801F047
:102DF00055F8002302A819462822019301F04EF845
:102E000002A8FFF7D1FE18B105200DF5157D30BDE4
:102E10001C4D4FF0FF312868FFF7BAFD0446F0B9AA
:102E20000020FFF7E5FDB0B90CAA02A901A800F047
:102E3000D5FB04460120FFF7DBFDF0B92868FFF75A
:102E4000AFFD10B11048FFF73BFF2046002CDBD14F
:102E50000DF5157D30BD0D48FFF732FFE4E70C4856
:102E6000FFF72EFF012CDBD12868FFF799FD002822
:102E7000CAD00548FFF724FFC6E70648FFF720FF42
:102E8000DCE700BF201400207047000088470000E6
:102E900058470000A847000008B5FFF7EBFD18B140
:102EA000FFF744FD032008BDFFF712FD68B9FFF7E7
:102EB0009FFD60B9154B1B681B0EF02B12D0FFF75E
:102EC000DBFDFFF733FD062008BD042008BDFFF73A
:102ED000D3FDFFF72BFDFFF783FF00280CBF002079
:102EE000052008BD0A4A0B4B12689A4205D0FFF72D
:102EF000C3FDFFF71BFD072008BD0120FFF778FD8C
:102F00000028E4D1044B1860E5E700BF281984507D
:102F1000241A84500000E0200C1A845018B111B11A
:102F20000B681C2B01D0012070474FF47F033A4AF5
:102F3000D3F8101C91425AD0D3F8102C013256D03D
:102F4000D3F8102C4FF47F030260D3F8141C334ADB
:102F500091425ED0D3F8142C01325AD0D3F8142CFD
:102F60004FF47F034260D3F8182C12F5947F4DD0B4
:102F7000D3F8182C013249D0D3F8182C4FF47F0322
:102F80008260D3F81C1C264A91423CD0D3F81C2CFA
:102F9000013238D0D3F81C2C4FF47F03C260D3F831
:102FA000002C70322DD0D3F8002C013229D0D3F868
:102FB000002C4FF47F030261D3F8042CAF321ED0F3
:102FC000D3F8042C01321AD0D3F8042C4FF47F0329
:102FD0004261D3F8081C134A91420BD0D3F8082C55
:102FE000013207D0D3F8083C83610020704740F6D7
:102FF000FC02A7E740F2373383610020704751227B
:10300000E4E79022D5E742F60412C5E740F6D8621D
:10301000B4E742F2D002A3E7FCF8FFFFD020FFFFA5
:103020000429FFFF37F3FFFFA8B32DE9F0414C1E41
:10303000B4F5047F2CD25BB352B34FF0000CC9003F
:10304000E646654664464F1E03F1FF380CE0AB428E
:1030500016D08E4501D10CF1010CA84516D00134D3
:10306000BC4205F1010518D8610950F8211004F09F
:103070001F06F1401F2E18BF01F00101002CE6D100
:103080000025A8458E464FF0010CE8D16245E6D2F6
:103090000348BDE8F081024870470020BDE8F08198
:1030A000370CF1002DE9F04F8FB00D46DDE91941E5
:1030B0008346002957D12969039100211C60189B80
:1030C0001960002A00F02281814A824B11686A6AE5
:1030D0001B689A4257D10A2955D19BF803300693B1
:1030E0000399042308467C4A0293A2FB000292083B
:1030F000CB0002EB420204F10800A1EB4202013BCB
:10310000DFF8D091DFF800A2049000920593189B9D
:10311000039C1C60002C00F0CC800026049F00F073
:10312000A9FA00230793069BBBF1000F3AD0002DAC
:1031300034D053BB5B000693BBF1000F36D0002D9B
:1031400034D0E3B106A9284600F084FA002800F044
:103150007D81624B984212D0009000F08BFA00986B
:103160000FB0BDE8F08F4FF47F01D1F80C0C0130A7
:103170000CBF4FF40471D1F80C1C03919DE72B6A2E
:1031800073B95648E8E75648E6E706A9284600F02E
:1031900061FA68B1534B9842DED0069B082BC9D127
:1031A0005148D9E7082BFBD05B0006934F48D3E783
:1031B0002946069800F030FA0028EBD1069B082B30
:1031C00000F00E81042B00F03181A3F10203B3FA69
:1031D00083F35B09019301231946454A136042F8C2
:1031E000843C434B19606B6AC9F80030D9F8002061
:1031F0006B6A9A42F5D14FF000084FF0FF30CAF8E1
:103200000080FFF73BFC3B4A3B4B40461A60FFF710
:1032100043FC0A22019839492D4B08601A602A693B
:10322000A8F15538A8FB02126B6A120903EB43039D
:10323000DB0303FB02F3324A9B0913600123CAF844
:1032400000300699DBF800200B0243EA016322F00C
:103250007F421343CBF8003007A800F0CDF90028D7
:1032600098D1284BA8FB04281A681433089253F805
:10327000102CB6EB980F099253F80C2C0A9253F8C5
:10328000082C0B9253F8042C0C921B680D9301D15F
:10329000009B9BB93846182208A9FFF713FB183C7E
:1032A00018370136002C7FF43AAF049B002B40F016
:1032B0009A800023189A1360069B6FE71A463846D7
:1032C00008A9E41AFFF7FEFA009B1F44E9E700BFD4
:1032D0003811845030118450ABAAAAAA310CF100E5
:1032E000300CF100020CF100320CF100350CF10051
:1032F000C4118450FEFFFF0F001184500C11845044
:10330000D8118450141184502C118450BBF1000F3B
:103310003FF44CAF002D3FF449AF01230EA941F813
:10332000203DCBF80020284600F094F900287FF4D7
:1033300013AF2946069800F06FF900287FF40CAF10
:10334000069F082F00F0EB80042F00F0EA80A7F121
:103350000207B7FA87F77F0901221646734B7449B3
:103360001A6018460A60943B06606A6A1A60196817
:103370006A6A9142F8D14FF000086E4B4FF0FF306F
:10338000C3F80080FFF77AFB6B4B6C4A40461A602B
:10339000FFF782FB0A226A496A4B0F601A601A998A
:1033A0002B6901296A6A00F0B1806749A1FB031308
:1033B0001B09012102EB4202D20303FB02F3634A21
:1033C0009B0913605B4B19600699DBF800200B0228
:1033D00043EA016322F07F421343CBF800307FE6DB
:1033E00003230193F7E6039BB3F5047F3FF661AF38
:1033F000DDE9047C204623466E6904E001200133A8
:103400006345144615D85A0957F8222003F01F01C6
:10341000CA401F2918BF02F00102002BEED0A242C1
:10342000ECD101308642EAD149480BE002230193F6
:10343000D1E64FF48063DDE90310AA69FFF7F4FDDC
:1034400000285DD00023189A1360A3E62946069849
:1034500000F0E2F800287FF47CAE069C082C51D0E6
:10346000042C51D0A4F10204B4FA84F464090123B9
:103470001E4619462D4A136042F8843C2B4B1960B6
:103480006B6AC9F80030D9F800206B6A9A42F5D10E
:1034900000274FF0FF30CAF80070FFF7EFFA264B15
:1034A000264A38461A60FFF7F7FA0A222449254BC4
:1034B0000C601A602A6924496B6AA1FB021203EBB3
:1034C00043031209DB0303FB02F3204A9B09136049
:1034D000CAF80060069BDBF800101A0242EA036398
:1034E00021F07F421A43130A03F47F03134323F0AE
:1034F0007F43CBF80030029B013B02937FF407AE81
:10350000002029E60324B2E70224B0E74FF47F034A
:10351000D3F80C1C013106D0D3F80C3C45E7032747
:103520001AE7022718E7162343E700BFC4118450A7
:10353000401184502C11845000118450FEFFFF0F65
:103540000C11845038118450ABAAAAAAD811845007
:10355000360CF1002DE9F0431B4C85B00746DDE940
:103560000D56884620684FF0FF319146FFF710FA5C
:1035700028BB0020FFF73CFAE8B90023CDE900564C
:1035800002934A46414638460C9BFFF78BFD0546A1
:103590000120FFF72DFA50B92068FFF701FA10B1AA
:1035A0000A48FFF78DFB284605B0BDE8F0830848C0
:1035B000FFF786FBF0E70748FFF782FBDDE70648E9
:1035C000FFF77EFBD5E700BF201400207047000006
:1035D000A8470000884700005847000010B50124A4
:1035E00086B005ABCDE901240093002204ABFFF7C0
:1035F00059FD06B010BD00BF08B501464FF480600C
:10360000FFF750FA00230249024A0B60136008BD1D
:10361000C81184502C1184500138072815D8DFE8D0
:1036200000F0100C140814141404CB6800204B6232
:1036300070478B6800204B6270474B6800204B62DC
:1036400070470B6800204B6270470148704700BF0D
:10365000310CF1000B6802E0082B0B6006D8026AFF
:1036600013424FEA4303F7D00020704700487047E9
:10367000310CF10000230449044A0B604FF48060D0
:103680001360FFF7FBB900BF2C118450C4118450A4
:1036900008B5FDF7C3F9BDE80840FDF753B9FF23AE
:1036A0002DE9F74F4568002229464FF00C0A4FF0EC
:1036B000200B0789046805FB07FCC372837A644406
:1036C0000193019B934208DC002319468F4205EBCE
:1036D000030C21DC03B0BDE8F08FBCFBF1F3202B21
:1036E00084BF1F3393FBFBF30AFB02FED0F80C8070
:1036F0004FEA910108EB0E0606F10409C6E90199AB
:1037000021F0030194BFC27248F80E4002F1010299
:1037100088BF04EB8304D4E7C268066802F1040E94
:10372000F41846F803E093680131636093681C6005
:1037300094606346CAE70020704770B50D460446A2
:103740004520A04729465220A04729462346BDE8E8
:103750007040522018472DE9F04F002705460E46CD
:1037600092461C464FF0FF39B846BB4689B09AF8DE
:10377000000010B909B0BDE8F08FBBF1000F07D110
:10378000252800F04E813146A8470AF1010AEEE7EC
:10379000642868D01AD839280BD831285AD22D2855
:1037A00000F04681302846D0252808D13146A84768
:1037B0007AE0582800F0B480632800F02C8131466C
:1037C0002520A84731469AF80000F0E7702800F05D
:1037D0009D800DD8692846D06C2803D16C2F26D146
:1037E0004C27D2E76828EAD1682F20D14827CCE7B8
:1037F000752870D017D87328E1D1226804F1040B22
:1038000011460C4614F8010B002840F0F980B8F17D
:10381000030F40F013818C1AA9EB0404002C00F371
:10382000F5805C4640E078287AD07A28C7D1002F0E
:10383000C5D10746A9E7B9F1000F0EDAB8F1000FBC
:1038400000F0F980A0F13009B8F1000F08BF4FF087
:1038500002089AE7B9F1000FF4DB0A2202FB09091A
:10386000A9F13009F0E77A2F03D1D4F800B004347D
:103870001EE06C2FF9D04C2FF7D14FF0000C4FF019
:10388000FF3B073424F0070303F10804D3E90023C6
:1038900012F1004043F100018C4508BF834506D278
:1038A00031462846FFF749FF4FF0000B6DE793467E
:1038B000BBF1000F06DA31462D20A847CBF1000BF3
:1038C00009F1FF3943465A46CDF800903146284663
:1038D000FCF774FEE8E77A2F02D12268043411E085
:1038E0006C2FFAD04C2FF8D100214FF0FF30073465
:1038F00024F0070303F10804D3E90023994208BF29
:103900009042CDD3CDF800904346DFE731463020DA
:10391000A84731467820A8474FF008094FF0010822
:103920009AF80020702A05D12368043404930023F8
:1039300002930CE06C2FF7D04C2FF5D1073424F014
:103940000702136802F108040493536802930022EB
:103950001023039205924022043A02990498C2F17E
:10396000200CA2F1200ED04001FA0CFC40EA0C0021
:1039700021FA0EFE40EA0E0010F00F0008D1059962
:1039800001B942BB4FF0300C08E0CDF814B0E3E7CA
:1039900009288CBF4FF0570C4FF0300C3146604473
:1039A000CDE90523A847039B01330393DDE90523F4
:1039B000002AEAD1B8F1030F7FF476AF039BC3EB83
:1039C000490BBBF1000F7FF76FAF31462020A847AE
:1039D0000BF1FF3BF5E7591E9945069107DBB8F15E
:1039E000010F06D1314630200792A847079A069B5F
:1039F000B2E7B8F1020FFAD1079231462020F4E77E
:103A000031460292A8472146029AFAE63146202022
:103A1000A847013C02E73146206804F1040BA8479F
:103A2000FFE65F46D8464FF0FF394FF0010BACE69A
:103A30004FF00308A9E64FF00108A6E65C4683466E
:103A4000A3E60FB407B504A951F8040B0191FCF7E4
:103A500007FE03B05DF804EB04B07047044608B5F8
:103A6000084611461A46A047FEF7A4FDFDF79EFC46
:103A70007047FEF71DB80C228368C9B202FB013102
:103A80004B7A23B9087AB0FA80F0400970470220D7
:103A900070470268F8B59768CCB286684FF020038B
:103AA000EFF3118583F31188BFF36F8F0C2262430C
:103AB000B1180B7A1BB3013BDBB20B7213BBB350D3
:103AC0003A444B605368B3B90C23012103FB0473E0
:103AD000DA7A1B8902F150221160002203F150238F
:103AE0001A600C21002001FB0464607285F31188C8
:103AF000BFF36F8FF8BD98470028E5D1F1E76FF06D
:103B00004400F3E70020F1E738B50C24836805464C
:103B100004FB0134012363724FF02003EFF31181A2
:103B200083F31188BFF36F8F23682BB160681A6825
:103B30008342226008BF626081F31188BFF36F8FF8
:103B400003B938BDD3E9012128469047E4E703686B
:103B50002DE9F041D0F808C005469F68CEB24AB1C1
:103B60000C2373435CF803309A425CD013B11B689A
:103B7000002BF9D14FF02003EFF3118083F311886C
:103B8000BFF36F8F0C2171430CEB01031C7A0134DE
:103B9000E4B21C7280F31188BFF36F8F32B34FF021
:103BA00050204FF0030EC0F808E3587AA0B94FF048
:103BB000200EEFF311888EF31188BFF36F8F106022
:103BC000D3F804E0BEF1000F20D15A604CF8012078
:103BD00088F31188BFF36F8F4FF050230321C3F890
:103BE000041318B1D2E9013128469847012C0BD1B2
:103BF0000C237343FB586BB90C23012203FB06769D
:103C0000B37A03F150231A6000200EE0CEF80020B2
:103C10005A60DDE7284698470028EDD1314628460E
:103C2000FFF772FFF0E76FF00F00BDE8F0810022B0
:103C3000FFF78DBF10B50022044601210520FDF7D6
:103C4000C1F90520FDF7AEF94FF050230222C3F869
:103C5000182503220020C3F80423A368C3E9000049
:103C6000A368C3E9030010BD70477047002307B580
:103C700002A800F8043DFEF733FF03B05DF804FB33
:103C8000902908B5134639D10A4601460020FEF7AF
:103C900033FFBDE80840714672467346B7EE000A2E
:103CA000F7EE000AB7EE001AF7EE001AB7EE002A98
:103CB000F7EE002AB7EE003AF7EE003AB7EE004A08
:103CC000F7EE004AB7EE005AF7EE005AB7EE006A78
:103CD000F7EE006AB7EE007AF7EE007A8EF3008C0A
:103CE00010B4F1EE10CA4FF66074C0F6FF740CEA1F
:103CF000040CE1EE10CA10BCF44674476FF01500D6
:103D0000C7E7FEE7FDF7C6B943B2A9B1002B12DB46
:103D100001215B099B0003F1604303F56143D3F884
:103D2000802200F01F0001FA00F022EA0000C3F830
:103D30008002D3F880327047002BFCDB01225B0944
:103D40009B0003F1604303F56143D3F8801200F058
:103D50001F0002FA00F00843E9E700F009B9014644
:103D6000006800F005B908B5FDF79EF9BDE8084008
:103D7000FDF7B6B807B5002101A8FDF7ADFC03B00B
:103D80005DF804FB30B585B09DF808200D890B68FF
:103D90004C68498965F3040261F3471200938DF87A
:103DA000082023F01F03621E134423F01F030F2873
:103DB0000393044605D86946FDF748FB204605B045
:103DC00030BD6FF01504F9E740E800F313F4803FCD
:103DD000D8B208BF6FF0150070470138013910F8EC
:103DE000013F11F8012F934202D1002BF7D11A465F
:103DF000981A704710B55AB10139841810F8012B80
:103E000011F8013FA04201D09A42F7D0D01A10BD5C
:103E10001046FCE7431A934210B500EB020308D3A7
:103E2000024601399A420BD011F8014F02F8014BBA
:103E3000F8E70A4412F8014D8A4203F8014DF9D11E
:103E400010BDF0B581EA0004A50703460BD0013B85
:103E50000A4491421DD1F0BD002AFCD011F8014B5B
:103E6000013A03F8014B9C07F6D10C461D1F8F1831
:103E70003E1B032E08D86FF00305940805FB0422AF
:103E8000A40023442144E2E754F8046B45F8046F8E
:103E9000EEE711F8014B03F8014FDAE70346F0B5FE
:103EA000C9B29C070FD11D4641EA012444EA0444EB
:103EB0009F187E1B032E0CD8940803EB8404134434
:103EC0009C4209D1F0BD002AFCD003F8011B013A45
:103ED000E7E745F8044BECE704F8011BF0E74FF087
:103EE000FF3070470B46826892E8030083E80300C6
:103EF0000020704703689B681B68D3F88004C3F8F0
:103F000080047047036882689B681B68D3F81001BF
:103F100038B1127A00200A700122C3F810011A6029
:103F200070474FF0FF30704782B002AA02F8011DBF
:103F3000002103689B681B68C3F82011C3F844255F
:103F40000122C3F848259A60D3F820110029FBD03C
:103F5000DA6002B0704708B50020FDF709FA08B52D
:103F6000FCF728FFFCF7A6FFBDE80840FEF77CBE83
:103F700070B505460E46FEF71DFB31460446284641
:103F8000FFF7E9FF2046BDE87040FDF70FBAFFF7E5
:103F90006CBE30B50024846141EA020414F00304CD
:103FA000C0E9023201610CD14461A34203D1C0E9EE
:103FB0000000002030BD456901340D6041611144AD
:103FC000F3E76FF01500F5E703460020C3E900337F
:103FD000C3E902007047437BDB0603BF8069B0FA88
:103FE00080F040090020704721B9EFF3058008B93F
:103FF000FCF784BF81F31188BFF36F8F70470346CE
:1040000020B9EFF305820AB9FCF778BF83F3118872
:10401000BFF36F8F70474FF02003EFF3118083F3EE
:104020001188BFF36F8FFFF7EABF0368984214BF90
:1040300018460020704750F8103C70B50446A0F1B7
:104040001805CBB14FF02003EFF3118683F31188ED
:10405000BFF36F8F294650F8100CFEF799F814F84B
:104060000B3C23F0020304F80B3C86F31188BFF3EA
:104070006F8F002344F8103C14F80B3C284623F0C3
:10408000140304F80B3CFFF7A6FF20B12846BDE857
:104090007040FEF7CDB870BD38B54FF02003EFF398
:1040A000118283F31188BFF36F8FFFF7BEFF0446C1
:1040B00082F31188BFF36F8FC8B14FF02003EFF385
:1040C000118583F31188BFF36F8F01468068FEF777
:1040D0005FF8637B23F00203637385F31188BFF3FA
:1040E0006F8F002304F11800A36000F011F8204640
:1040F00038BD10B5029C8373047300230424C3737A
:104100004473C0E90633C0E91333C0E9161210BD89
:1041100010B54FF02002EFF3118482F31188BFF342
:104120006F8F03683BB1FEF7EDFA002084F311882E
:10413000BFF36F8F10BD6FF01500F7E710B54FF0AC
:104140002003EFF3118483F31188BFF36F8FFEF721
:10415000EFFA84F31188BFF36F8F10BD70B504467A
:104160000E464FF02003EFF3118583F31188BFF360
:104170006F8FFEF7DDFA012805DDA04203DD314631
:104180002046FCF73FFB85F31188BFF36F8F70BDAE
:104190007047FFFFD8C0FF7F010000000000000053
:1041A000053D000000000000053D0000000000008B
:1041B000053D000000000000053D0000000000007B
:1041C000053D0000000000000507000000000000A1
:1041D000053D000000000000053D0000000000005B
:1041E000053D000000000000053D0000000000004B
:1041F000053D000000000000053D0000000000003B
:10420000053D000000000000053D0000000000002A
:10421000053D000000000000053D0000000000001A
:10422000053D000000000000053D0000000000000A
:10423000053D000000000000053D000000000000FA
:10424000053D0000000000005907000000000000CC
:10425000053D000000000000053D000000000000DA
:10426000053D000000000000053D000000000000CA
:10427000053D000000000000053D000000000000BA
:10428000053D000000000000053D000000000000AA
:10429000053D000000000000053D0000000000009A
:1042A000053D000000000000053D0000000000008A
:1042B000053D000000000000053D0000000000007A
:1042C000053D000000000000053D0000000000006A
:1042D000053D000000000000053D0000000000005A
:1042E000053D000000000000053D0000000000004A
:1042F000053D000000000000053D0000000000003A
:10430000053D000000000000053D00000000000029
:10431000053D000000000000053D00000000000019
:10432000053D000000000000053D00000000000009
:10433000053D000000000000053D000000000000F9
:10434000053D000000000000053D000000000000E9
:10435000053D000000000000053D000000000000D9
:10436000053D000000000000053D000000000000C9
:10437000053D000000000000053D000000000000B9
:10438000053D000000000000053D000000000000A9
:10439000053D000000000000053D00000000000099
:1043A000053D0000E147000081060000000000001C
:1043B000E1470000E9060000000000009D49000000
:1043C000353C000054440000CF470000990700002E
:1043D00000000000E1470000D515000000000000CB
:1043E000C847000081190000B8460000E1470000FE
:1043F000ED19000000000000F04A00005F3F0000DF
:1044000000000000E14700006D1E000000000000F9
:10441000E14700009D28000000000000DEE61E28A5
:104420004CBBCE8F025B0000DEE61E28EAAC45B82E
:10443000025B0000DEE61E284CBBCE8F025B000054
:104440002F3C0000933A00004F3B000000000000AA
:10445000773A0000000000000000000000010004A6
:1044600000000000000000000401080C170100001B
:10447000070100000701000007010000070100001C
:10448000070100000701000007010000070100000C
:1044900007010000070100000701000007010000FC
:1044A00007010000070100000701000007010000EC
:1044B00007010000070100000701000007010000DC
:1044C00007010000070100000701000007010000CC
:1044D00007010000070100000701000007010000BC
:1044E00007010000070100000701000092490000D9
:1044F000420100009949000005010000A3490000A5
:1045000014010000AC49000015010000B54900008D
:1045100039010000BE49000009010000C94900003E
:104520000A000000D44900000A010000DE49000032
:104530000B010000E84900000F010000F3490000F2
:1045400010010000FE49000011010000094A0000AE
:104550000E010000134A0000210100001C4A000067
:1045600022010000254A0000230100002E4A00001D
:1045700024010000374A0000180100003F4A0000F3
:104580002A010000474A00003A0100004F4A00009B
:104590002C010000574A00001C010000604A000086
:1045A0001D010000694A000017010000734A000065
:1045B000310100007F4A00000401000017010000E3
:1045C000170100001701000017010000170100008B
:1045D000170100001701000017010000070100008B
:1045E00007010000070100000701000007010000AB
:1045F000070100000701000007010000070100009B
:10460000070100000701000007010000070100008A
:10461000070100000701000007010000070100007A
:10462000070100000701000007010000070100006A
:104630000701000007010000070100000000000062
:10464000000200000004000000080000001000004C
:1046500000000000033D0000510E0000110E00009C
:10466000E10D0000C10D0000EC130020D413002068
:10467000E413002000000000DC1300200200000012
:104680008446000000000000E14A0000060000002F
:10469000E0FF0F0000000020E94A000021000000B8
:1046A000E0FF0020053F0000293F0000F53E00002C
:1046B00011180000E53E00000080005001000000DD
:1046C00050140020A4140020B0140020C8140020AE
:1046D000C8140020F5FFFFFF436F756C64206E6FF8
:1046E00074206C6F636B20706F77657220736176D6
:1046F00065206D7574657800FF8FFFFFFF8FFFFFEA
:10470000FE8FFFFFFE8FFFFFFD8FFFFFFC8FFFFF80
:10471000FC8FFFFF43616E277420696E69746961C5
:104720006C697A65206D757465782C2077617320CB
:104730004E554C4C0D0A000043616E277420756E77
:104740006C6F636B206D757465782C2077617320B6
:104750004E554C4C0D0A00004661696C20746F2068
:1047600061637175697265206D757465780A000002
:104770004661696C20746F2072656C656173652099
:104780006D757465780A00004661696C20746F204D
:10479000696E63726561736520504D20636F756E3D
:1047A0007465720A000000004661696C20746F2015
:1047B000646563726561736520504D20636F756E2B
:1047C0007465720A00000000554152545F30007356
:1047D00079735F636C6F636B005365637572650912
:1047E00009004E6F6E2D53656375726509004E6F3B
:1047F0006E2D53656375726500466C617368207237
:104800006567696F6E0909446F6D61696E090950CA
:1048100065726D697373696F6E730A002530327546
:1048200020307825303578203078253035782009CB
:10483000002563004E6F6E2D73656375726520638E
:10484000616C6C61626C6520726567696F6E2030A7
:1048500020706C6163656420696E20666C617368AA
:1048600020726567696F6E202564207769746820FF
:1048700073697A652025642E0A00436F756C642085
:104880006E6F7420696E697469616C697A652073F2
:104890006563757265207365727669636573202838
:1048A000657272202564292E0A005352414D2072F0
:1048B0006567696F6E0909446F6D61696E0909501A
:1048C00065726D697373696F6E730A002530327596
:1048D000203078253035782030782530357809003B
:1048E0005065726970686572616C0909446F6D6129
:1048F000696E09095374617475730A002530327545
:1049000020252D32317325730009534B49500A007D
:10491000094552524F520A00094F4B0A0053504D5D
:104920003A204E5320696D616765206174203078AC
:1049300025780A0053504D3A204E53204D535020B5
:10494000617420307825780A0053504D3A204E5338
:1049500020726573657420766563746F722061746C
:1049600020307825780A0053504D3A2070726570D7
:1049700061726520746F206A756D7020746F204EAF
:104980006F6E2D53656375726520696D6167652E65
:104990000A004E52465F5030004E52465F434C4F25
:1049A000434B004E52465F52544330004E52465FD6
:1049B00052544331004E52465F4E564D43004E52C4
:1049C000465F554152544531004E52465F55415263
:1049D000544532004E52465F5457494D32004E52B4
:1049E000465F5350494D33004E52465F54494D4542
:1049F0005230004E52465F54494D455231004E529E
:104A0000465F54494D455232004E52465F53414134
:104A10004443004E52465F50574D30004E52465F61
:104A200050574D31004E52465F50574D32004E5256
:104A3000465F50574D33004E52465F574454004E28
:104A400052465F495043004E52465F564D43004E1A
:104A500052465F465055004E52465F45475531001D
:104A60004E52465F45475532004E52465F445050C5
:104A70004943004E52465F4750494F544531004E1E
:104A800052465F524547554C41544F5253006D7545
:104A90007465785F696E69742063616C6C6564200D
:104AA00077697468204E554C4C20706172616D6559
:104AB00074657200436F756C64206E6F7420616C56
:104AC0006C6F63617465206D7574657820626566CE
:104AD0006F726520696E697469616C697A696E6765
:104AE00000464C4153485F30005352414D5F300007
:104AF00048575F43433331305F300076322E312EDA
:104B000039392D6E637331002A2A2A20426F6F745F
:104B1000696E67205A6570687972204F53206275FC
:104B2000696C64202573202573202A2A2A0A006DC7
:104B300061696E0069646C6500000000000000009F
:104B400037370000DC14002001000000F0140020C2
:104B500001000000041500200100000018150020CD
:104B600001000000DF3E000000C201000001030060
:104B7000000000000090D00308140020081400205A
:104B8000401400204C140020441400203C14002049
:104B900018140020000000009D2C0000052D0000CE
:104BA000DD2C0000212D0000E12C000088060020F3
:104BB0007C06002084060020000000008006002003
:104BC000A4430000000000000000000004440000B6
:104BD0000000000000000000104400000000000081
:104BE00000000000D44300000000000000000000AE
:104BF000BC430000404400000C000020E0430000E3
:104C0000A4460000F8130020B0430000000000009C
:104C100000000000C8430000000000000000000089
:104C2000F84300000000000000000000EC4300001A
:104C30000000000000000000C8140020C81400207C
:104C400000000000000000000F000000DC14002045
:104C5000DC14002000000000000000000F00000035
:104C6000F0140020F01400200000000000000000FC
:104C70000F000000041500200415002000000000B3
:104C8000000000000F00000018150020181500207B
:104C900000000000000000000F000000FFFFFFFF09
:104CA0000000000000000000000000000000000004
:104CB00000000000000000000000000000000000F4
:104CC00000000000000000000000000000000000E4
:104CD00000000000000000000000000000000000D4
:107FE0007FE97FE9F8F728BE7FE97FE9F8F77CBEF3
:107FF0007FE97FE9FBF744BE0000000000000000BD
:10C0000088180220C9DF0000F535010095DE000028
:10C0100095DE000095DE000095DE000095DE000054
:10C0200095DE000095DE000095DE00008DDD00004D
:10C0300095DE000095DE000039DD0000E5350100E9
:10C0400089DF000089DF000089DF000089DF000050
:10C0500089DF000089DF000089DF000089DF000040
:10C0600089DF000089DF000089DF000089DF000030
:10C0700089DF000089DF000089DF000089DF000020
:10C0800089DF000089DF000089DF000089DF000010
:10C0900089DF000089DF000089DF000089DF000000
:10C0A00089DF000089DF000089DF000089DF0000F0
:10C0B00089DF000089DF000089DF000089DF0000E0
:10C0C00089DF000089DF000089DF000089DF0000D0
:10C0D00089DF000089DF000089DF000089DF0000C0
:10C0E00089DF000089DF000089DF000089DF0000B0
:10C0F00089DF000089DF000089DF000089DF0000A0
:10C1000089DF000089DF000089DF000089DF00008F
:10C1100089DF000089DF000089DF000089DF00007F
:10C1200089DF000089DF000089DF000089DF00006F
:10C1300089DF000089DF000089DF000089DF00005F
:10C1400089DF000000000000000000000000000087
:10C1500000000000000000000000000000000000DF
:10C1600000000000000000000000000000000000CF
:10C1700000000000000000000000000000000000BF
:10C1800000000000000000000000000000000000AF
:10C19000000000000000000000000000000000009F
:10C1A000000000000000000000000000000000008F
:10C1B000000000000000000000000000000000007F
:10C1C000000000000000000000000000000000006F
:10C1D000000000000000000000000000000000005F
:10C1E000000000000000000000000000000000004F
:10C1F000000000000000000000000000000000003F
:10C20000DEE61E284CBBCE8F025B00003C00000027
:10C2100098A400000100000000C0000000C0000061
:10C22000FFFF02910000000000000000000000007D
:10C2300000000000000000000000000053B94AB9EF
:10C24000002908BF00281CBF4FF0FF314FF0FF301E
:10C2500000F07CB9ADF1080C6DE904CE00F006F8F1
:10C26000DDF804E0DDE9022304B070472DE9F04772
:10C270008C46089D04468A46002B4AD18A421746BE
:10C2800062D9B2FA82F64EB1C6F1200E01FA06F377
:10C29000B740B44020FA0EFE4EEA030A4FEA1748B0
:10C2A000230C1FFA87F9BAFBF8FE08FB1EAA0EFB47
:10C2B00009F243EA0A439A420BD9FB180EF1FF3107
:10C2C0002CBF012000209A4202D9002800F02A81C8
:10C2D0008E469A1AA3B2B2FBF8F008FB102200FBBC
:10C2E00009F943EA0244A14507D93C1900F1FF339B
:10C2F00002D2A14500F210811846A4EB090440EADD
:10C300000E4000211DB1F4400023C5E90043BDE803
:10C31000F0878B4208D9002D00F0F2800021C5E99A
:10C32000000C0846BDE8F087B3FA83F100294ED12E
:10C330006345C0F0E880824240F2E5800846002D67
:10C34000E5D0C5E9004AE2E702B9FFDEB2FA82F6BB
:10C35000002E40F099808B1A4FEA124E1FFA82F895
:10C3600001214FEA144CB3FBFEF20EFB123008FB26
:10C3700002F94CEA004CE14508D917EB0C0C02F12C
:10C38000FF3302D2E14500F2CA801A46ACEB090C39
:10C39000A3B2BCFBFEF00EFB10CC08FB00F843EA96
:10C3A0000C44A0450ED93C1900F1FF332CBF4FF0CF
:10C3B000010C4FF0000CA04503D9BCF1000F00F0B8
:10C3C000A8801846A4EB080440EA02409AE7C1F1AD
:10C3D00020048B4002FA01FE0CFA01F6E24020FA3A
:10C3E00004F72CFA04FC00FA01F813433E431F0C37
:10C3F000320C1FFA83F9BCFBF7F007FB10CC00FBF3
:10C4000009FA42EA0C4CE24508D913EB0C0C00F196
:10C41000FF3202D2E24500F289801046ACEB0A0CF2
:10C42000B6B2BCFBF7FA07FB1ACC0AFB09F946EADD
:10C430000C42914506D99A180AF1FF3601D291456E
:10C440007AD8B2464AEA0040A2EB0902A0FB0E6786
:10C45000BA42B446B94602D307D1B04505D2B6EBCD
:10C460000E0C67EB030301389946002D6BD0B8EB37
:10C470000C0362EB090202FA04F4CB40CA4000212B
:10C480001C43C5E9004242E7B740C6F1200201FA69
:10C4900006F3B44021FA02FC4FEA174E20FA02F2EA
:10C4A0001FFA87F8BCFBFEF11A430EFB11CC01FB0F
:10C4B00008F0130C43EA0C4C604507D917EB0C0C41
:10C4C00001F1FF3301D2604533D81946ACEB000CC3
:10C4D00092B2BCFBFEF00EFB10CC00FB08F342EA6C
:10C4E0000C4C634507D917EB0C0C00F1FF3201D25D
:10C4F000634525D81046ACEB030340EA014130E721
:10C500002946284603E7841A6CEB030301209A4668
:10C5100015E702383C4455E702383C44EDE6023A60
:10C52000BC4433E7AEF1020E3B44D2E602389C44F1
:10C5300074E70239BC44C9E7AAF1020A1A4481E748
:10C540000238BC44D7E72946E1E600BF704700BF88
:10C550007FB5484806F06DFE474C484B0646E41A46
:10C56000C4F3C90428B34FF00001012363F30201AF
:10C570006FF3C501424864F38F1106F070FB414828
:10C58000414CC46003F0B6F800286ED13F4806F075
:10C5900009FB214602A802F08BFF21460246002833
:10C5A00044D03B4806F0FEFA4FF47A7005F04AFE9C
:10C5B000FAE701AA01212F4806F085FE054650B191
:10C5C0004FF00001012363F3020166F3C50164F338
:10C5D0008F113048D1E703234FF0000263F30202CA
:10C5E00060F3C50264F38F1201992B4806F044FBF7
:10C5F00002AA02211F4806F066FE50B14FF000016A
:10C60000012363F3020165F3C50164F38F1123482D
:10C61000B3E70299224806F0C5FADDE90121A2FB41
:10C6200001232048110D06F0BDFAA8E71E4806F0C8
:10C63000B9FA1E4C1E4E651C1C4902A802F0B0FF40
:10C6400078B963786BB12378012B04D12946194856
:10C6500006F0A8FAF0E722692946304606F0A2FA69
:10C66000EAE702A803F01CF89EE7134806F09AFADE
:10C670009AE700BF3C56010000540100D853010066
:10C680003F560100B8270220BB560100C0560100EA
:10C69000CF560100535601006E5601007D56010031
:10C6A00097560100A7560100EA5601000800022033
:10C6B0000A570100FF560100225701000B680133A1
:10C6C0000B60014B1B681847D82702202DE9F04F5B
:10C6D00085B00E9C9B46012CB8BF0124012B0CBFDA
:10C6E0003023202316468246884601250A27002249
:10C6F000DFF86C900293B6FBF9F301930AB9B145E8
:10C700001CD8019B414603F13000D047012201357E
:10C71000019B013F09FB13660A23012FB9FBF3F9C3
:10C72000E9D1414606F13000D047BBF1030F02D1F9
:10C73000641B002C0EDC05B0BDE8F08FBC42E7DBCB
:10C74000BBF1020FE4D84146029803920135D0476D
:10C75000039ADDE741462020D047013CE9E700BFCE
:10C7600000CA9A3B014B1860704700BFD8270220CF
:10C77000002313B502AC44F8043D02460B460348BF
:10C78000214606F099F802B010BD00BFBDC60000FA
:10C790004FF02002EFF3118382F31188BFF36F8F04
:10C7A0000121044AC2F8401583F31188BFF36F8F4B
:10C7B000002070470090034020B1034B800143F0FC
:10C7C00001031847704700BF70540100014805F08D
:10C7D00067BD00BFAC29022030B5002287B00D49EB
:10C7E0000D4808F057FC00240E230C4DCDE9024300
:10C7F000CDE90444CDE90044094B4FF440720949A6
:10C80000284605F0D5FD0849284608F0DDFB2046FE
:10C8100007B030BDCDC7000060020220A802022090
:10C8200075CB0000880502204157010008B500F0D3
:10C8300031FA094806F0D0F90423282207490848AC
:10C8400008F0DBFA074B084A4FF400401A60BDE8D5
:10C85000084000F065BC00BF58020220C821022039
:10C860008C020220DC270220172C0100F8B50025DD
:10C870000C4BD3E8EF7FC3E8E25F002AF9D10A4C02
:10C880000A4E361B3611B54200DBF8BD63685B7992
:10C890002BB12368DB6813B1394620469847013530
:10C8A0001034F0E7500202204054010050540100BF
:10C8B000044BD3E8EF2F0132C3E8E12F0029F8D170
:10C8C000704700BF50020220044A054B9B1AB1EB8F
:10C8D000D30F34BF52F8310000207047D853010005
:10C8E00040540100094B4268C31A1B11013310B5B3
:10C8F000137101224368064C5A712278196012B9EB
:10C90000044805F0CDFC0123237010BD4054010004
:10C910007E050220AC290220F8B50F4BD3E8EF4F7B
:10C92000621CC3E8E12F0029F8D12CB90B4D0C4E45
:10C93000761B3611B44200DBF8BD2701EB191B7BD7
:10C9400043B1EB595B6903B1984704220021E81910
:10C95000FFF7C8FF0134EDE7540202204054010004
:10C9600050540100144B37B59842044602D3134B80
:10C9700098421BD3002201A9114805F031F8054661
:10C98000B8B90122019BD3E8EF1FC3E8E02F0028CC
:10C99000F9D1019821461F22043006F070FE7E2353
:10C9A000019C84F8233084F824500434204603B0DA
:10C9B00030BD044CFAE700BF045101008062010061
:10C9C0008C0202204957010048B1054B984205D31B
:10C9D000A03398422CBF00200120704700207047F0
:10C9E000C82102202DE9F84F434B05461B7803B9B7
:10C9F00040B34FF02003EFF3118683F31188BFF3A8
:10CA00006F8F3E4806F0F8F8044686F31188BFF3AE
:10CA10006F8F58B13A4BD3E8EF2F013AC3E8E12FBB
:10CA20000029F8D18DB1204606F0F3F925B9354B30
:10CA30001B680BB1FFF71AFF304806F0DBF8051C46
:10CA400018BF01252846BDE8F88F2F4B1B78ABB9DE
:10CA5000237ADB0712D406F0EBF98146204606F074
:10CA6000B8F90146484606F0DAF80746274B284A47
:10CA7000DFF8B4B09B1AC3F3C90A37B9254E264F65
:10CA80004FF00008BF1B3F1133E0B7FA87F6C6F13D
:10CA90001F063146204606F09FF9204B0246984279
:10CAA00002D31F4B984213D31046FFF78DFF78B97E
:10CAB0001C4B9A420CD0012363F3020860F3C508B3
:10CAC0006AF38F1843464A463146584606F0E8F85E
:10CAD000012303FA06F627EA0607CEE773685B79B7
:10CAE00023B1336821461B683046984708F1010896
:10CAF0001036B845F2DB96E77E0502205802022088
:10CB00004C020220500202207F050220F85301004F
:10CB1000D853010040540100505401000451010059
:10CB2000806201004957010067570100F8B50E4FB8
:10CB30003D7875B9FFF7F0FE0C4C0D4E361B3611E3
:10CB4000B54207DB0020FFF74DFF0028FAD1012393
:10CB50003B70F8BD63685B791BB1236820461B6995
:10CB6000984701351034EBE77F050220405401005F
:10CB70005054010008B5FFF7CFFE05F08BFB0B4BBF
:10CB8000186030B10A4B1B68092B02DD094805F01B
:10CB900087FB084C0020FFF725FF0028FAD14FF053
:10CBA000FF31204605F0A2FBF4E700BF140302208A
:10CBB0004C020220AC290220244B70B51B68418135
:10CBC00005469847224CE860D4E8EF3F0133C4E8BB
:10CBD000E23F002AF8D14FF02003EFF3118683F3F0
:10CBE0001188BFF36F8F1B48294605F0F9FF86F3C4
:10CBF0001188BFF36F8F184B1A787AB14FF020036A
:10CC0000EFF3118483F31188BFF36F8F0020FFF7D8
:10CC1000E9FE84F31188BFF36F8F70BD0F4923685D
:10CC200009680029F9D0012B06D1BDE870404FF406
:10CC30007A710B4805F07EBD0A2BEED1084808F04A
:10CC400035FABDE87040074805F02ABBDC27022012
:10CC50004C020220580202207F0502201403022009
:10CC600060020220AC29022007B504380190D0E808
:10CC7000EF3F5A1EC0E8E12F0029F8D1012B03D164
:10CC800001A9034804F0DAFE03B05DF804FB00BF1D
:10CC90008C020220202302491A46024808F0ADB84F
:10CCA0006822022018030220002373B50A4E02AC4A
:10CCB00044F8043D0120FFF795FE0546FFF7F8FD17
:10CCC00000222146304604F08BFE08B1002DF1D140
:10CCD000019802B070BD00BF1803022007B5002202
:10CCE00002A941F8042D054804F07AFE10B1FFF7BF
:10CCF000DBFF0190019803B05DF804FB18030220EC
:10CD0000F0B5047A457A85B014F0010401904FEA39
:10CD1000151510D0019B1A7A920706D55B6904ACF1
:10CD2000184D44F8043D039B2BBB01A9154804F0A2
:10CD300085FE05B0F0BD002DECD0264617E031464B
:10CD400006F04AF80746FFF73FFE78B13CB9019B71
:10CD50002946186905F063FF04460028DAD024FA52
:10CD600006F3DB0702D53846FFF77EFF0136AE42F9
:10CD70000198E4D3CEE71E682146284604F05EFE03
:10CD80000396D0E7180302200EB403B503AB53F8A3
:10CD9000042B01460448019305F08EFD002002B0EB
:10CDA0005DF804EB03B07047E53101002DE9F04F69
:10CDB00011F0020485B0064690469DF8387001F0E7
:10CDC000010901F0080507D011F0440F37D11A46C8
:10CDD0003249FFF7D9FF0446B9F1000F0AD0304BB2
:10CDE000304953F82720304B3046002A08BF1A46F6
:10CDF000FFF7CAFF3DB12D4B2D4953F82720304690
:10CE0000FFF7C2FF0546B8F1000F44D0012303FA33
:10CE100007F7284B17F0100F274F18BF1F46BDF814
:10CE200040109DF83C00FFF74FFD39460246304662
:10CE3000FFF7AAFF2844204405B0BDE8F08F1F4A41
:10CE4000116831B31E4A4FF4616E14684FF47A7C56
:10CE5000B3FBF4F3B3FBF1F4B4FBFEF20EFB124EA2
:10CE600001FB14340CFB04F4B4FBF1FB4FF03C0A5F
:10CE700001FB1B440CFB04F4BEFBFAF3B4FBF1F121
:10CE8000CDE901B10AFB13E100910E49FFF77CFFE8
:10CE9000A1E708469FE7084FC1E700BFE35701003D
:10CEA00078540100E05F0100D55701008C54010067
:10CEB00008580100DA570100DE5701003403022050
:10CEC00038030220EC57010038B50C46E10705464F
:10CED00003D5084A0849FFF757FFE20608D4A3061E
:10CEE0002846BDE838404CBF04490549FFF74CBF10
:10CEF00038BD00BFD5570100E05F0100C7570100F2
:10CF0000C65701002DE9F0479846089B0446DD0608
:10CF10000E46174605D499064CBF29492949FFF703
:10CF200033FF0025DFF8A49045452ADB0025DFF814
:10CF3000A080DFF8A090DFF894A0AF422ED9725DF8
:10CF400049462046FFF720FF0135102D1FD11E490D
:10CF50002046FFF719FF0025DFF87080DFF8789092
:10CF6000AF4227D9725D4946A2F120035F2B28BF4B
:10CF70002E222046FFF708FF0135102D13D1BDE802
:10CF8000F08749462046FFF7FFFE0135CCE76A07E8
:10CF9000D3D151462046FFF7F7FECEE74146204663
:10CFA000FFF7F2FED0E76B07DAD141462046FFF7E4
:10CFB000EBFED5E741462046FFF7E6FEDCE700BF83
:10CFC000C7570100C6570100A35701004D6101007A
:10CFD0004B6101009D570100A55701002DE9F04765
:10CFE00017460A7A8B7AD24313F007048AB00546B3
:10CFF0000E46D2B21BD04989C3F3C20389090291FC
:10D00000CDE9004302F00102F3683946FFF7CEFE96
:10D010008146337ADA070CD42946304605F078FF8A
:10D020004CB3224639462846FFF74EFF23E0A1467F
:10D03000EFE734BB2746EB6806AA0693A9683B4690
:10D04000304605F051FF069A6B681A603AB1AB683A
:10D05000134413F8014CA4F10A035C425C412846D6
:10D0600006F0B3F8069B1F44002BE4D11CB1154910
:10D070002846FFF789FE284606F0A7F80AB0BDE863
:10D08000F087304605F0D4FE0F4902462846FFF7E8
:10D090007BFE4FF000084FF0100A05AA434606A990
:10D0A0003046CDF814A005F01FFF059A002AB8D02D
:10D0B0004B46009706A92846FFF724FF059B984496
:10D0C000EBE700BFA8570100E05F010073B5D0E9AE
:10D0D00000435D6842F20F738B4228BF0B460D4A36
:10D0E0000521684602F06CF906462B4620460B22C5
:10D0F000094905F000FF2B4632466946204605F0F7
:10D10000FAFE2B461B220549204605F0F4FE02B02C
:10D1100070BD00BF01620100C9570100AA5701009C
:10D1200001230021074A10B5074C1360A04204D820
:10D1300001B11360054B186010BD40085B00012170
:10D14000F4E700BF3803022040420F0034030220FE
:10D1500008B5034804F0AAFA024B586008BD00BFA6
:10D160002E58010044030220014806F02EB800BFEB
:10D17000B85401000148FFF7A9BF00BFB85401002F
:10D1800010B50C46084605F01BFE214604480F2248
:10D19000FFF724FF2046BDE8104005F03ABE00BF6F
:10D1A000B854010008B5044807F042FE034B0020C4
:10D1B000C3E9003308BD00BF58030220500302201A
:10D1C000F8B5074606F07CFA0646114D4FF0FF31E0
:10D1D000104804F061FC2C68AC420ED100240D48CC
:10D1E00004F0CCFC2046F8BDA06806F069FAB04215
:10D1F00006D06B689C42F1D02468002CF4D1EDE796
:10D200003246A168384606F070FA0028F1D1E6E708
:10D21000500302205803022010B504464FF0FF319E
:10D220001B4804F039FC0CB1A068B0B901234FF0E1
:10D230000001184A63F30201174B6FF3C5019B1AF3
:10D24000DB08164863F38F1105F009FD6FF0150434
:10D250000F4804F093FC204610BDFFF7B1FF70B1FA
:10D2600001234FF000010B4A63F302010A4B6FF3F5
:10D27000C5019B1ADB0863F38F110948E4E7094BEA
:10D280005A68236062605A6814605C600446DFE795
:10D2900058030220D8530100E05301004658010012
:10D2A0005F5801005003022010B50B4B88B0CDE948
:10D2B00000320123CDE903310146059204AACDF8DD
:10D2C00008D0CDE9062351F8040B436802AA1C6874
:10D2D00006ABA04708B010BDFD58010038B5036982
:10D2E0000C469D680B4895F8201006F019F848B9CF
:10D2F000611E04290AD8DFE801F0030609060500CB
:10D30000EB69136038BD4FF40073FAE76FF0150056
:10D31000F8E700BFF558010070B50546846810486D
:10D3200004F0C4F94FF404530E4A2060C4E9012309
:10D330000D4804F0BBF9102301266361AB6820613E
:10D340000A4883F820600561FFF766FFD4E904020C
:10D35000436800211C683346A446BDE8704060471E
:10D360004D590100801A060053590100E0270220A0
:10D370002DE9F047074688B08846164607F07CFE40
:10D38000002300F5FA7006900793384605F0B8FFC1
:10D39000FF2804461BD106A805F0D8FF0028F4D1C9
:10D3A00002234FF000022B4963F302022A4B60F381
:10D3B000C5025B1ADB08214663F38F12274805F08C
:10D3C0005BFC6FF03B04204608B0BDE8F087002806
:10D3D000F9DBFE283AD100254FF00109DFF880A0E3
:10D3E000731B402B28BF4023394608EB0502CDE9CB
:10D3F00000A3CDE9042304ABCDF808D0CDF80C9000
:10D40000CDE9063951F8040B436802AA1C6806AB43
:10D41000A04704460028D6D14035AE42E0DC0322C6
:10D4200006A93846FFF740FF04460028CBD19DF8F7
:10D4300018309DF819503246414645EA032505F05B
:10D44000BBF9854218BF6FF08904BCE76FF0040494
:10D45000B9E700BFD8530100205401005A59010018
:10D46000FD58010070B505460E4605F0F5FF04466F
:10D4700060B9284605F086FF192E044603D80449F2
:10D48000F140CB0702D4284605F03AFF204670BD94
:10D490000006060308B5FFF7E5FFBDE808400146B2
:10D4A000014805F03DBF00BF3D5901002DE9F74F90
:10D4B00015460E4698460021044605F03DFFDFF86C
:10D4C000F4B0A844C6EB4529454509D14FF0000A00
:10D4D0002046012105F030FF504603B0BDE8F08F33
:10D4E000237E002B5FD106EB090218212046FFF7AF
:10D4F000D1FFB0F1000AEBDBFE2302AF07F8043DD9
:10D5000001223946204605F096FF82460028DFD1E9
:10D510004FF400723146204605F08DFF8246002808
:10D52000D6D14FF40072314605F046F90222030AC3
:10D530008DF80500394620468DF8043005F07BFF54
:10D5400082460028C4D1204605F0DAFE014618487C
:10D5500005F0E6FE82460028BAD1204605F045FFD8
:10D5600082460028B4D102460D21204605F074FF02
:10D5700082460028ACD1204605F004FF01465846FB
:10D5800005F0CEFE0746204605F0BAFE824620464C
:10D5900005F0B6FE002F08DBBAF1000F98D106F5B2
:10D5A0000076013590E72A469FE7BA4690E700BF2C
:10D5B000ED5801003D59010003692DE9F0419C68D7
:10D5C000AB4B92B06360012384F8203007F054FD28
:10D5D0004FF4A01300F59C500830A64DA64E0290C3
:10D5E00003930121204605F0A7FE0A222946204682
:10D5F00005F021FF0021204605F09EFE0022204676
:10D600001146FFF72FFF011E55DB012904D03046DC
:10D6100005F086FE00284ED14FF4D5720821204631
:10D6200005F01AFF064620B908A9204605F0C3FEFA
:10D630000646002E13DB012E05D031468E4805F03C
:10D640006FFE064658B9089BDAB2AA2A30D103F415
:10D650007063B3F5807F14BF6FF0220600260122AD
:10D660003B212046FFF7FEFE051E2BDB012D05D0DA
:10D670002946814805F054FE054618BB002E0CBF14
:10D680004FF080450025002237212046FFF7EAFEB3
:10D690002A4629212046FFF7FDFE002800F0E18000
:10D6A00002A805F053FE0028EDD16FF03B0509E01C
:10D6B0006FF00106D3E702A805F048FE002890D1DC
:10D6C0006FF001052046012105F036FE284612B014
:10D6D000BDE8F08102A805F039FE98B100223A2198
:10D6E000204605F0B9FE18B901A9204605F063FEF1
:10D6F0000146304605F014FE05460028E2D1019BA4
:10D70000002BE7DA019B13F0804309D123764FF415
:10D71000007210212046FFF7BDFE054610B1D1E78B
:10D7200001232376002209212046FFF7B3FE054698
:10D730000028C7D1102220460DEB0201FFF718FE8A
:10D7400005460028BED19DF810309B0904D0012B5E
:10D7500078D06FF02205B5E79DF8155005F00F055C
:10D76000A5F10903022BF4D80DF1160005F0BDFD5B
:10D770009DF819209DF81A30C0F38B3043EA02233C
:10D78000C3F3C2131D440130073D00FA05F5E561FE
:10D790004FF003084FF00002384B394EE169F61A9A
:10D7A00068F302026FF3C502C6F3C90666F38F126F
:10D7B000C90A344805F060FA00220A212046FFF722
:10D7C00069FE054600287FF47DAF102220460DEB50
:10D7D0000201FFF7CDFD054600287FF473AF4FF03F
:10D7E00000079DF8103068F3020708939DF8113088
:10D7F00060F3C50709939DF812300DF119000A93E3
:10D800009DF8133066F38F170B939DF814300C932B
:10D810009DF815300D939DF816300E939DF8173036
:10D820000F939DF81830109305F05FFD3B46119063
:10D830000A2208A9144805F066FA144B84F820500F
:10D8400063603FE70DF1160005F04FFD41F20F0355
:10D85000C0F3150098427FF67CAF01308002E06192
:10D8600096E70190002E7FF44DAF034E36E700BFE0
:10D87000801A0600FD5801003D590100D8530100EF
:10D880002054010088580100A358010000093D0000
:10D890002DE9F0411F4603690D469C68144894F831
:10D8A0002010164605F03CFD28B93B462946204687
:10D8B00005F0F2FDD0B110F13C0F04D0431D02D0B1
:10D8C00010F18A0F12D10D2100222046FFF7E2FD50
:10D8D00094F82010064805F023FD38B93B4632463F
:10D8E00029462046BDE8F04105F0D6BDBDE8F081EF
:10D8F000F55801002DE9F0411F4603690D469C686B
:10D90000144894F82010164605F00AFD28B93B4645
:10D9100029462046FFF7CAFDD0B110F13C0F04D0D4
:10D92000431D02D010F18A0F12D10D210022204692
:10D93000FFF7B0FD94F82010064805F0F1FC38B967
:10D940003B46324629462046BDE8F041FFF7AEBDD2
:10D95000BDE8F081F55801000A2838B50446074DA6
:10D9600004D1286843680D215B689847286843689C
:10D97000E1B25B689847204638BD00BF90030220A3
:10D9800010B5044C204601F015FD2046BDE81040BE
:10D99000FEF7E8BE59D9000008B5044803F086FE3A
:10D9A000034B1860FFF7ECFF002008BD2E58010064
:10D9B0009003022003682DE9F041D0F808C0054625
:10D9C0009F68CEB24AB10C2373435CF803309A428D
:10D9D0005BD013B11B68002BF9D14FF02003EFF39C
:10D9E000118083F31188BFF36F8F0C2171430CEB0F
:10D9F00001031C7A0134E4B21C7280F31188BFF376
:10DA00006F8F22B34FF0030E2248C0F808E3587A14
:10DA1000A0B94FF0200EEFF311888EF31188BFF3F9
:10DA20006F8F1060D3F804E0BEF1000F20D15A6070
:10DA30004CF8012088F31188BFF36F8F0321154B39
:10DA4000C3F8041318B1D2E9013128469847012CD4
:10DA50000CD14FEA061857F808306BB90122474439
:10DA6000BB7A03F1804303F5A0431A6000200EE067
:10DA7000CEF800205A60DDE7284698470028EDD10F
:10DA80003146284605F088FDF0E76FF00F00BDE84D
:10DA9000F08100BF0050004010B500220446012173
:10DAA000052000F093F9052000F080F90222074BD1
:10DAB0000020C3F818250322C3F80423A368C3E990
:10DAC0000000A368C3E9030010BD00BF0050004080
:10DAD00008B5104B1A6862B10F4AD2F80423D10777
:10DAE00007D500220D481A608368597A09B905F0F4
:10DAF00053FD0B4B1A6862B1074AD2F80423920710
:10DB000007D5002201211A600448BDE8084005F04D
:10DB100043BD08BD0051004000500040D8280220FD
:10DB20000451004000220D4BC3F840214FF0200269
:10DB3000EFF3118182F31188BFF36F8F084AD3F896
:10DB400004051368C01A20F07F400344136081F37A
:10DB50001188BFF36F8F04F055BD00BF0050014026
:10DB6000AC03022070B5154803F0A0FD10B3436864
:10DB700001211B689847002401264FF480334FF49D
:10DB800000120F4D3146C5F80845C5F84065C5F887
:10DB900004330C4B15201C600B4BC3F8802122462C
:10DBA00000F014F9152000F001F92046074B1E6023
:10DBB0002E6070BD4FF0FF30FBE700BF8D590100B4
:10DBC000005001404051014000E100E00850014098
:10DBD00070B5264EB0F1FF3F08BF30464FF020032E
:10DBE000EFF3118483F31188BFF36F8F204BD3F8C9
:10DBF0000455204B1B68EA1A22F07F42B2F5000F51
:10DC00001AD2411E21EAE171B142A8BF3146501C2F
:10DC10000844B04294BF18189819451B25F07F4559
:10DC2000134A20F07F43022DC2F8403506D984F311
:10DC30001188BFF36F8F70BD0021E8E7D2F804357B
:10DC40000D49C31A23F07F435D1E8D4205D94FF461
:10DC500000120A4BC3F80021E9E7012B02BF023092
:10DC600020F07F40C2F84005E1E700BFFEFFFF0063
:10DC700000500140AC030220FEFF7F0000E100E005
:10DC80004FF02002EFF3118382F31188BFF36F8FFF
:10DC9000064AD2F80405064A1268801A20F07F402E
:10DCA00083F31188BFF36F8F704700BF00500140AE
:10DCB000AC0302204FF02003EFF3118283F31188AD
:10DCC000BFF36F8F0649074B0868D3F8043582F31A
:10DCD0001188BFF36F8F1B1A23F07F4318447047DE
:10DCE000AC0302200050014004488168406A884229
:10DCF00003D003494FF080520A6070473C05022070
:10DD000004ED00E0094A0A49936809685866996673
:10DD100008494B6843F080534B60002383F311881C
:10DD2000BFF36F8F9368986E704700BF3C05022069
:10DD30000856010000ED00E012498A684FF0280003
:10DD40001044EFF3098C80E8F01F202080F3118845
:10DD5000BFF36F8F0C4F4FF000664A6A8A603E60D7
:10DD6000506E0023536680F3118804B5104605F009
:10DD700048FCBDE8044002F1280090E8F01F8CF355
:10DD8000098870473C05022004ED00E01EF0040FF6
:10DD90000CBFEFF30880EFF30980816911F8021CD2
:10DDA0000229FFD001B505F021FC01BD43B2002BD3
:10DDB00008DB012200F01F0002FA00F0024A5B09B2
:10DDC00042F82300704700BF00E100E043B2002B9F
:10DDD00001F10101A8BF03F160434FEA4111B8BF4F
:10DDE000054BC9B2ABBF03F5614300F00F0083F8E8
:10DDF00000131954704700BF14ED00E073B51E46C0
:10DE00000A9B05460093099B8C1807F0E2F80B4A21
:10DE1000A4F1200323F0070322F001029A61069A7D
:10DE20001E605A60079A9A60089ADA604FF0807212
:10DE3000DA61AB6400236B6602B070BDBF2B0100DA
:10DE4000F8B505460C4617461E4600F0F9FB0A4B8E
:10DE50003C4428469D6024F0070405F0D2FB304680
:10DE600084F30988002163B681F31188BFF36F8FB3
:10DE70000022002304F0A3FE3C05022001491022E9
:10DE80000A60704710ED00E0404080F3118830BF19
:10DE9000704700BFEFF30880EFF30981724601B5C8
:10DEA00000F082FA01BD00BFF7B507460C46002915
:10DEB0003DD001264FF00003204A214D66F30203B6
:10DEC000AD1AC5F3C9056FF3C50365F38F13ADF83C
:10DED0000030D1E901231B48096804F0F9FE4FF036
:10DEE000000366F302036FF3C50365F38F13ADF808
:10DEF0000030D4E90423E168134804F0E9FE4FF050
:10DF0000000266F302026FF3C50265F38F12E16946
:10DF10000E4804F0B1FE4FF0000266F302026FF308
:10DF2000C50265F38F12A169094804F0A5FE2146D8
:10DF3000384603B0BDE8F04003F0DEBBD853010023
:10DF400010540100B7590100E6590100155A0100AB
:10DF5000245A010030BFFFF7FDBF00BF08B5084BD2
:10DF6000084A23F07F039360BFF34F8FBFF36F8F97
:10DF700003F048FC03F050FC00F030FB03F08AFC97
:10DF800000C0000000ED00E001B572B60B4A106A57
:10DF900000281EBF0021116206F02DFF62B6EFF3CC
:10DFA0000580A0F110004FEAC0000549014409C9ED
:10DFB0009847BDE801400349084700003C0502209E
:10DFC00004510100E9DC000004F004FE202080F38D
:10DFD000118808484FF40061401880F30988EFF376
:10DFE00014800221084380F31488BFF36F8FFFF77A
:10DFF000B5FF0000C819022070B54FF000010126DE
:10E00000404B414C66F30201E41A6FF3C501C4F3BF
:10E01000C9043E4D64F38F113D4804F020FEAA6A06
:10E0200092010AD54FF0000166F302016FF3C501BA
:10E0300064F38F11374804F012FEAB6ADB010BD595
:10E040004FF00001012363F302016FF3C50164F394
:10E050008F11314804F003FE2C4DAA6AD6020BD56D
:10E060004FF00001012363F302016FF3C50164F374
:10E070008F112A4804F0F3FDAB6A18030BD54FF05B
:10E080000001012363F302016FF3C50164F38F11F3
:10E09000234804F0E4FD1D4DAA6A51030BD54FF04F
:10E0A0000001012363F302016FF3C50164F38F11D3
:10E0B0001C4804F0D4FDAB6A9A030BD54FF0000165
:10E0C000012363F302016FF3C50164F38F11164856
:10E0D00004F0C5FD0D4DAB6ADB030BD54FF000011D
:10E0E000012363F302016FF3C50164F38F110F483D
:10E0F00004F0B5FDAB6A00206FEA03436FEA1343F7
:10E10000AB6270BDD85301001054010000ED00E077
:10E11000B25B0100CA5B0100DD5B0100F75B01003F
:10E12000215C01003F5C0100645C01007E5C010039
:10E130002DE9F0410E464FF001084FF000013D4B34
:10E140003D4C68F30201E41A6FF3C501C4F3C9043E
:10E150003A4D64F38F110746394804F080FDAA6AEE
:10E16000D1060AD54FF0000168F302016FF3C50133
:10E1700064F38F11334804F072FDAB6A1A070BD5B4
:10E180004FF00001012363F302016FF3C50164F353
:10E190008F112D4804F063FD284DAB6A9B0720D5F5
:10E1A0004FF001084FF0000168F302016FF3C50161
:10E1B00064F38F11254804F052FD696BAB6A1806B1
:10E1C0000FD54FF0000268F302026FF3C50264F34B
:10E1D0008F121F4804F050FD1FB1AB6A23F080037B
:10E1E000AB62164DAA6AD2070BD54FF0000101238E
:10E1F00063F302016FF3C50164F38F11154804F056
:10E200002EFDAB6A9B060BD54FF00001012363F393
:10E2100002016FF3C50164F38F110F4804F01FFD75
:10E220000020064B9A6A9A6A42F0FF029A623070A6
:10E23000BDE8F081D85301001054010000ED00E06A
:10E24000DA5A0100F05A0100235B0100365B01003D
:10E250004E5B0100645B0100835B01002DE9F0412E
:10E260000E464FF001084FF00001444B444C68F358
:10E270000201E41A6FF3C501C4F3C904414D64F30C
:10E280008F110746404804F0EAFCAA6AD1040AD577
:10E290004FF0000168F302016FF3C50164F38F11C1
:10E2A0003A4804F0DCFCAB6A1A050BD54FF00001CC
:10E2B000012363F302016FF3C50164F38F11344846
:10E2C00004F0CDFC2F4DAB6A9B0520D54FF0010823
:10E2D0004FF0000168F302016FF3C50164F38F1181
:10E2E0002C4804F0BCFCA96BAB6A18040FD54FF0A6
:10E2F000000268F302026FF3C50264F38F1226482E
:10E3000004F0BAFC1FB1AB6A23F40043AB621D4DAD
:10E31000AB6A59050BD54FF00001012363F30201ED
:10E320006FF3C50164F38F111C4804F098FCAB6ACD
:10E3300013F4807314D04FF00001012363F3020142
:10E340006FF3C501164864F38F1104F088FC0020B8
:10E350000C4A936A43F47F4393623070BDE8F081C6
:10E36000AA6A9204F3D54FF00001012262F3020180
:10E3700063F3C50164F38F110A48E6E7D85301003F
:10E380001054010000ED00E0525A0100685A0100EB
:10E39000235B0100795A0100925A0100A75A01003B
:10E3A000C25A0100835B01002DE9F041704B8AB035
:10E3B0005F68064688461446C7F30807002585F3BC
:10E3C0001188BFF36F8F02F07F43B3F17F4F2CD1E1
:10E3D00012F0010329D1620604D4230723D546464F
:10E3E000002512E001224FF0000162F3020163F305
:10E3F000C501604A604B61489B1ADB0863F38F11CB
:10E4000004F02DFC14F00405E9D100238DF8073049
:10E41000FB1E092B00F28E80DFE803F00972766F95
:10E420008C8C8C8C8C7A0125EFE72E46EDE74FF033
:10E4300001084FF0000100244E4B4F4F68F30201DA
:10E44000FF1A6FF3C501C7F3C90767F38F114C4873
:10E4500004F005FC464A8DF80740D36A13F0020326
:10E4600024D04FF0000168F3020164F3C50167F3A3
:10E470008F11444804F0F3FB9DF807309BB920222C
:10E48000314602A805F050F9099B002D6AD0C3F36C
:10E49000080222B96FEA53236FEA4323099302A9C2
:10E4A0002046FFF701FD0AB0BDE8F081D46A14F000
:10E4B0008044E4D04FF0000168F3020163F3C5012A
:10E4C00067F38F11304804F0CAFB304B1B7833B12F
:10E4D00040460DF10701FFF72BFE0446CCE72C4B1D
:10E4E0001B782BB140460DF10701FFF7B7FEF4E7AB
:10E4F000284B1C88A4B2002CBED0FFF77DFDECE7B2
:10E500000DF107010020E6E70DF107010020ECE71F
:10E5100001234FF00001174A63F30201164B6FF31A
:10E52000C5019B1ADB0863F38F111B4804F097FBAE
:10E530000024A1E701224FF000030E4962F3020319
:10E540000D4A1648521A1649D2086FF3C50362F3F2
:10E550008F130F2FC8BF0146A7F11002114804F016
:10E560009FFBE5E723F4FF7323F0010396E700BF69
:10E5700000ED00E0D853010010540100A95C010037
:10E58000CC5C0100E35C0100045D010028ED00E0CB
:10E5900029ED00E02AED00E0235D01006E5D010041
:10E5A000595D0100875D0100024A536943F0100381
:10E5B0005361704700ED00E0BFF34F8F0549064BF4
:10E5C000CA6802F4E0621343CB60BFF34F8F00BF11
:10E5D000FDE700BF00ED00E00400FA050023202164
:10E5E0000348C2180133412B82F80013F9D1704758
:10E5F00000E100E038B505464FF02003EFF3118449
:10E6000083F31188BFF36F8F03F090FC0A4B9B6874
:10E61000AB420BD1094B5A68C2F3080212B920462B
:10E62000FFF770FB5A6842F080525A602046BDE8FE
:10E63000384006F041BC00BF3C05022000ED00E080
:10E6400010B50E4B88B002930D4B0E4C03930E4B3E
:10E6500008A8049302AB40F81C3D0C4A2346012154
:10E6600000F056F900230793094B0121E41A05A88D
:10E670000593069400F056F908B010BD0000022082
:10E68000000000000000042006000100000002203D
:10E690000000022010B50B680C7A23F01F0304F071
:10E6A0001F021A43CB68640923F01F03044943F097
:10E6B000010343EA44038860CA600B6110BD00BFD8
:10E6C00090ED00E008B54FF000020123084963F324
:10E6D0000202084B6FF3C5025B1ADB08014663F3C5
:10E6E0008F12054804F0C8FA6FF0150008BD00BF8E
:10E6F000D853010008540100E45D01002DE9F04FFA
:10E700000746884614460026604D85B0464541DAE6
:10E7100057F82630D3F80490B9F1000F5DD0B9F165
:10E720001F0F24D919F01F0F21D1D3F800A01AF020
:10E730001F0F1CD1504604F08FFF834609EB0A00DF
:10E74000013804F089FF834528D06FF0150B0123B1
:10E750004FF000024E4963F302024E4B6FF3C502C5
:10E760005B1ADB0863F38F1259464B480EE0012316
:10E770004FF00002464963F30202464B6FF3C502B5
:10E780005B1A3146DB08454863F38F1204F074FAD4
:10E790006FF01504204605B0BDE8F08F1BF1160F91
:10E7A000D5D0631E5B45D2DBC5F808B0E868C5F874
:10E7B00008B02B6957F8261020F01F0043F01F0AFD
:10E7C000D1E900321A44984202F1FF3918D1CA4502
:10E7D00005D15FFA8BF004F01CFF013696E7C5F80F
:10E7E00008B0EB6822F01F0203F01F031A43EA602F
:10E7F000E0B204F00EFF10F1160FC9D0441CECE794
:10E80000C5F808B02A69013B23F01F0302F01F027C
:10E810001343CA45E0B22B61EBD004F0FAFE10F1CD
:10E82000160FB5D0C5F808B0EA689DF808300AF1AF
:10E83000FF3A62F304038DF808302B699DF8082035
:10E840005B0863F3471257F826308DF80820D3E9A8
:10E8500000130B44009323F01F03441C5344A3EB09
:10E860000903E4B223F01F030F2C039308D92046B9
:10E87000FFF728FF10F1160F044689D00134ACE7EA
:10E8800069462046FFF706FFF8E700BF90ED00E07D
:10E89000D853010008540100C15D01009E5D0100D4
:10E8A0000522034B5A60BFF34F8FBFF36F8F704742
:10E8B00090ED00E0BFF35F8F0022014B5A6070477C
:10E8C00090ED00E070B50E4D2E68102E15D8002486
:10E8D000FFF7F0FF0B4B0C4A1A63A64205D10B4B16
:10E8E0001E70FFF7DDFF002070BD6968204601EB58
:10E8F0000411FFF7CFFE0134EFE74FF0FF30F3E7ED
:10E900001055010090ED00E0AAFF440081050220AF
:10E9100010B5034C2278FFF7F1FE207010BD00BF48
:10E92000810502202DE9F74F894607460026DFF8CA
:10E930009080DFF890A0214C4E4519DAD7F804B04A
:10E94000BBF1000F36D03B681846019304F084FEFB
:10E95000019B05460BEB0300013804F07DFE1423F8
:10E96000854203FB06F306D06FF0150248F803203A
:10E9700003B0BDE8F08F15F1160F48F80350F7D03B
:10E980009AF80020AA42F3DDA5604344A560E06840
:10E99000197B60F3040119732169187B490861F33D
:10E9A00047101873E26822F01F025A60226922F0B1
:10E9B0001F021A6101360C37BEE700BF90ED00E080
:10E9C000B00302208105022070B50C4B0E461C7866
:10E9D0000546234600210A4A0F2B0BDD094B191D62
:10E9E0001868FFF757FE224631462846BDE87040BA
:10E9F000FFF784BE936011610133EDE781050220CA
:10EA000090ED00E0B00302202DE9F04F1E460023F8
:10EA10009DB0CDE9020101931078531C069358B1C3
:10EA2000252800F089800399029B9847013040F027
:10EA30000B844FF0FF33019301981DB0BDE8F08FB8
:10EA4000232C70D065D8002CF6D0202C0C9B08BF4E
:10EA500001230C93CDF81880DDF81880BB4818F816
:10EA6000014B214604F01EFE0028E9D12A2C6AD170
:10EA70003268331D002A0792BEBF5242079201221C
:10EA80001E46B8BF0D92069A547802F102082E2C49
:10EA90007ED198F800302A2B77D1356808F101082B
:10EAA000043698F8004008F101082146A848274696
:10EAB00004F0F8FD00286ED008F10103682F0693DA
:10EAC00098F8004007D1682C05D1482708F10203C7
:10EAD00098F801400693672C7CD8652C80F03A8129
:10EAE000472C5CD8452C80F03581002CA4D0252CF7
:10EAF00000F0A68303992520029B9847013098D007
:10EB000003992046029B9847013092D0019B023323
:10EB10009CE32D2C0DD0302C08D02B2C099B08BF4A
:10EB20000123099396E70123059393E701230893B3
:10EB300090E701230D938DE7002308930C9309932D
:10EB40000D93059388E7A4F13003092B07909ED815
:10EB50000A22DDF8188018F8014BA4F13003092BC4
:10EB600095D8079B02FB0344A4F13003CDE906834B
:10EB7000EFE7904601FB0535303D424612F8013B78
:10EB8000A3F130000928F4D98BE700250A21F4E726
:10EB90004FF0FF3589E7CDF8188007469BE7632CD7
:10EBA00059D021D8582CA5D1331D6F2C049331682E
:10EBB00015AF40F01B83059B002B00F00B83302327
:10EBC0008DF85430002940F00E838DF855108B4697
:10EBD000012726E0702C00F0E88227D86E2C00F088
:10EBE000CF82E1D8692C85D13468331D002C049381
:10EBF00080F29E802D2361428DF854300DF155072F
:10EC000038460A2204F0DEFD099B074415A83F1A86
:10EC1000002B40F01E830C9B002B40F01A834FEA20
:10EC2000D47B002DC0F21A8315AE1EE0752CBBD02C
:10EC3000782CB9D0732C7FF45DAF002DB8BF6FF086
:10EC400000450027331D36680493BD4240F0BD8265
:10EC50000025AB4609E04FF0000B01275D46331D50
:10EC6000049333681CAE06F81C3DA5EB070A00258B
:10EC7000A846A946DA442AEAEA7A079B0AEB07047F
:10EC80001C1B0D9B13B9002C00F3078306EB0B0331
:10EC90009E4240F00483534613F1FF3380F00B8310
:10ECA000A7EB0B07B9F1000F00F02A833078F219B7
:10ECB000A0F130010929A2EB060340F207834A467E
:10ECC000002A40F00E83A3EB0909B8F1000F18D019
:10ECD00006EB090316F8012B079303991046029BD4
:10ECE0000592984701303FF4A4AE059A079B2E2A5F
:10ECF000A3EB0609EED14346002B00F30383A9EBF7
:10ED000008099DB1307806EB0908A0F13003092B02
:10ED1000A8EB060940F203832E2800F00083A846E2
:10ED2000B8F1000F00F30483A9EB0509B14412E325
:10ED3000099B23B12B238DF8543021465EE70C9BB1
:10ED40000BB12023F7E7214615AF59E70A5E010012
:10ED5000105E0100073626F00706D6E90001C20260
:10ED6000904606F108030493CB0243EA505300286F
:10ED700023F0004971F10003C1F30A56CDE910896F
:10ED800042DA2D218DF854100DF1550740F2FF7134
:10ED90008E4254D158EA0903A4F1410407F103005B
:10EDA00042D1192C3AD849233B704E237B7046231D
:10EDB0000025A846A946BB70FD7015AFC01B099B76
:10EDC000002B40F0DA810C9B002B40F0D6819DF89F
:10EDD00054B0ABF12D03D3F1000B4BEB030B1CAB89
:10EDE0005B4413F81C3C08EB0907303B2F44092B0C
:10EDF000074400F23782089B002B00F03982079B02
:10EE000015AEA3EB070A36E7099B0BB12B21B9E737
:10EE10000C9B0BB12021B5E715AFB7E769233B7019
:10EE20006E237B706623C3E7192C99BF4E234122C2
:10EE30006E23612294BF3B703B707A70B8E7462C1A
:10EE400048EA060049EAE67108BF662450EA010371
:10EE500000F0DA80002E7AD0DDE910231046A6F209
:10EE6000FE38002643F000410DF1700969E90C01FC
:10EE700018F1020F7ADB6FF0004A4FF0000BB8F187
:10EE8000000F00F3A48010A808F1010804F0BAFCF8
:10EE9000B8F1040FF7D1002D04F0DF03B8BF062549
:10EEA000472B40F0B980F21C02DBB54280F2AF8004
:10EEB000023CE4B2002D00F07382059B013D002B63
:10EEC00040F06E82002DD4BF4FF0000A4FF0010ACF
:10EED000662C40F0678215EB060840F1A3801023F2
:10EEE00066244FF000080F9300224FF000630DF1ED
:10EEF000700969E90A2318F1FF3880F09580DDE98F
:10EF00001023DDE9120112EB000843EB0109CDE902
:10EF1000108909F070484FF0000958EA090306D03B
:10EF200010A804F082FC10A804F06CFC0136662CDA
:10EF300040F0C480002E7DDC30233B70059B07F140
:10EF4000010B002B40F08D80994685E0013E18EBC7
:10EF5000080849EB0909B8F1000F79F10003F5DA67
:10EF6000CDE9108978E7484604F04CFCDDE910A0B3
:10EF700000230B9300230A90BC4ADDE90ABC6345D9
:10EF800008BF5A4508F10108EDD305224FF0000CE7
:10EF9000AAFB02AB02FB00BBCDE910AB013E002394
:10EFA00000216FF00040994208BF584506D2BCF1DD
:10EFB000000F3FF45DAFCDE910AB59E71AEB0A0A39
:10EFC0004BEB0B0B08F1FF384FF0010CE7E710A8F3
:10EFD00004F02BFCDDE910014FF0000C08F1FF38C4
:10EFE000013600239B4508BF8A4506D2BCF1000FBD
:10EFF0003FF445AFCDE9100141E70018494108F160
:10F00000FF384FF0010CECE70026B0463BE7059BCC
:10F01000AD1B23B9662455E74FF0000A58E74FF0BF
:10F02000000A58E76624BFE1484604F0FEFB04F0FE
:10F03000E9FB60E7BB460F9B002B07DD0FA910A87B
:10F0400004F023FC013E0BF8010BF4D1059B002BCF
:10F0500040F09D81B1461E46002D04DC4FF00008B3
:10F0600020E04FF000092E220BF101038BF8002065
:10F07000002E00F09381002D1EDDC6F10008A8458A
:10F08000A8BFA846A5EB08059B4606E00FA910A857
:10F0900004F0FBFB013D0BF8010B002D02DD0F9B83
:10F0A000002BF3DCBAF1000F1ED1002315AF8BF853
:10F0B0000030ABEB070082E69B46CFE70FA910A814
:10F0C00004F0E3FB059B3028387018BF06F1FF36CB
:10F0D000002B3CD1002D3ADC07F1010BBAF1000FF7
:10F0E00048D04FF00009C8461BF8012C0BF1FF3344
:10F0F000302A3DD02E2A08BF9B46002504F0DF03AE
:10F10000452BD2D1002EB4BF2D232B235A46B8BF96
:10F110007642632E02F8024B8BF801300ADD64213F
:10F1200096FBF1F301FB136603F130000BF10302D0
:10F130008BF802000A2196FBF1F3934601FB13665C
:10F1400003F1300030360BF8020B5670ADE72E237A
:10F1500007F1020B7B70002DC0DD0F9B002BBDDD86
:10F160000FA910A804F091FB013D0BF8010BF2E789
:10F170009B46B9E7D146D046C0E74FF0010B2EE6DB
:10F18000324652F8043B682F049206D06C2F09D007
:10F19000482F07D1019A1A7001E0019A1A80049E43
:10F1A000069A39E4019A1A60F9E7331D049347F689
:10F1B0003003316810220DF15600ADF8543004F0E0
:10F1C00001FB4FF0020B871C2BE5F35D002B43D0B6
:10F1D00001373AE538460822C71B04F0F3FA074422
:10F1E0004FF0000B1DE50DF15500F4E7752C05D12E
:10F1F00038460A2204F0E6FA0746F1E7059BEBB130
:10F2000047F630030DF15606ADF854301022304663
:10F2100004F0D8FA582C0BD13B461A78A2F16101C0
:10F2200019299CBF203A1A7013F8012B002AF4D137
:10F23000059BF71B07444FEA430BF2E43E46E5E724
:10F2400003992046FFF7F0BB019B0133019304961D
:10F25000A5E74FF0010BE4E41D46FAE40025A846BB
:10F26000A946C8E515AE4FF0000A06E53233333340
:10F2700015AEDDF820A000E505930399029B202040
:10F2800098470130059B3FF4D4AB13F1FF33F3D221
:10F29000019A224401921C46F8E42346F5E70593BF
:10F2A0000399029B16F8010B98470130059B7FF4E8
:10F2B000EFACFFF7BEBB05930399029B3020984744
:10F2C0000130059B7FF4E8ACFFF7B3BBDDE9023109
:10F2D0000592984701303FF4ACAB16F8010F059A40
:10F2E000E6E405930399029B302007929847079A1A
:10F2F000013002F1FF32059B7FF4E2ACFFF799BBCE
:10F30000B946E2E405930399029B30209847059B98
:10F31000013003F1FF337FF4EFACFFF78ABBDDE987
:10F320000231984701303FF484AB16F8010FECE44A
:10F3300003993020029B9847013008F1FF387FF491
:10F34000EFACFFF776BB039916F8010B029B9847C9
:10F3500001303FF46EABA9EB0603002BF3DC019BFD
:10F36000002C5B449B46D34407EB0B0301937FF7D0
:10F3700016AF2344019314F1FF34FFF410AF039947
:10F380002020029B98470130F5D1FFF752BB2E2277
:10F39000B14600260BF101038BF80020B04673E65E
:10F3A0004FF0000A05F10108102398450F93A8BFFC
:10F3B000984699E5014B1860704700BFF42702207A
:10F3C0000CB41FB509B90DF10300CDE9020107AB7B
:10F3D000069A02A905480193FFF716FB0022029B3B
:10F3E0001A7005B05DF804EB02B07047C738010031
:10F3F000014802F0C3BB00BFD40302204FF0FF312D
:10F40000014802F049BB00BFD403022008B50448FC
:10F4100005F00EFD034B0020C3E9003308BD00BF1B
:10F42000D4030220CC0302202DE9F74F01900846B7
:10F4300015468A4604F044F94FF000098346FFF769
:10F44000DDFF1A4A4F4614689046944208BF0024D4
:10F450005CB9FFF7CDFF1FB3019B1F601DB30020F8
:10F46000BB692B6003B0BDE8F08FA669B14511D828
:10F47000B3450FD3012E04D91AF806202F2A00D045
:10F4800042B93246E168504604F02FF9002804BF23
:10F49000B1462746D8F804209442DAD02468D7E74A
:10F4A0006FF00100DEE72846DCE700BFCC03022056
:10F4B00073B506460D46A1B901234FF00001304A4D
:10F4C00063F302012F4B6FF3C5019B1ADB0863F353
:10F4D0008F112D4803F0C3FB6FF01504204602B0D6
:10F4E00070BD084604F0ECF80028E5D02B782F2BEF
:10F4F000E2D12649284604F0EBF8044658B9FFF754
:10F500007DFF234A74601368934208BF0023336071
:10F51000FFF76EFFE2E70022294601A8FFF784FF0C
:10F52000041E11DA01234FF00002154963F30202B1
:10F53000144B6FF3C5025B1ADB081649164863F3D8
:10F540008F1203F099FBC9E7019B7360DB691B6AAB
:10F55000002BC3D0294630469847041EBEDA01234B
:10F560004FF00002064963F30202064B6FF3C50237
:10F570005B1ADB0863F38F1221460848E1E700BFFE
:10F58000D8530100F0530100F05E0100345F010028
:10F59000CC030220235E0100045F0100365F0100FE
:10F5A00043682DE9F04107460E4613B3DB695B6AF9
:10F5B000002B50D0DFF8E4804D1C7B683146DB69BE
:10F5C00038465B6A9847041E4BDB737873B1337817
:10F5D000012B0BD14146284604F07AF80028ECD0E4
:10F5E0002949284604F074F80028E6D02046BDE8F2
:10F5F000F08104680CB94C70F8E7FFF7FFFE234B6D
:10F600001C6898469C4208BF00245B680CB92546DC
:10F6100013E03A68A24216D101253046E1680C2277
:10F6200000F8015B294404F02AF80023D8F80420EC
:10F630007373944233610AD02468FFF7D9FE6DB129
:10F640003C600024D2E79C4203D02468DEE71C46DD
:10F65000F3E70024DBE76FF01504C7E76FF0010460
:10F66000C4E701234FF00002094963F30202094B8A
:10F670006FF3C5025B1ADB0863F38F12214606485D
:10F6800003F0FAFAB2E700BF505F0100CC0302209A
:10F69000D8530100F0530100535F01009B57010054
:10F6A00038B54468054614B90460204638BDE3699E
:10F6B0009B6AA3B19847041E13DA01234FF000029E
:10F6C000094963F30202094B6FF3C5025B1ADB08B9
:10F6D00063F38F122146064803F0CEFAE5E76FF098
:10F6E000150400236B60E0E7D8530100F0530100DC
:10F6F0002E5E0100F8B5044608B1C3689BB901232A
:10F700004FF00001524A63F30201524B6FF3C501FF
:10F710009B1ADB0863F38F114F4803F0A0FA6FF0D8
:10F7200015063046F8BDFFF769FE237A012B03D892
:10F730004A4A52F82370A7B901234FF00001444A06
:10F7400063F30201434B6FF3C5019B1ADB0863F3BC
:10F750008F11434803F083FA6FF00106FFF748FE6C
:10F76000DFE7E06803F0ACFFA061E06803782F2BCF
:10F7700012D001234FF00001354A63F30201354BEB
:10F780006FF3C5019B1ADB08364863F38F1103F052
:10F7900066FA6FF01506E1E703F092FF0128E8D959
:10F7A000FB6A73B901224FF0000162F3020163F3B7
:10F7B000C501274A274B2C489B1ADB0863F38F119E
:10F7C000E5E72A4D2E68AE421AD1FB6A20469847DB
:10F7D000061E34DA01234FF000021D4963F30202D2
:10F7E0001C4B6FF3C5025B1ADB0863F38F123146C3
:10F7F0001F4803F041FAB1E76B689E42E5D03668D6
:10F80000002EE2D0A269B3699A42F5D1F168E068AE
:10F8100003F06BFF0028EFD101234FF000010C4AE9
:10F8200063F302010B4B60F3C5019B1ADB0863F322
:10F830008F11104803F013FA6FF00F068EE76B6814
:10F84000256063606B68E7611C606C6086E700BFE1
:10F85000D8530100F0530100495E0100C4030220A7
:10F86000675E01008E5E0100A45E0100CC030220F1
:10F87000DC5E0100BF5E010038B504460D46FFF7AF
:10F88000BDFD012C15D901234FF000010B4A63F394
:10F8900002010B4B6FF3C5019B1ADB0863F38F1159
:10F8A000084803F0DCF96FF01504FFF7A1FD2046CE
:10F8B00038BD054B43F824500024F6E7D853010027
:10F8C000F05301006D5F0100C403022001490020D4
:10F8D000FFF7D2BFF827022030B587B0481C694631
:10F8E000154605F038F8044680B928469DF80830DA
:10F8F0000DF10901C3F3001300F8013B03F0B5FE5D
:10F90000009B2B61044B185707B030BD1328F9D961
:10F910006FF00400F8E700BF915F010008B5481CD4
:10F9200005F02BF9132896BF024B6FF00400185610
:10F9300008BD00BF915F010008B5481C05F0D0F874
:10F94000132896BF024B6FF00400185608BD00BF85
:10F95000915F010030B5541C87B00D4620466946C2
:10F9600004F0F9FF48B9204605F0BAF828B1132889
:10F9700008D96FF0040007B030BD2146681C05F0BF
:10F98000ACF9F4E7014B1856F5E700BF915F0100B1
:10F990000122C16808B51144002001F0BDF9132807
:10F9A00096BF024B6FF00400185608BD915F01002E
:10F9B000012210B5C168ADF5027D0446114400690D
:10F9C00001F0AAF90D2810D14FF40073E0680093FC
:10F9D000002202AB0921013001F0C6F928B9012249
:10F9E000E1682069114401F097F913288EBF6FF088
:10F9F0000400024B18560DF5027D10BD915F010009
:10FA000038B50546006804F07CFF044629460548E1
:10FA100002F014F8132C96BF034B6FF00400185734
:10FA200038BD00BF74290220915F010030B587B056
:10FA30000C460068694604F06DFF054668B90DF193
:10FA40000901601C03F011FE607848B19DF8083090
:10FA5000C3F300132370009B2361132D284603D8A2
:10FA6000034B185607B030BD6FF00400FAE700BF33
:10FA7000915F010037B505460C46002201A90D48EB
:10FA800001F0AEFF014670B92C22019803F079FE17
:10FA90000198611C286004F001FF132806D8064B6A
:10FAA000185603B030BD6FF00B00FAE76FF004009A
:10FAB000F7E700BF74290220915F010038B50546C1
:10FAC000006804F05FFE04462946054801F0B6FFD1
:10FAD000132C96BF034B6FF00400185738BD00BFBE
:10FAE00090290220915F010008B5006804F016FE1D
:10FAF000132896BF024B6FF00400185608BD00BFD4
:10FB0000915F0100012A08B50FD0022A11D09AB9DD
:10FB1000002911DB0068C3688B420DD304F03FFE5F
:10FB200013280CD8074B185608BD03685B691944A5
:10FB3000EEE70368DB68FAE76FF01500F4E76FF0B3
:10FB40000400F1E7915F0100F7B5054600680F4634
:10FB5000C66804F024FE28B1132815D96FF00400FC
:10FB600003B0F0BDBE423446286802DD04F07CFFDD
:10FB7000F2E73146476904F012FE0028ECD18DF817
:10FB80000300BC4203DB0020064B1856E8E701AB3C
:10FB900001220DF10301286804F004FD0028DBD1E7
:10FBA0000134EEE7915F010007B5006801AB04F096
:10FBB000F9FC30B1132806D8044B185603B05DF891
:10FBC00004FB0198FAE76FF00400F7E7915F01008A
:10FBD00007B5006801AB04F055FC30B1132806D816
:10FBE000044B185603B05DF804FB0198FAE76FF078
:10FBF0000400F7E7915F010037B505460C46002287
:10FC000001A90D4801F0ECFE014678B928220198BF
:10FC100003F0B7FD019813222860611C04F059FB22
:10FC2000132806D8054B185603B030BD6FF00B00F3
:10FC3000FAE76FF00400F7E790290220915F0100D6
:10FC400008B5094B1A786AB90121312019700521CC
:10FC5000FEF7BCF83120FEF7A9F84FF00042034B45
:10FC6000C3F80423002008BD8205022000100340D1
:10FC7000F0B5036882689B684D4C187901F01F034A
:10FC800043EA40130020D4F80453EDB200F5A27605
:10FC900054F82660C6F30426B34269D125FA00F66B
:10FCA000F60765D5850005F1804505F54435D5F89D
:10FCB000106526F00106C5F81065012505FA00F06B
:10FCC000C4F808033B4D05EB8305D5F8000220F48A
:10FCD0004030C5F800029068C84010F0010046D0DE
:10FCE000D068C84010F0010041D05069C84010F001
:10FCF000010049D09069C840C0073DD41069D2695D
:10FD0000C84022FA01F100F0010001F0010188422F
:10FD10000CBF02210121002505F5A27254F8220032
:10FD200010F003002AD1AF0007F1804202F54432FF
:10FD3000D2F810651B0226F4473626F44076C2F846
:10FD40001065D2F8106503F4F85343EA01411A4BE9
:10FD50003143C2F81015D851D2F8103543F00103E1
:10FD6000C2F81035012303FA05F5C4F80453F0BDB9
:10FD7000013008288AD1A5E70321CCE70135082DF9
:10FD8000CAD16FF01200F2E71369D269534023FA27
:10FD900001F111F0010F14BF4FF400324FF4403263
:10FDA000D5F8003223F440331343C5F80032DEE7C0
:10FDB0000010034000258440001103402DE9F74F57
:10FDC0008046856803F47040B0F5804F1E4649D0E8
:10FDD0002CDCB0F5805F3DD0B0F5405F3ED060BB1D
:10FDE00006F44077B7F5807F3ED0A7F500746342F4
:10FDF0006341012919BFD4B2A1464FF01F09002465
:10FE00004FF0010B06F0010C4FEA4C0747EA0C07D4
:10FE100047EA0020DFF8C8A040EA830706F00203A3
:10FE2000A14523D2002003B0BDE8F08FB0F5E04F2C
:10FE300016D005DCB0F5A04F0ED06FF01500F2E73C
:10FE4000B0F5404F04D0B0F5504FF6D10720C7E7CA
:10FE50000620C5E70120C3E70320C1E70420BFE770
:10FE60000520BDE70220BBE70323C2E7D8F8002046
:10FE70009268117904F01F0242EA411280324AF876
:10FE80002270A9680BFA04F2002B25D01143A96057
:10FE90006969B0064CBF114391436961A969700655
:10FEA0004CBF11439143A961296970074CBF1143AD
:10FEB00091432961E96930064CBF0A4321EA0202F5
:10FEC000EA61214640460193FFF7D2FE0028AAD1FD
:10FED0000134E4B2019BA3E721EA0201D7E700BFA6
:10FEE000002584404E492DE9F0410D68002D61D078
:10FEF0004C4B00269A681B68DFF834E19F68D2E912
:10FF000002030340D2E90504204323EA00033868D2
:10FF1000D4691269006954404440012023EA040472
:10FF20009BBB0B60002301269C463F483F4FD0F807
:10FF3000042306FA03F111420ED0D91989000A6888
:10FF400052B103F5A27250F82220C1F800C0C2F3EA
:10FF5000042206FA02F214430133082BE7D15CB302
:10FF6000304FD7F80880D8F8001029B30E68D8F8B9
:10FF70000C308A682340134203D04B68224638462F
:10FF80009847CEB131463668F1E703420FD097F873
:10FF900004C006F01F0242EA4C120EEB8202D2F8B5
:10FFA00000C223EA00032CF4403CC2F800C2013630
:10FFB0004000B5E72C46B5E785B101240025194B73
:10FFC000DFF86CC09A681B689E68D2E902130B4088
:10FFD000D2E90510014323EA01030BB9BDE8F08122
:10FFE0001C421AD0307905F01F01D76941EA40114F
:10FFF00010690CEB81017840E84010F0010F14BF4C
:020000040001F9
:100000004FF400374FF44037D1F8000223EA0403DD
:1000100020F440303843C1F8000201356400DCE7C9
:100020007C1103402C2902200010034040C4001022
:100030000025844010B50446002201210B20FDF765
:10004000C5FE2368114A9868234600F10C0101F0AF
:10005000C3F90F4B984214D001234FF000020D4911
:1000600063F302020C4B6FF3C5025B1ADB0863F308
:100070008F1223680948196802F0FEFD6FF00F0027
:1000800010BDA06803F01AFD0020F9E72D01010062
:100090000000AD0BD853010030540100C35F0100D4
:1000A0007FB58568EA6B6B6C8AB9002B33D11C462F
:1000B00000222846114603F0D7FC6C6205F11400BB
:1000C00002F0EEF8002385F84C3004B070BD23B385
:1000D0009342194628BF11460068AC6B80680094B3
:1000E0008668B14228BF3146A964C4B1002A18BF4E
:1000F0000A4601922A6C02929AB1002B18BF0B4655
:1001000000226946039301F009FA074B9842DCD0BC
:100110006FF00404CCE71946DEE71146DCE722461F
:10012000E7E71346ECE700BF0000AD0B007838B5F9
:100130000D4600285BD18C68E36B93B1A26C9A42A8
:1001400029D901234FF00001294A63F30201294B09
:1001500060F3C5019B1ADB0863F38F11264802F098
:100160007EFD636C93B1A26C9A422AD901234FF0B1
:1001700000011F4A63F302011E4B6FF3C5019B1A76
:10018000DB0863F38F111C4802F069FD2846BDE8C7
:100190003840FFF785BF9B1AE36363B9E36A013B0D
:1001A000E36263B1A36A03F10802A2629A68DB68A2
:1001B000A263E363D5E7A36B002BD2D01344A36300
:1001C000CFE79B1A636463B9636B013B636363B1FD
:1001D000236B03F1080222639A68DB68226463647C
:1001E000D4E7236C002BD1D013442364CEE738BD71
:1001F000D853010030540100A55F01002DE9F047FC
:1002000007468068884616461D4604304FF0FF3189
:1002100002F06CF8BC682368984500F0BE80B8F81E
:100220000430386813F0010C18D001234FF000029D
:10023000884963F30202884B6FF3C5025B1ADB083F
:10024000016863F38F12854802F016FD6FF0150503
:10025000201D02F025F82846BDE8F08713F00802BB
:1002600010D001234FF000017A4A63F302017A4B68
:100270006CF3C5019B1ADB08794863F38F1102F018
:10028000EEFCE3E713F4C0510ED001234FF0000160
:1002900063F3020162F3C5016F4B6E4A71489B1A0A
:1002A000DB0863F38F11EAE7C3F34513082B0FD084
:1002B00001234FF0000263F3020261F3C502664BB3
:1002C000644969485B1ADB0863F38F121146D6E76D
:1002D000D8F80020654B9A420FD801234FF0000256
:1002E00063F3020261F3C5025B4B5A4960485B1A33
:1002F000DB0863F38F121146C1E7D8F80830D0F855
:100300000890C4F80080002B6FD0186800286CD0CB
:100310005A684368D3F800A00123D0472268936845
:10032000B2F90420D3E90001D243D20F03F093FBCA
:10033000B8F80430D9F80010980703F0040265D526
:10034000002A0CBF02220322022AC3F3001361D049
:10035000032A62D0012A01D143F00203C1F85435C7
:10036000444AD8F8003093425AD9434A93425AD962
:10037000424A93425AD9424A93425AD9414A9342F5
:100380005AD902F5741202F5106293428CBF4FF0F5
:1003900000434FF08043C1F82435012384F84C30EA
:1003A000002E4CD033687268A362E2621A685B6800
:1003B000A263E363002D47D02B686A6823636263FE
:1003C0001A685B682264636400220121626220462D
:1003D00003F04AFB3846FFF763FE4FF0FF3104F1AC
:1003E000140001F083FF656A32E703234FF0000138
:1003F000184A63F30201184B6FF3C5019B1ADB081F
:1004000063F38F11204802F02AFC91E7003218BFF5
:10041000012299E743F00403A0E743F006039DE7B8
:100420004FF00073B7E74FF08063B4E74FF000631D
:10043000B1E74FF08053AEE74FF00053ABE7C4E9AC
:100440000A66C4E90E66B5E7C4E90C55C4E910555F
:10045000BAE700BFD853010030540100E35F010048
:1004600005600100246001004760010047E80100C9
:10047000766001008FD003001FA107003F420F00EC
:100480007F841E00FF083D00A7600100024B0B6047
:1004900001231360704700BF08040220F8B50D4621
:1004A000164604F0A2FC31460746B6FBF0F4284697
:1004B00003F026FBD8B1B5FBF7F307FB1353B3B931
:1004C00007FB14679FB9ACB14FF0FF310A4801F048
:1004D0000DFF04F08AFC0446284600F053FF361B4B
:1004E0002544F9D1044801F0DBFE3046F8BD6FF039
:1004F0001500FBE72046F9E71004022010B50122A1
:100500000648114604F052FD04F072FC044C2060D1
:1005100004F06BFC6060002010BD00BF10040220DE
:100520000804022070B50D461946284616461C469A
:1005300003F0E6FAF8B1A9071DD1A2071BD1ECB16F
:100540004FF0FF310E4801F0D1FE24F003042C449B
:10055000761BA54209D10B4AD2F80034DB07FBD544
:10056000074801F09DFE002070BD7159284600F03B
:1005700025FF0435EDE76FF01500F5E72046F3E7BA
:100580001004022000900340F0B54B79012B29D0D4
:10059000032B24D110268B79032B20D1CC792CB1BD
:1005A000012C1CD103689B681B79C3B10A7912B175
:1005B000022A14D10E2247F6122703689B681D6891
:1005C0000B68BB426FD029D8B3F5965F65D014D8BD
:1005D000B3F5167F4FD007D8B3F5967F78D06FF07C
:1005E000220056E00026D6E7B3F5966F52D0B3F559
:1005F000166FF4D14FF41D233FE0B3F5615F4ED089
:1006000004D8B3F5165FEAD1334B36E0B3F5964F15
:1006100047D0B3F5E14FE2D1304B2EE0B3F5E13FE7
:100620004AD012D84DF6C027BB423FD005D8B3F50B
:10063000164FD4D14FF41D031FE0B3F5614F38D0EE
:10064000B3F5963FCBD1264B17E0B3F5E12F39D068
:1006500008D8B3F5613F32D0224FBB42BFD14FF033
:1006600080630AE0B3F5612F2FD01F4FBB42B6D194
:100670004FF0805301E04FF41C33C5F8243544EAB1
:1006800006031343C5F86C35836803C983E8030088
:100690000020F0BD4FF49E23EFE7144BEDE7144B21
:1006A000EBE7144BE9E74FF40003E6E74FF465038B
:1006B000E3E74FF46B03E0E74FF0EB73DDE74FF058
:1006C0006C73DAE74FF0E863D7E74FF07063D4E775
:1006D0004FF4A033D1E700BF0050270000C07500E1
:1006E00000903A0190D0030040420F0000B0130088
:1006F00000F03A0000A04E00026870B59268184BF6
:1007000014684FF00052856803219A601D2600226C
:10071000C3F87412C3F87022C4F80C651C26C4F820
:1007200014654FF000669E60C3F86C12C3F868222F
:100730001B23C4F808351A232946C4F81035FFF7DF
:1007400023FF58B90823C4F800351D440123C4F819
:100750001001C4F83455C4F83835236070BD00BFAB
:100760000025844008B5FCF7E1F901234FF00001B2
:10077000074A63F30201074B6FF3C5019B1ADB08BD
:10078000054863F38F1102F06AFA0020FDF714FFA9
:10079000D8530100E8530100FE6001002DE9F04349
:1007A00000261E4C85B054F8049C1D4F01ADB14588
:1007B00003D8002005B0BDE8F083636A97E807001E
:1007C000D3F8008085E807000C222946404602F055
:1007D0009BFFA0B9B8F1000F11D0636A21691B68B3
:1007E0001A6991420BD19A69A169914207D8E169CE
:1007F000914204D962695B6932EA030307D0236A34
:100800004BB1404080F311884FF0040002DFE368F1
:1008100001361C44CBE7626A1360F8E73CC2000073
:1008200050540100F0B50468054624B323461A4627
:1008300013F8011B202929D93A29F8D12378A3F1EB
:10084000300009281AD90023DFF84CC001322046B5
:100850005CF8237010F8011B17F8016BA1F1610E11
:10086000BEF1190F9CBF2039C9B28EB1B142F1D08F
:100870000133082BEBD14FF0FF3008E0631C9A42A4
:10088000E1D10728F7D801322A6000E00020F0BD4E
:100890008242EDD11846F7E7B4550100002310B5A8
:1008A000C3704FF0FF33C362044603F044FA30BB19
:1008B00094F82F2294F82E3243EA02234AF6552266
:1008C00093421ED194F83030E92B05D0236B104AA7
:1008D00003F0FF13934216D104F1660003F079F997
:1008E0000C4B20F07F4098420FD004F1820003F0BF
:1008F00070F9094B984214BF0220002010BD04205B
:10090000FCE70320FAE70220F8E70020F6E700BF43
:10091000EB009000464154004641543300232DE93A
:10092000F0430B6085B00F461546FFF77BFF061EB0
:10093000C0F22D81994B53F82640002C00F02981FC
:100940003C60237805F0FE0573B1607800F0C0FCD0
:10095000C10709D4002D00F0F58010F0040000D08C
:100960000A2005B0BDE8F0830023F0B22370607068
:1009700000F0BAFCC20700F10E810DB14307EFD4BD
:1009800000212046FFF78AFF022840F0E680002180
:1009900004F5FB7515F8040C10B1284603F019F99D
:1009A0004DF821000131042905F11005F2D100268E
:1009B0005DF82650002D00F0C78029462046FFF73D
:1009C0006DFF012800F2C18094F83C2094F83B3080
:1009D00043EA0223B3F5007F40F0C38094F8473028
:1009E00094F8466056EA032604D104F1540003F05B
:1009F000F0F8064694F84090A66109F1FF33012B08
:100A000084F8029000F2AD8094F83D70BBB263812F
:100A1000002B00F0A6807B1E3B4240F0A28094F8A1
:100A2000423094F8418048EA032818F00F0FA4F8E8
:100A3000088040F0968094F8441094F8430050EAFF
:100A4000012003D104F1500003F0C3F894F83F20D3
:100A500094F83E3053EA022300F0838006FB09FC41
:100A600003EB1812624490427BD3811AB1FBF7F179
:100A7000002976D04FF6F57740F6F570B9428CBF75
:100A800003270227814298BF01272B4402312A44C1
:100A9000032F6161E5612362A26266D194F85B2055
:100AA00094F85A3053EA02235BD1B8F1000F58D1C1
:100AB00004F15C0003F08DF86062890001F2FF111F
:100AC000B6EB512F4DD34FF0FF33C4E903338023EE
:100AD000032F23712FD194F8612094F8603043EAFA
:100AE0000223012B27D1691C204603F024F910BBF7
:100AF00094F82F2294F82E32207143EA02234AF60A
:100B00005522934217D104F1300003F062F8244BD0
:100B1000984210D104F5057003F05BF8214B984220
:100B200009D104F5067003F054F8206104F507704C
:100B300003F04FF8E0601C4A2770138801339BB222
:100B40001380E38000200CE703200136042E7FF49D
:100B50002FAF042805D1012003E70428FBD001288A
:100B600001D90D20FDE600252EE7B8F1000FF8D0E1
:100B7000022F4FEA410018BF4018634418BF01F02C
:100B8000010163620CBF014601EB500196E70B20A7
:100B9000E7E60C20E5E60320E3E600BF20040220A0
:100BA00052526141727241617C0502202DE9F0418F
:100BB000044607680D4611F8013B2F2BFAD05C2B39
:100BC000F8D00023A3602B781F2B58D904F12006FE
:100BD0000B222021304603F00CF800220820114699
:100BE00005F1FF3C1CF8013F0131202B0DD92F2BC3
:100BF00001D05C2B4BD16818411B10F801CBBCF124
:100C00002F0FF9D0BCF15C0FF6D00D44002A4ED066
:100C100094F820202046E52A04BF052284F82020ED
:100C2000212B34BF0423002384F82B30D4F8008018
:100C300003F04CFA00283ED1A169404603F07BF84E
:100C4000002838D1E3691A78002A3FD0DA7A02F016
:100C50003F02A271DA7A11070CD4314603F10B0C72
:100C600013F8012B11F801EB6345A2EB0E0220D023
:100C7000002AF5D00021204603F05BFADAE7802352
:100C8000204684F82B30BDE8F04103F01FBA2E2B2C
:100C900030D090420BD913F0800F08D1DFF8748068
:100CA00018F801EFBEF1000F29D07345F8D10620E6
:100CB0000AE0002ADED194F82B3048B1042803D191
:100CC00013F0040F08BF0520BDE8F0810420F2E70F
:100CD0005A07F9D4A379DB060AD5236907F1300155
:100CE000C3F308033878194402F0B8FFA0606FE737
:100CF0000520E9E70B28DAD008220B2072E7A3F1E0
:100D0000610EBEF1190F01D8203BDBB2B3540132A2
:100D100068E700BF4E6101001FB5CDE9001004A8CF
:100D200040F8041D1446FFF77DFD011E15DB0D4B39
:100D300053F8210008B100220270019808B1002286
:100D4000027043F8210030B1012C08D1002201A922
:100D50006846FFF7E3FD04B010BD0B20FBE7002061
:100D6000F9E700BF200402202DE9F04F89B008AE5A
:100D700046F80C0D30460D4617461C46FFF752FD4F
:100D80000028C0F23982A04B53F820300BB100226A
:100D90001A70C6B2304600F0A7FAC20700F12E82E0
:100DA000430700F12D8206AA0321304600F0C0FA65
:100DB00030B9069A531EB3F5004F01D21A4201D042
:100DC0000123069347B1914BA7F500729A4203D9CC
:100DD000132009B0BDE8F08F7B1E3B42F8D1129B77
:100DE00023F4FF7323F0010304930BB90E20F0E703
:100DF00007AA0121304600F09BFA002840F0E58068
:100E000015F008030CBF4FF03F094FF000090393A2
:100E1000079B4B45EAD3A3EB09037F2B0793E5D947
:100E20007A0A802AD4D815F0020E07D005F00701FF
:100E3000022900F0EB81E80740F1E881E907C7D516
:100E4000002A3AD14FF0010871481D0B30F8021FFB
:100E500009B1A9421BD9B3FBF8F540F6F5718D42F3
:100E60004FF020019BBF05EB4505013502356D08AC
:100E70008CBF6D00033505F2FF158CBF02270127DB
:100E80006D0A4FF0010A0291E1E15200C3E14FEA1D
:100E90004808DBE7022F1DD14FF6F5718B450ED9BF
:100EA000002A40F0AF814FEA4802402AC8D9BEF17B
:100EB000000F40F0AD81802A98D89046CBE740F6ED
:100EC000F5718B450BD8002A90D14FEA4802802A51
:100ED000B6D98BE740F6F5739B4587D801274FF4C9
:100EE00000720021204602F084FE0B224949204670
:100EF00002F0ABFE00230222032FE372227363741D
:100F00004FF0010218BF0223079984F80EA0B1F533
:100F1000803FCAF3072A84F80D8084F80FA022745A
:100F2000A37454D2E174C1F307212175F8236375CA
:100F30003F2300222376FF236276A376E27649469A
:100F400004F11C0002F04DFE032F4FF0210343D1AA
:100F500084F84530482384F8432084F8442084F8FA
:100F60004630294604F1240002F03BFE022384F8B7
:100F70002C30012384F83030062384F8323080236B
:100F800084F84030292384F82D2084F82E2084F81A
:100F90002F2084F8312084F8332013221E4984F84E
:100FA000423004F1470002F050FE4FF0550384F840
:100FB000FE316FF055034A4684F8FF312146012384
:100FC000304600F0A9F9824650B3012001E704F150
:100FD000200002F006FEA9E784F82930482384F8AF
:100FE0002A30C5F30723E375802384F824302923AE
:100FF00084F8272084F82820A57584F82630132249
:10100000064904F12B00CEE72004022000FEFF0079
:101010001E5601001B610100276101003B610100B8
:10102000032F41D1012309F106022146304600F089
:1010300073F94FF400725146204602F0DAFD522354
:1010400041227221237063706123E270A37084F8DF
:10105000E41184F8E51184F8E62184F8E7310BF116
:10106000FF3104F5F47002F0BCFD022384F8EC318A
:101070004FF0550384F8FE316FF0550309F1070274
:1010800084F8FF312146012384F8EDA184F8EEA114
:1010900084F8EFA1304600F03FF90123214609EB27
:1010A0000302304600F038F9049A0021204602F08D
:1010B000A0FD032F58D1F8232370FF236370A37082
:1010C000E37023716371A371E37123726372A3727E
:1010D0000F23E372129B4FEA532B5D45AA4628BFAC
:1010E000DA4621465346019A304600F015F901468A
:1010F00000287FF46AAF4FF40072204602F079FDB9
:10110000019BB5EB0A0553440193E6D1029B032FE3
:1011100008BF43460293029B019A5B4528BF5B468A
:10112000214630461D4600F0F7F800287FF44DAF09
:10113000019B2B440193029B5B1B0293EBD1032F7A
:101140001BD0079BB3F5803F19D2022F14BF012398
:101150000423039AAAB100223046114600F0E8F8B1
:10116000003018BF012034E6012F5649204618BF31
:101170006FF0070102F035FDACE70C23E9E7062329
:10118000E7E74FF400720399204602F032FD552242
:1011900084F8FE21AA2284F8C23143F6C16384F8A0
:1011A000FF21039A012584F8BE2184F8C121079A02
:1011B00049464A44B2FBF3F2FE2384F8C331930854
:1011C00043F03F0384F8C43184F8C52104F5E3708B
:1011D00084F8BF5184F8C05102F003FD079904F56B
:1011E000E57002F0FEFC2B46039A2146304600F0E3
:1011F00093F80028AFD0E8E60B20EAE50320E8E505
:101200000A20E6E5BEF1000F3FF4F0AD002A57D109
:1012100001222D485D0C30F8021F19B1A9427FF65A
:1012200034AE0021B3FBF2F0284F8500A0F57F40DB
:10123000F63805F20725B8424FEA55253FF6D6ADF8
:1012400090460A4600214FF0200A032702910AEB3C
:10125000090101910299DDF818C068180199032F5E
:1012600008440CF1FF310144CCF1000C01EA0C0CF4
:1012700008BF0199ACEB000C04BF61440191C9EBBC
:10128000081108440CBFE24465448342FFF4AEAD4C
:10129000A3EB0A0B0299ABEB050BABEB010B032F96
:1012A000BBFBF8FB7FF4F6AD4FF6F5718B453FF6CF
:1012B00016AE002A7FF49AAD5FEA58023FF496AD6D
:1012C0001146AFE7F8FFFF002C560100FFFFFE0FAD
:1012D00008B5044B53F8200001F0B9FF003018BFE7
:1012E000012008BDD455010008B5044B53F8200077
:1012F00001F09FFF003018BF012008BDD455010048
:1013000010B5044C54F8200001F0AFFF003018BFB6
:10131000012010BDD455010010B5044C54F8200034
:1013200001F0BAFF003018BF012010BDD4550100F4
:10133000012908B505D003D303290BD0042008E008
:101340000521054B53F8200001F0BDFF003018BF08
:10135000012008BD0421F4E7D4550100014B024AE5
:101360001A6070479C2802200090D003044AD2F8EB
:101370000834DB07FBD50160BFF35F8F704700BF08
:1013800000900340C0F30B037BB90222084BC3F863
:1013900084254FF0FF320260D3F80024D207FBD53A
:1013A00000220448C3F8842570470348704700BFF3
:1013B000009003400000AD0B0A00AD0B012310B5F7
:1013C000044CC4F88435FFF7D1FF0023C4F88435FA
:1013D00010BD00BF009003402DE9F047964624223F
:1013E00004794A4D6243AE18377F002F40F08C805D
:1013F000006845F802E00122736091F8008091F8DE
:101400000CC0434B02FA08F2BCF1010F94BFDA6042
:101410009A60012208F1800643F826204E78FF2EBC
:101420001FBF0327B240DA6006F1800218BF43F8FD
:1014300022708F7808BF4FF0FF36FF2F1FBF8A7BC7
:1014400007F1800A920043F82A204FF0240202FBA1
:10145000045282F8207018BFB946CF7808BF4FF009
:10146000FF39FF2FD77710D0012291F804A0BA409E
:10147000BAF1000F40D0DA600322803743F827200A
:10148000242303FB045383F81EA08B68C0F808854F
:10149000C0F80C65C0F81095C0F824354B7B0033BC
:1014A00018BF0123BCF1020F28D0BCF1030F28D0D4
:1014B000BCF1010F01D143F00203C0F854358B7920
:1014C000C0F8C035BEF1000F02D04023C0F804338D
:1014D0000723C0F80035BEF1000F03D040F30730FA
:1014E000FCF764FC242303FB0454002363770123EB
:1014F00008482377BDE8F0879A60BDE743F004030E
:10150000DBE743F00603D8E70348F3E74004022093
:10151000002584400000AD0B0500AD0B24232DE910
:10152000F04104793F4D63431746EA180E46517F58
:101530008046002973D1EB5823B117F0140F04BF74
:10154000012353774FF0240C96E80F000CFB045C4A
:101550000CF10C0E8EE80F009CF81F20FF2A06D01D
:1015600001239CF81E1093402F4AB1B1936031685B
:1015700021B101F06043B3F1005F06D1B26872B1EE
:1015800002F06043B3F1005F09D0242303FB04544D
:10159000002326486377BDE8F081D360E7E7D8F8F9
:1015A00000307068C3F84415C3F84805F168C3F803
:1015B00034250022C3F83815C3F8182117F00102AA
:1015C00018BF0122C3F8502517F0020218BF0122EC
:1015D000C3F840253A075CBF01221A612422624306
:1015E000AA589AB9D3F81821002AFBD0242303FB68
:1015F0000454E27FFF2A05D00123A17F93400A4AC9
:1016000011B1D3600A48C6E79360FBE7402217F0A8
:10161000040F14BFC3F80823C3F80423F2E70548F6
:10162000B9E700BF40040220002584400A00AD0B4A
:101630000000AD0B0B00AD0B0D4BD3F81821AAB178
:101640000022C3F818210B4BD97FFF2905D00122B6
:10165000987F8A40084938B1CA60002207485A7703
:101660001A72D3E9002110478A60F6E7704700BF7D
:1016700000B00040400402200025844048040220BD
:1016800070B50026084B53F82040013053F8205025
:10169000A54200D870BD236820465B68984700B11A
:1016A00066600C34F4E700BFF4550100104B70B5D0
:1016B00005461E460F4C9C4204D10E4CB44209D143
:1016C000002412E062681AB122681268AA420CD0A3
:1016D0000C34F0E763680BB90C34EFE72368284655
:1016E000196801F0F5FF0028F6D1204670BD00BF53
:1016F00074290220A82802202DE9F34105468846D6
:1017000000F0C8FD01224FF00003294C62F30203F0
:10171000284A042DA4EB02046FF3C50398BF264AA0
:10172000C4F3C90464F38F13ADF8003007464FF0DB
:10173000000394BF52F82520204A2946204801F092
:10174000C7FAD8F81C30C3F308035BB14FF00001AF
:10175000012363F302016FF3C50164F38F1119488C
:1017600001F07DFA4FF00006012363F302066FF3E8
:10177000C506384664F38F1603F029FCB0B1027831
:10178000114B002A08BF1846FBF7ECF83346024617
:1017900039460E4801F084FA41462846FEF7E2FF3A
:1017A000384602B0BDE8F041FCF724BF0648EBE73D
:1017B00010540100D85301000C560100C66101000D
:1017C000DC61010004620100D461010025620100B6
:1017D00008B50B4D4FF02002EFF3118382F311880F
:1017E000BFF36F8F03F01AFC012104460228D8BF13
:1017F000084603F023FC2C62FCF746FBEAE700BF37
:101800003C0502200248034A0021121A01F0B9BF28
:10181000000002208405022008B50648064A074950
:10182000121A01F081FFBDE80840054A0549064843
:1018300001F07ABFB8270220D0290220806201007F
:10184000000000008062010000000220012208B5B3
:101850000B4B02201A70FFF713FF0A4A0A490B4884
:1018600001F0A0F90320FFF70BFF00F0F1FDFAF7FC
:101870006FFE074A137B23F00103137308BD00BFFB
:1018800083050220C85701003D6201004A62010041
:10189000D004022080B5A2B0FAF7C8FF334B83F31F
:1018A00008880024E023324D012785F82230EC77A8
:1018B0002C766C76AC766B6A2E4E43F4E0236B622A
:1018C000FCF772FEFCF7DAFA4FF0FF33AB62EB6223
:1018D00007AB6C222146184601F053FFB06020464A
:1018E0008DF82970FFF7CCFE3846FFF7C9FE224D70
:1018F00000F04EFC214B4FF48052CDE90473CDE94A
:1019000002441F4BCDE900441E492846756200F091
:1019100035FD6B7B23F0040213F01B0F6A7304D1B7
:10192000AB6913B9284600F01BFA174B0122059347
:101930000F23CDE903320023144DCDE90133009389
:101940004FF4A072124B1349284600F017FD6B7B31
:101950004FF4805223F004036B730F4B0949C6E91F
:1019600006330548064BF560FCF76AFAC8210220E9
:1019700000ED00E03C050220D004022038570100B1
:101980004D180100880802207462010064040220DE
:10199000D1170100881802205405022070B50E4BA3
:1019A0000E4CA34201D3002070BDD3E9030141EAEC
:1019B000000212F003020BD19D685A61AA4201D1C4
:1019C0001C33EEE75E6901320E6059610144F5E7B0
:1019D0006FF01500E8E700BF74290220AC2902204F
:1019E00010B513460C464FF02002EFF3118182F33D
:1019F0001188BFF36F8F426962B1226043691B682F
:101A00004361836901338361002081F31188BFF34F
:101A10006F8F0DE01BB923606FF00B00F5E70246F6
:101A2000044800F031FB18B9034B9B685B692360E5
:101A300010BD00BF840502203C05022070B504469D
:101A40000D464FF02003EFF3118683F31188BFF3A7
:101A50006F8F03F07EFA80B100212A6881664261AF
:101A6000427BD20603D183690BB900F079F9314684
:101A7000BDE87040074803F014BA2B6862691A6029
:101A80002B686361A369013BA36186F31188BFF3EF
:101A90006F8F70BD84050220F8B504460F464FF0E5
:101AA0002003EFF3118583F31188BFF36F8FC268B2
:101AB00030495AB180688E68B04215D0B7B985F305
:101AC0001188BFF36F8F6FF00F000CE08B6893F9F4
:101AD0000E3023618B680132E260A36085F31188C8
:101AE000BFF36F8F0020F8BD2369F2E790F90E3045
:101AF00096F90E109942A8BF194621EAE171994260
:101B00002BDA00F003FB06463B46224629461A48DC
:101B100000F0BAFA0028E6D04FF02003EFF3118569
:101B200083F31188BFF36F8F236821699C4207D02C
:101B300033B193F90E309942A8BF194621EAE171F9
:101B4000A06890F90E30994209D16EB129460A4831
:101B500003F0A7F96FF00A00C5E70026D4E700F00C
:101B6000D5FA0028F2D1F0E785F31188BFF36F8F23
:101B7000F0E700BF3C0502208405022038B58368E9
:101B80000446002B3BD0214A926893423AD1DA7B3B
:101B9000013ADA73C368012B05D0013BC36000F042
:101BA000C3F8002038BD4FF02003EFF3118583F315
:101BB0001188BFF36F8F0169806890F90E309942E8
:101BC00001D000F0A3FA204603F0C3F9A06080B171
:101BD00090F90E20226100228266427BD20603D158
:101BE00083690BB900F0BCF82946094803F059F99C
:101BF000D5E7E06085F31188BFF36F8FCFE76FF013
:101C00001500CFE74FF0FF30CCE700BF3C050220C6
:101C10008405022010B5084C23685BB1FCF730F84E
:101C20002368064A184410610021BDE81040184698
:101C300003F004BA10BD00BF740502203C05022069
:101C4000F8B50D464FF02003EFF3118483F31188AC
:101C5000BFF36F8F4FF4004140F2E73600270022B8
:101C6000E1FB0067094B30461A6139464FF47A723E
:101C70000023FAF7E3FA064B1860064B1D60FFF7E6
:101C8000C9FF84F31188BFF36F8FF8BD3C050220B4
:101C900074050220700502204FF02003EFF311813C
:101CA00083F31188BFF36F8F044B9A68D37B013B9A
:101CB000D37381F31188BFF36F8F70473C05022007
:101CC000094B03F12802824205D19B688B4202D165
:101CD0004B7BDB0607D1D1E900231A600A68536009
:101CE0000023C1E9003370473C05022038B50D4C94
:101CF000024604F1280003F0F5F8054600B9E5684E
:101D0000A3684AB95A7BD20606D1AA6922B9DA89F0
:101D10007F2A01D9636238BD9D4201D0FFF77AFF67
:101D20006562F8E73C05022010B54FF02003EFF3A1
:101D3000118483F31188BFF36F8F084B00209A68DA
:101D4000D37B0133D373FFF7D1FF84F31188BFF343
:101D50006F8FBDE8104003F0BBB800BF3C05022008
:101D6000F8B54FF02003EFF3118483F31188BFF32C
:101D70006F8F164A114651F8283F8B420CD05BB149
:101D8000D66A90F90E5093F90E70AF420BDCB34255
:101D900002D01B68002BF6D1D36A01604360D36A7E
:101DA0001860D06205E05A68C0E900325A681060D5
:101DB0005860437B63F07F0343730020FFF796FF77
:101DC00084F31188BFF36F8FF8BD00BF3C0502207C
:101DD000F8B504464FF02003EFF3118583F3118823
:101DE000BFF36F8F90F90D30002B03DA01461848CE
:101DF000FFF766FF174A02F12801D2E90A308B4249
:101E00000BD053B194F90E6093F90E70B7420ADC0F
:101E1000834202D01B68002BF6D1C4E90010D36ABC
:101E20001C60D46205E05968C4E9003159680C604F
:101E30005C60637B906863F07F036373031B5842AD
:101E40005841FFF753FF85F31188BFF36F8FF8BD3B
:101E5000640502203C050220154A164938B50C6875
:101E60009368A342144603D1BDE83840FFF7D2BEC1
:101E700000250D6010490968B9B1D9897F2914D8A6
:101E80000E4993F90E5009688D420EDB0C498B42C6
:101E90000BD0996949B91169814203DC1846FFF7F3
:101EA00097FFE1E7091A116138BD00232361FBE7C1
:101EB0003C0502206C0502207405022070050220FA
:101EC0006404022070B50446183003F091F84FF016
:101ED0002003EFF3118683F31188BFF36F8F94F91A
:101EE0000D30002B07DA21460E48FFF7E9FE637B31
:101EF00003F07F0363730C4D637BA86843F010030A
:101F00006373031B58425841FFF7F0FE86F31188B4
:101F1000BFF36F8FAB68A34203D1BDE8704002F0FE
:101F2000D7BF70BD640502203C050220036D70B56B
:101F3000044603B1984704F1180003F059F84FF034
:101F40002003EFF3118583F31188BFF36F8F2046D1
:101F500002F075FF0646D8B194F90D30002B07DA70
:101F600021461248FFF7ACFE637B03F07F036373E7
:101F70000F4B9868021B50425041FFF7B7FE637B3E
:101F800043F00803637385F31188BFF36F8F70BD4F
:101F9000637B9B07F3D52146A068FFF791FE637B27
:101FA000A66023F002036373E9E700BF6405022023
:101FB0003C05022038B504464FF02003EFF31185AD
:101FC00083F31188BFF36F8F90F90D30002B07DA80
:101FD00001460948FFF774FE637B03F07F036373D8
:101FE000064B9868031B58425841FFF77FFE85F364
:101FF0001188BFF36F8F38BD640502203C050220B5
:1020000070B504460D461646FFF7D4FF637B43F0D8
:1020100002036373EDB12B68A5609D420CD05BB1E8
:1020200094F90E2093F90E1091420CDC69688B42F2
:1020300002D01B68002BF5D16B68256063606B686C
:102040001C606C6005E05A68C4E900325A6814608C
:102050005C60731C15D04FF4004540F2E73000215E
:1020600026EAE6764FF47A72C5FB06010023FAF7FA
:10207000E5F80449421C04F11800BDE8704000F086
:102080007DBA70BDF14E010010B50C461146064AEE
:102090009068064A10601A46FFF7B2FF2046BDE876
:1020A0001040FBF72FBE00BF3C0502206C0502204C
:1020B000F8B5461C02F0DCFF34184FF02003EFF3B4
:1020C000118783F31188BFF36F8F0D4D0D4BA868F7
:1020D0001860FFF76FFFA8680B493246183000F010
:1020E0004DFAAA683846537B43F010035373FBF74D
:1020F00009FE02F0BDFF201A20EAE070F8BD00BF23
:102100003C0502206C050220F14E01002DE9F84348
:1021100004464FF02003EFF3118983F31188BFF3D6
:102120006F8F02F08CFE4EB2804668B3174D214689
:1021300005F128073846FFF7C3FDAB6AA673BB421B
:102140002A460AD04BB1E96A93F90E00B0420BDC83
:10215000994202D01B68002BF6D1D36A27606360D6
:10216000D36A1C60D46205E05A68C4E900325A6838
:1021700014605C600120FFF7B9FD89F31188BFF39B
:102180006F8F4046BDE8F883A673F6E73C05022052
:102190000021044B084603F12802C3E90A22FFF795
:1021A0004FBD00BF3C050220F8B5244C244BA2686B
:1021B0009A4236D04FF02003EFF3118683F3118853
:1021C000BFF36F8F04F12805A1682846FFF778FD5B
:1021D000A26AA368AA420CD05AB1E06A93F90E1021
:1021E00092F90E708F420BDC824202D01268002AF4
:1021F000F6D1E26A1D605A60E26A1360E36205E0AC
:102200005168C3E9002151680B6053605A7B01207B
:1022100062F07F025A73FFF769FD86F31188BFF3FE
:102220006F8F4FF02003EFF3118083F31188BFF31A
:102230006F8FBDE8F840FBF765BD00BF3C0502208D
:102240006404022038B5431C044605D1104B98683D
:1022500000F0DEF8204638BD4FF4004540F2E7308C
:1022600000214FF47A72E5FB04010023F9F7E6FF41
:10227000044648B9FFF798FF4FF47A7084FB0001D9
:10228000C40B44EA4140E6E7FFF712FF0446F3E7D8
:102290003C050220014B9868704700BF3C050220B6
:1022A00070B504464FF02003EFF3118683F31188D5
:1022B000BFF36F8F02F04DFE054670B1437BDB0626
:1022C00003D183690BB9FFF74BFD0023AB663146A1
:1022D000BDE87040044802F0E4BDD4E902329A42FD
:1022E00018BF0133A360F2E78405022010B4024650
:1022F0000B464FF02000EFF3118180F31188BFF3FC
:102300006F8F946844B1013C946081F31188BFF3EE
:102310006F8F002010BC704733B981F31188BFF371
:102320006F8F6FF00F00F5E7014810BCFFF7ACBEF0
:102330008405022010B54FF02002EFF3118482F3E0
:102340001188BFF36F8F427B510704D484F3118847
:10235000BFF36F8F10BD22F0040112F01B0F417309
:1023600003D183690BB9FFF7FBFC2146BDE81040A0
:10237000014802F096BD00BF8405022030B587B049
:102380000E9D044604950D9D03950C9D02950B9D95
:1023900001950A9D0095FBF731FD044B9B6813B92D
:1023A000236607B030BD1B6EFAE700BF3C05022074
:1023B00070B5002686B005960E9E0F9D04960D9E64
:1023C000044603960C9E02960B9E01960A9E00966A
:1023D000FFF7D4FF6B1C03D02DB92046FFF7AAFFEF
:1023E000204606B070BD4FF4004640F2E7300021B1
:1023F0004FF47A720023E6FB0501F9F71FFF03494A
:10240000421C04F1180000F0B9F8E9E7F14E0100B0
:1024100038B505464FF02003EFF3118483F311889C
:10242000BFF36F8FFFF74EFD074B9B68AB4205D1A3
:102430002146BDE83840054802F033BD84F31188D9
:10244000BFF36F8F38BD00BF3C050220840502201A
:102450002DE9F04F284E294DB04687B0B54205F121
:10246000300410D3FFF718FC4FF4004940F2E73670
:102470000027224CDFF888A0444521D307B0BDE8EF
:10248000F04FFFF751BC54F8043C059354F8103C4E
:10249000049354F8143C039354F8183C029354F8F2
:1024A0001C3C019354F8203C009354E90A2354E95E
:1024B0000C01FFF763FF54F8303CDD642546CDE79F
:1024C000616A4B1C04D0256821B92846FFF732FF0A
:1024D0003034D1E7B346BC46E9FB01BC4FF47A7215
:1024E000002358466146F9F7A9FE5146421C05F102
:1024F000180000F043F8EBE7742902207429022049
:10250000F14E0100034B1B680BB9FBF7B9BB002070
:10251000704700BF78050220036840B1084A52683E
:10252000904204D01BB19A6881680A449A6042685C
:10253000136003685A600023C0E90033704700BF8E
:10254000A02802200B4B10B51C689C4208BF002439
:10255000FFF7D8FF54B1A368181A20EAE070064BC1
:102560001B6913B19842A8BF184610BD6FF0004018
:10257000F5E700BFA02802203C05022070B5044604
:102580001646C1604FF02003EFF3118583F31188E5
:10259000BFF36F8FFFF7B6FF012EACBF801901307C
:1025A000174BA0601A689A4201D05E6832B95A6827
:1025B000236062605A6814605C600BE09068A168F8
:1025C000884216DD411A91605168C4E900215168C2
:1025D0000C6054601A689A4206D0944204D1FFF706
:1025E000B1FF0021FBF7F4FA85F31188BFF36F8F79
:1025F00070BD091A9642A160D9D01268D6E700BF13
:10260000A02802202DE9F04B0446FFF725FC4FF0EF
:102610002003EFF3118583F31188BFF36F8F214FF0
:10262000214EB846DFF884903460D9F80040326813
:102630004C45D7E900BC05D024B1A368934214DD12
:102640009B1AA36000241BEB02004CEBE271C8E96B
:1026500000013460FFF776FF2146FBF7B9FA85F3F6
:102660001188BFF36F8FBDE8F08B1BEB03004CEBC1
:10267000E371D31A33600023C7E90001A360204649
:10268000FFF74AFF85F31188BFF36F8FE368984720
:102690004FF02003EFF3118583F31188BFF36F8FA1
:1026A000C3E700BF0000022078050220A028022016
:1026B0002DE918484FF02003EFF3118483F31188BC
:1026C000BFF36F8FFBF7DCFA074BD3E9002312EB64
:1026D000000B43F1000C5846614684F31188BFF3A8
:1026E0006F8FBDE8188800BF00000220026A38B56D
:1026F000002A044602DD0E49FFF740FF636A0133FA
:102700006362A3690BB12046984754F8105FA54255
:102710000DD065B1284602F0ABFB6B7BDB0604D124
:10272000AB6913B92846FFF71BFB0023AB6638BD26
:10273000ED2601002DE9F34140F2E736002704467B
:1027400088464FF40045304639460023E5FB020138
:102750004FF47A72F9F772FD3946009030464FF423
:102760007A720023E5FB0801F9F768FD0190204625
:1027700002F03EFC009B204623620023019A03499D
:10278000636202B0BDE8F041FFF7F8BEED2601003C
:1027900038B5074C074DAC4201D3002038BD04F1D9
:1027A00014032046C4E9053300F02AF81C34F2E78C
:1027B000AC290220AC2902200A448A4200D1704789
:1027C00011F8013B40BA80B25840C0F3031358409F
:1027D00080EA003083B2580100F4FF505840ECE723
:1027E0000A44914200D1704711F8013B5840C30997
:1027F00083EA10135840030183EA4000C0B2F0E7B7
:10280000FF232DE9F74F4568002229464FF00C0AB7
:102810004FF0200B0789046805FB07FCC372837A1D
:1028200064440193019B934208DC002319468F42C4
:1028300005EB030C21DC03B0BDE8F08FBCFBF1F32A
:10284000202B84BF1F3393FBFBF30AFB02FED0F85F
:102850000C804FEA910108EB0E0606F10409C6E967
:10286000019921F0030194BFC27248F80E4002F1B1
:10287000010288BF04EB8304D4E7C268066802F152
:10288000040EF41846F803E093680131636093681E
:102890001C6094606346CAE70020704770B50D461F
:1028A00004464520A04729465220A04729462346F2
:1028B000BDE87040522018472DE9F04F002705462B
:1028C0000E4692461C464FF0FF39B846BB4689B0CB
:1028D0009AF8000010B909B0BDE8F08FBBF1000F05
:1028E00007D1252800F04E813146A8470AF1010A98
:1028F000EEE7642868D01AD839280BD831285AD284
:102900002D2800F04681302846D0252808D13146B0
:10291000A8477AE0582800F0B480632800F02C81A2
:1029200031462520A84731469AF80000F0E7702884
:1029300000F09D800DD8692846D06C2803D16C2FFB
:1029400026D14C27D2E76828EAD1682F20D1482722
:10295000CCE7752870D017D87328E1D1226804F12C
:10296000040B11460C4614F8010B002840F0F980C6
:10297000B8F1030F40F013818C1AA9EB0404002C6A
:1029800000F3F5805C4640E078287AD07A28C7D1F9
:10299000002FC5D10746A9E7B9F1000F0EDAB8F14B
:1029A000000F00F0F980A0F13009B8F1000F08BF66
:1029B0004FF002089AE7B9F1000FF4DB0A2202FB9C
:1029C0000909A9F13009F0E77A2F03D1D4F800B052
:1029D00004341EE06C2FF9D04C2FF7D14FF0000CCF
:1029E0004FF0FF3B073424F0070303F10804D3E959
:1029F000002312F1004043F100018C4508BF8345DC
:102A000006D231462846FFF749FF4FF0000B6DE72D
:102A10009346BBF1000F06DA31462D20A847CBF1D3
:102A2000000B09F1FF3943465A46CDF80090314674
:102A30002846F9F74BFEE8E77A2F02D122680434E2
:102A400011E06C2FFAD04C2FF8D100214FF0FF305D
:102A5000073424F0070303F10804D3E90023994263
:102A600008BF9042CDD3CDF800904346DFE7314612
:102A70003020A84731467820A8474FF008094FF08A
:102A800001089AF80020702A05D1236804340493C1
:102A9000002302930CE06C2FF7D04C2FF5D10734B4
:102AA00024F00702136802F10804049353680293A8
:102AB00000221023039205924022043A02990498BE
:102AC000C2F1200CA2F1200ED04001FA0CFC40EA29
:102AD0000C0021FA0EFE40EA0E0010F00F0008D1A3
:102AE000059901B942BB4FF0300C08E0CDF814B0A5
:102AF000E3E709288CBF4FF0570C4FF0300C3146FC
:102B00006044CDE90523A847039B01330393DDE926
:102B10000523002AEAD1B8F1030F7FF476AF039BB7
:102B2000C3EB490BBBF1000F7FF76FAF314620209D
:102B3000A8470BF1FF3BF5E7591E9945069107DBC6
:102B4000B8F1010F06D1314630200792A847079A05
:102B5000069BB2E7B8F1020FFAD107923146202066
:102B6000F4E731460292A8472146029AFAE6314636
:102B70002020A847013C02E73146206804F1040BFD
:102B8000A847FFE65F46D8464FF0FF394FF0010BEC
:102B9000ACE64FF00308A9E64FF00108A6E65C4654
:102BA0008346A3E60FB407B504A951F8040B0191BD
:102BB000F9F7DEFD03B05DF804EB04B0704704469E
:102BC00008B5084611461A46A047FFF763FBFBF716
:102BD00011FD7047FEF7C2BB0023C0E90033704708
:102BE000036823B90160002341600B6070474368AC
:102BF0001960F8E70068704703680BB11A68026053
:102C00001846704708B5FAF769F818B10123436010
:102C10000023038108BDFBF74DB800207047002357
:102C2000F0B51A461C46012710F8015B0DB18A4227
:102C300001D31846F0BD252D02D184F00104F3E73D
:102C4000002CF1D045F02006613E192EECD8732DF2
:102C500004BF07FA02F4234301320024E4E738B545
:102C600005460C46FFF7CEFF28B105612146BDE8B9
:102C70003840F9F7A1BF38BD70B504460E46154679
:102C8000FFF7C0FF58B101220461447A466162F344
:102C9000071444722946BDE87040F9F78DBF70BD36
:102CA0002DE9F0410546884617461E46FFF7AAFF64
:102CB00060B102230561457AC0E9058763F3071512
:102CC00045723146BDE8F041F9F776BFBDE8F081C5
:102CD0002DE9F8430546894690461F46BDF8206019
:102CE000FFF790FF68B103230561457AC0E90598B5
:102CF00063F307154572C7613146BDE8F843F9F73C
:102D00005BBFBDE8F88310B51C4600F093F820B116
:102D10002146BDE81040F9F74FBF10BD2DE9F8433B
:102D20001C4603890E469B08A3429DF8207003D8D9
:102D300000231360BDE8F88311682144994284BFE1
:102D4000191B11600C2BD2F8009028D9072CD0F851
:102D500014802BD8082318304B4528BF4B462044FD
:102D60001D461A46FFB1314600F0DEFCA9EB05090D
:102D70002E44B9F1000FDDD0C4F11C054D4528BF2C
:102D80004D46201D40442A46BFB1314600F0CCFCE0
:102D9000A9EB0509D8F800802E440024E9E7143097
:102DA0004FF00008D8E701463046DDE7083C1B2C11
:102DB000DFD9D8F800801C3CF9E701463046E5E74A
:102DC0000430D0E8EF3F0133C0E8E23F002AF8D1F9
:102DD0007047407A00097047437A1B098B4216D925
:102DE000032B03D800EB810148697047012903D800
:102DF00000EB81018869704743690239062903D8CD
:102E000003EB81014868704707391B68F6E700202B
:102E100070470346021DD2E8EF1F0139C2E8EC1FDC
:102E2000BCF1000FF7D15B680BB9F9F769BF7047C8
:102E3000006970472DE9F84F824688461546F9F734
:102E40004DFF044660B301230026032D4360068135
:102E50000FD9427AA5F1020966F307124272027A8B
:102E600000F1140B42F0020202724661B9F1000F48
:102E70000EDC637A032D65F30713C4F810A06372A8
:102E800018D8AA00414604F1140000F04DFC07E0F8
:102E9000F9F724FF074630B92046F9F731FF3C46E1
:102EA0002046BDE8F88FCBF80000A9F107090660BD
:102EB0008346DBE74146082204F11800676900F009
:102EC00033FC023D08F10808072D2E4628BF0726CF
:102ED0004FEA86094146381D4A4600F025FCAD1BE5
:102EE000C8443F68F0D1DBE713B500240094FFF736
:102EF00015FF02B010BDF8B506460D4614461F4634
:102F0000214628463A46B047241A0544F8D1F8BD70
:102F10002DE9F0478EB00EAF81460D46FFF788FFD2
:102F200006464846FFF755FF4FF0000882468300EB
:102F30000E3323F00703ADEB030D0EACD04516D1D5
:102F40004846FFF746FF0F281ED8DFE810F01900AB
:102F5000200026002D00360041004E005D006E006E
:102F600081009600AD00C600E100FE001D01414653
:102F70004846FFF731FF44F8280008F10108DDE773
:102F800031462846F9F700FFBD46BDE8F0872268C4
:102F900031462846F9F7F8FEF6E7D4E90023314632
:102FA0002846F9F7F1FEEFE7A36831460093D4E92C
:102FB00000232846F9F7E8FEE6E7E3683146019387
:102FC000A36828460093D4E90023F9F7DDFEDBE788
:102FD000236931460293E36828460193A36800936E
:102FE000D4E90023F9F7D0FECEE7636931460393B5
:102FF000236928460293E3680193A3680093D4E908
:103000000023F9F7C1FEBFE7A36931460493636962
:103010002846039323690293E3680193A36800930E
:10302000D4E90023F9F7B0FEAEE7E3693146059332
:10303000A369284604936369039323690293E368B1
:103040000193A3680093D4E90023F9F79DFE9BE761
:10305000236A31460693E36928460593A3690493DE
:103060006369039323690293E3680193A368009360
:10307000D4E90023F9F788FE86E7636A31460793AF
:10308000236A28460693E3690593A3690493636959
:10309000039323690293E3680193A3680093D4E93F
:1030A0000023F9F771FE6FE7A36A31460893636A5C
:1030B00028460793236A0693E3690593A36904935B
:1030C0006369039323690293E3680193A368009300
:1030D000D4E90023F9F758FE56E7E36A314609932D
:1030E000A36A28460893636A0793236A0693E369F1
:1030F0000593A36904936369039323690293E368C7
:103100000193A3680093D4E90023F9F73DFE3BE760
:10311000236B31460A93E36A28460993A36A08930E
:10312000636A0793236A0693E3690593A36904938B
:103130006369039323690293E3680193A36800938F
:10314000D4E90023F9F720FE1EE7636B31460B93A9
:10315000236B28460A93E36A0993A36A0893636A78
:103160000793236A0693E3690593A369049363694C
:10317000039323690293E3680193A3680093D4E95E
:103180000023F9F701FEFFE6A36B31460C93636B56
:1031900028460B93236B0A93E36A0993A36A089367
:1031A000636A0793236A0693E3690593A36904930B
:1031B0006369039323690293E3680193A36800930F
:1031C000D4E90023F9F7E0FDDEE6426810B5D2E964
:1031D0000023044681680068FFF78DFE00226368C3
:1031E0001A6010BD38B54B6805461A68CB680C46A6
:1031F0009A4202D10846FFF7E8FF6368D3E8EF2F51
:10320000511CC3E8E01F0028F8D1A36800209D549A
:1032100038BDF8B50D46164604464718BC4201D1E4
:103220002846F8BD14F8011B736830465B68984760
:10323000F4E710B5F9F7C4FF30B1C36823B11B68D8
:1032400013B1BDE8104018476FF0150010BD10B560
:10325000F9F7B6FF30B1C36823B15B6813B1BDE8BD
:10326000104018476FF0150010BD2DE9F0410D46D4
:1032700016461F46F9F7A4FF50B1C46844B1A468CC
:1032800034B13B4632462946A446BDE8F04160478A
:103290006FF01500BDE8F0812DE9F0410D461646AE
:1032A0001F46F9F78DFF50B1C46844B1E46834B1EA
:1032B0003B4632462946A446BDE8F04160476FF0E0
:1032C0001500BDE8F08170B50C461546F9F778FF9A
:1032D00040B1C36833B11B6923B12A462146BDE81A
:1032E000704018476FF0150070BD03784278817800
:1032F00042EA0322C37843EA012343EA02407047CB
:1033000007B5012201A9F9F7CFFF08B99DF804001C
:1033100003B05DF804FB03699B6893F820007047D5
:10332000002902DA08467047023003780BB18B435C
:10333000FAD141784942F5E710B4D0E904020B46CE
:1033400041684C680021A44610BC604738B504466B
:10335000056801F091FEB4F90430132B07DCE08816
:103360000133A38008B1FEF76DFF012038BD2D1A8F
:10337000002D05DBE0880028F5D1FEF715FFF4E706
:103380000020F3E713B5044601F076FE002300F5B4
:10339000FA70009001932046FFF7B2FF002808DB87
:1033A000030606D56846FFF7D1FF0028F3D16FF07A
:1033B0003B0002B010BDF7B505460F46FFF7E2FF30
:1033C000042206460DEB02012846F9F76DFF04467C
:1033D00001A8FFF78AFF38602846FFF791FF002C0D
:1033E00014BF2046304603B0F0BD13B5044601F0CB
:1033F00043FE002300F5FA70009001932046FFF78A
:103400007FFF002807DB08D16846FFF79FFF0028F1
:10341000F4D16FF03B0002B010BDFF2806D020466B
:10342000FFF76EFF0028F6DBFF2801D10020F2E74E
:103430006FF04B00EFE71FB50123CDE90012014605
:10344000CDF808D0039351F8040B436802AA1C6816
:103450000023A04704B010BD13B5130C41F0400188
:103460008DF80010190A04468DF801108DF802300D
:103470008DF80420C2F307236946052200208DF849
:103480000330FFF7ADF906228DF8050069462046A6
:10349000FFF7D1FF02B010BDF8B51E46037E04460B
:1034A0000F46154603B9550200212046FFF744FF99
:1034B0002A4612212046F9F7EDFF054648B976B9AC
:1034C00032460C212046F9F7E5FF2046FFF78DFF35
:1034D000054620460121FFF72FFF2846F8BD4FF48F
:1034E000007239462046F9F743FF05460028F0D11F
:1034F00007F50077013EE2E70C228368C9B202FBC0
:1035000001314B7A23B9087AB0FA80F0400970474C
:103510000220704702682DE9F041D2F80880CCB251
:1035200087684FF02003EFF3118683F31188BFF310
:103530006F8F0C226243B9180B7A43B3013BDBB2A5
:103540000B723BBB2501BB504B6008EB05035B686E
:10355000CBB901224544EB7A03F1804303F5A04344
:103560001A6000222B8903F1804303F5A0431A60FF
:103570000C21002001FB0474607286F31188BFF3F4
:103580006F8FBDE8F08198470028E2D1F0E76FF037
:103590004400F2E70020F0E738B50C2483680546C4
:1035A00004FB0134012363724FF02003EFF3118118
:1035B00083F31188BFF36F8F23682BB160681A689B
:1035C0008342226008BF626081F31188BFF36F8F6E
:1035D00003B938BDD3E9012128469047E4E700222A
:1035E000FAF7E8B970477047FAF754BC014600682B
:1035F000FAF75ABC08B5FAF7ADFCBDE80840FAF78F
:1036000073BB07B5002101A8FBF7DEF903B05DF835
:1036100004FB30B54B6885B00C689DF808200D8917
:103620000094498924F01F04013B234465F30402FC
:1036300061F3471223F01F030F288DF8082003932E
:10364000044605D9FBF73EF80446204605B030BDD8
:103650006946FBF71FF8F8E740E800F313F4803FF2
:10366000D8B208BF6FF0150070470346013911F852
:10367000012F0AB91A70704703F8012BF7E770B5EC
:10368000054601392C4642B111F8013F561E2BB9AF
:103690002A4404F8013BA242FBD170BD05F8013B6E
:1036A0003246EFE7C9B2027803468A4200F10100D0
:1036B00004D0002AF7D1002918BF0023184670470C
:1036C00002460346981A13F8011B0029FAD17047E5
:1036D0000138013910F8013F11F8012F934202D14E
:1036E000002BF7D11A46981A704730B50024A24231
:1036F00008D0035D0D5DAB4202D10134002BF6D141
:10370000581B00E0002030BD10B55AB101398418B3
:1037100010F8012B11F8013FA04201D09A42F7D0D6
:10372000D01A10BD1046FCE7F0B581EA0004A507E9
:1037300003460BD0013B0A4491421DD1F0BD002A43
:10374000FCD011F8014B013A03F8014B9C07F6D16C
:103750000C461D1F8F183E1B032E08D86FF0030563
:10376000940805FB0422A40023442144E2E754F812
:10377000046B45F8046FEEE711F8014B03F8014FB5
:10378000DAE70346F0B5C9B29C070FD11D4641EAFE
:10379000012444EA04449F187E1B032E0CD894088D
:1037A00003EB840413449C4209D1F0BD002AFCD0F1
:1037B00003F8011B013AE7E745F8044BECE704F88E
:1037C000011BF0E7034670B5B1FBF2F602FB1611E0
:1037D00009298CBF272500251C463031294404F8CF
:1037E000011B31462EB95E70241A834203D820464D
:1037F00070BD2346E8E71A78017803F8011900F84C
:10380000012BF2E7D0E900232DE930485FEA530CA1
:103810004FEA320B002502F001041BEB04024CEBD3
:103820000503C0E90023BDE830880521D0E9002365
:103830002DE9F04F12F1020843F10009B9FBF1F54F
:10384000002601FB05F7B8EB060869EB07094FEA0C
:10385000D80646EA4976B6FBF1FC0024C2464FEA98
:10386000CC06A6FB0189A2194FEA5C7745EB07035A
:103870001446BAEB0802B2FBF1F21D46A41845F15A
:103880000005C0E90045BDE8F08F0B682DE9104840
:10389000002B13DD013B0B600A2102684468A2FB88
:1038A00001BC5A4601FB04CC2CF07043C0E9002354
:1038B0004FEA1C7130310846BDE810883021FAE724
:1038C0004FF0FF3070474B68012B07DD0B68187015
:1038D0000B6801330B604B68013B4B600020704765
:1038E00003685869704713B51446C06801AA04F10B
:1038F0000C01013001F051F858B94FF40073019AEE
:10390000236053895B0263605369023BA36002B08A
:1039100010BD6FF00400FAE710B504688068A46871
:1039200001292468C06903D158406060002010BD9F
:1039300000334FF0010118BF0123D04000F0010017
:103940009140834214BFA160E160EFE770B5046865
:103950008068A468C069256801296E692C696D6852
:1039600080EA040084EA050404EA060480EA04000C
:103970001CBFD04000F001001860002070BD8368BB
:1039800030B5186858B10024814213D108685CB979
:103990005C681860A14200D158600020086072B9CC
:1039A000002030BD2846EFE720605868814208BFFC
:1039B0005C60F2E705680446002DF3D13AB11A685D
:1039C0000A60586819600028EAD15960E9E76FF089
:1039D0001500E6E701292DE9F04118BFD4B20646EB
:1039E00012BF25461F2500244FF001088768AC420E
:1039F00002D90020BDE8F081FB6808FA04F223EA4E
:103A00000203FB6021463046FCF732F90028F1D171
:103A10000134E4B2EBE701292DE9F04118BFD4B23B
:103A2000064612BF25461F2500244FF0010887686F
:103A3000AC4202D90020BDE8F081FB6808FA04F22C
:103A40001343FB6021463046FCF712F90028F2D1FF
:103A50000134E4B2ECE710B41346426854680A46F5
:103A6000A446002110BC604738B50468054624B35D
:103A7000A36813B3186800B361B1B4F9042059689E
:103A8000D20FFFF7E8FF2B689B689868BDE83840C5
:103A900001F098BA12B9A28892040ED4986801F085
:103AA00091FA2A689368B2F90420D3E90001D2435D
:103AB000BDE83840D20FFFF7CEBF38BD10B50122A8
:103AC00000210446FFF7D0FFE36823B9201DBDE8BD
:103AD0001040FEF7E5BB10BD806810B503688B424F
:103AE00006D190F84C4034B9FFF7E8FF204610BDEE
:103AF0006FF01500FBE76FF00F00F8E7002070474C
:103B000038B504460D4601F06DF9844209D2002C07
:103B100007DBA84205D32C4484428CBF002001203F
:103B200038BD0020FCE770B50D46194628461646FC
:103B30001C46FFF7E5FF70B184B1B5F5404F224652
:103B40002946304603DABDE87040F4F749BAFFF77A
:103B5000EBFD002070BD6FF01500FBE72046F9E794
:103B60000B46826892E8030083E803000020704758
:103B700003689B681B68D3F88004C3F8800470470F
:103B8000036882689B681B68D3F8100138B1127A09
:103B900000200A700122C3F810011A6070474FF02C
:103BA000FF30704782B002AA02F8011D00210368AD
:103BB0009B681B68C3F82011C3F844250122C3F891
:103BC00048259A60D3F820110029FBD0DA6002B0B2
:103BD000704742884378007843EA022340EA032092
:103BE00070470B0A017043700B0C090E8370C17093
:103BF0007047024400F8011B9042FBD170474369B3
:103C00000239023B8B4283BF4389806A01FB030078
:103C10000020704738B50D46044618B90023092026
:103C20002B6038BD0368002BF8D01A78002AF5D035
:103C3000D98882889142F1D15878FDF749FB10F07C
:103C40000100EBD123682B60EBE701380A4411F83F
:103C5000013B914200F8013FF9D17047CA7E8B7E4B
:103C6000032843EA022301BF487D0A7D42EA00227D
:103C700043EA024318467047C2F307238A76CB769D
:103C80000378032B01BF120C0A75120A4A7570479C
:103C9000F8B50023C4692E261846651E15F8012FB5
:103CA0000130202A0AD0052A08BFE522092802BFD0
:103CB000CF1801337E72CF187A7201330B28EDD101
:103CC00000220B445A72E37A04F11C000B72FFF7D6
:103CD00080FF086004F11600FFF77BFFC880000C2E
:103CE0008880F8BDF8B5C56A00F1300704460123A5
:103CF0002A4639464078FDF70FFBA0B9236AA2692E
:103D0000EB1A9342E07001D30020F8BDA678012E93
:103D1000FAD9A36939461D442A4601236078FDF784
:103D2000FBFA013EF3E70120EFE7C3780BB1FFF7A1
:103D3000D9BF18467047C36A70B58B4206460D4618
:103D400012D0FFF7F2FF044660B92A46012306F1BC
:103D500030017078FDF7D4FA00281CBF4FF0FF3512
:103D60000124F562204670BD0024FBE701292DE9FE
:103D7000F04705460C46174672D943698B426FD906
:103D80000378022B3FD0032B50D0012B68D101EBDD
:103D90005108016A01EB5821FFF7CDFF064638BBF9
:103DA00014F0010405F1300908F1010AC8F308080C
:103DB00017BF19F80830FBB203F00F023B011CBF1C
:103DC00003F0F003134309F808300123296AEB706C
:103DD00001EB5A212846FFF7AEFF064640B9CAF369
:103DE000080A44B1C7F3071709F80A700123EB70FA
:103DF0003046BDE8F08719F80A30C7F3032723F0EF
:103E00000F031F43F0E7016A01EB1421FFF793FF53
:103E100006460028ECD1640005F1300304F4FF7479
:103E20001F551A19C7F307275770DFE7016A01EB1F
:103E3000D411FFF780FF06460028D9D1A40005F170
:103E4000300304F4FE741C442046FFF7C2FE27F042
:103E5000704700F0704139432046FFF7C2FEC5E7C6
:103E60000226C5E70129F8B505460C4652D9436933
:103E700099424FD20378022B29D0032B38D0012B43
:103E800048D101EB5106016A01EB5621FFF753FFC0
:103E900010B14FF0FF30F8BD296A771CC6F3080651
:103EA0002E4401EB5721284696F83060FFF743FF78
:103EB0000028EED1C7F308073D4495F83000E3072A
:103EC00046EA00204CBF0009C0F30B00E3E7016A9B
:103ED00001EB1421FFF72FFF0028DAD16400303501
:103EE00004F4FF742B195B78285D40EA0320D2E7C5
:103EF000016A01EBD411FFF71EFF0028C9D1A4000D
:103F000005F1300004F4FE742044FFF762FE20F057
:103F10007040C0E70120BEE72DE9F041804605680A
:103F20000F4671B9EE68F6B16B69B34298BF0126CE
:103F300034466B690134A34218D8012E15D80024E9
:103F400009E02846FFF78EFF0128044637D9431CB5
:103F500004D14FF0FF342046BDE8F0816B69834205
:103F6000F9D83E46E4E70126E2E702242146D8F8E4
:103F70000000FFF777FF30B1012820D00130E8D0F2
:103F8000B442D6D1DBE74FF0FF3221462846FFF797
:103F9000EDFE90B957B9D5E90432023A9342EC608C
:103FA0000FD32B7943F001032B71D4E72246394616
:103FB0002846FFF7DBFE0028EDD00128C9D00124F8
:103FC000C9E7013B2B61ECE7F8B50D46012D07462B
:103FD00011462CD904686369AB4228D92AB14FF045
:103FE000FF322046FFF7C2FE30B929463868FFF796
:103FF00039FF064608B90020F8BD012817D0431C38
:1040000017D0002229462046FFF7B0FE0028F3D142
:10401000D4E90432911E8B4205D201332361237906
:1040200043F001032371B2423546DED8E3E70220B4
:10403000E2E70120E0E7F8B50446FFF776FE054623
:10404000002842D12378032B37D12779012F34D18F
:1040500004F1300601464FF400723046FFF7C9FD07
:10406000552384F82E32AA2384F82F32522341227A
:10407000722184F8303084F83130612384F83320A1
:1040800084F8323084F8162284F8173284F8141237
:1040900084F8151204F506702169FFF7A2FDE168A6
:1040A00004F50770FFF79DFDE2693B460132E262CD
:1040B00031466078FDF730F92571002260781146AD
:1040C000FDF736F9003018BF0120F8BD38B50023E0
:1040D000826805460468036192B92378022B01D9EE
:1040E000636A73B923890BB9022038BD636AAB6177
:1040F000AB696A61002BF7D03034EC610020F4E743
:10410000134661891A4661B911462868FFF7AAFE6D
:10411000431C02460BD00128E6D963699842F3D3C9
:10412000E2E719462046FFF76AFDA861E0E70120B3
:10413000DBE783692DE9F04705460F46ABB102691D
:1041400002F12008B8F5001F0FD2C8F3080904686F
:10415000B9F1000F4DD141690133836139B9238928
:10416000B3EB581F45D80023AB6104200BE06389F3
:10417000013B13EA58233CD12046FFF773FE012888
:10418000064602D80220BDE8F087421C01D101207A
:10419000F9E76369834226D8002FE4D0696928468D
:1041A000FFF7BAFE0646002836D00128EAD0431CA5
:1041B000EDD02046FFF7B9FD07460028E7D10146BC
:1041C0004FF4007204F13000FFF713FD3146204632
:1041D000FFF715FD4FF0010AE06263899F420FD39C
:1041E000E36ADF1BE7626E6131462046FFF707FD99
:1041F000A86130344C44C5F81080EC610020C2E75F
:1042000084F803A02046FFF76DFD0028BFD1E36AC4
:1042100001370133E362E0E70720B4E738B504462D
:1042200005680420A16909B9A8B11CE02846FFF778
:1042300082FDC0B9E3691A78C2B1DB7AE52A03F0DE
:104240003F03A37109D02E2A07D00F2B05D023F0EE
:104250002003082B01D0002038BD00212046FFF7A5
:1042600068FF0028DED00023A361F5E70420FAE709
:1042700070B505460668FFF729FF044628BBA96903
:104280003046FFF758FD0446F8B9EB691B78E52B7B
:1042900014D1A9693046FFF74EFD044660B90146C6
:1042A0002022E869FFF7A5FC0B2205F12001E8694F
:1042B000FFF7CBFC0123F370204670BD002BE8D044
:1042C00001212846FFF735FFD7E7042C08BF072454
:1042D000F2E72DE9F0478EB001911646044600281A
:1042E00000F0CE8002F03F052A4602A901A8FCF7A3
:1042F00015FB002840F0BC80029B0EAF47F82C3D18
:1043000001993846FCF752FC024620B99DF9373036
:10431000002BB8BF062216F01C0F55D0002A4AD039
:10432000042A45D13846FFF7A3FF024600283FD1B3
:1043300045F008052B0751D50026212148220A9B6C
:10434000DDF8089019745A749E73DE730A9B5A76CE
:10435000202219769E75DE750A9BDA72DDF828A098
:1043600099F800005146FFF779FC324680464846EE
:10437000FFF782FC01220A9B1E775E779E77DE772D
:10438000029BDA70B8F1000F28D032464146384619
:10439000D3F82C90FFF718FE024648B94946029818
:1043A000FFF7C9FC029B08F1FF31D9600246A8B1B2
:1043B0000023236033E09DF8123013F0110F5BD11E
:1043C0007207B7D50822F3E7002AF1D19DF8123021
:1043D000DF064FD4B60701D5D8074DD4029F0A9EF9
:1043E000FB6A6662236238782907314648BF45F088
:1043F0004005FFF733FC0146A06006F11C00FFF703
:10440000E8FBFB88AA06A3804FF000030646E060A5
:10441000276025746374E361636104D4002210464D
:104420000EB0BDE8F0870028F8D07D8960616D028C
:10443000B5420FD30022A161002AB9D1C6F3080307
:10444000002BEBD00298FFF7DAFBB8B100EB562057
:10445000E061E4E72068FFF705FD01280146A6EBCF
:10446000050603D9431CE3D10122E4E70222E2E777
:1044700002469DE704229BE7072299E7022297E77D
:104480000922CCE72DE9F04F9946002385B08846F4
:10449000C9F8003003A904461546FFF7BBFB0646E2
:1044A000E0B9667CD6B9237CDA0779D5E368676919
:1044B000DF1BAF4228BF2F4687B16269C2F30803F2
:1044C000002B54D1039B5B89013B13EA522A13D181
:1044D00042B9A06801280AD802266674304605B0A1
:1044E000BDE8F08FA1692068FFF7BCFCF2E7431C30
:1044F00001D10126F1E7A061DDF80CB0A1695846B1
:10450000FFF77DFB0028E7D00AEB00037D0A01934B
:104510002BD0BBF80A200AEB0501914288BFA2EB21
:104520000A052B46019A41469BF80100FCF7E8FE7C
:104530000028DED10399CB785BB1C86A019BC01A11
:10454000A84206D24FF40072303108EB4020FFF74A
:104550007CFB6D026369A8442B446361D9F8003089
:104560007F1B2B44C9F80030A6E7019BE361656916
:10457000E169C5F30805C5F50075BD42039828BF7C
:104580003D46FFF7D8FB0028B3D10399636930316A
:10459000C3F308032A4619444046FFF756FBD9E700
:1045A00007269BE72DE9F04F9B46002385B08946FF
:1045B000CBF8003003A904461746FFF72BFB06464D
:1045C00010BB667C06BB237C9A0740F1A58063691B
:1045D000FB4200D3DF439FB16369C3F30802002AA3
:1045E0007DD1039A5289013A12EA532201921ED1D7
:1045F00073B9A06870B901462046FFF78DFC48B931
:10460000237C43F040032374304605B0BDE8F08FAF
:10461000A169F1E7012802D102266674F4E7431C80
:1046200001D10126F9E7A368A06103B9A06003984E
:10463000E369C26A9A4203D1FFF777FB0028F0D101
:10464000DDF80CA0A1695046FFF7D9FA0028E3D0A5
:10465000019B7D0A03EB000833D0019ABAF80A30B7
:104660002A449A4288BF019A9AF8010088BF9D1A8D
:104670002B4642464946FCF74FFE82460028D0D1E1
:104680000398C16AA1EB0801A94209D24FF4007254
:1046900009EB41213030FFF7D8FA039B83F803A0E0
:1046A0006D026369E2682B4463619A422CBFE26049
:1046B000E360DBF80030A9442B44CBF800307F1BCB
:1046C00089E76269E3689A4207D35046FFF72DFBFA
:1046D0000028A6D1039BC3F82C80C4F81C80656910
:1046E000E169C5F30805C5F50075BD42039828BF0B
:1046F0003D46FFF720FB002893D1039863693030D3
:10470000C3F308032A4618444946FFF79EFA4FF0C0
:104710000102039BDA70C4E7072675E773B501A9A8
:104720000646FFF777FA054648BB337C5B0626D57D
:10473000316A0198FFF7FFFA054600BB746AE37A15
:10474000214643F02003E372B2683068FFF794FA21
:10475000F16804F11C00FFF744FA21232376482373
:10476000637601230198A575E575A574E574C3709A
:10477000FFF761FC0546337C23F040033374284681
:1047800002B070BD13B50446FFF7C8FF28B901A9F0
:104790002046FFF73FFA00B9206002B010BDF7B520
:1047A0000D4601A90446FFF735FA064600283FD119
:1047B000667C002E3CD1E368AB4204D2227C12F02E
:1047C000020F08BF1D460022636962610DB92846C9
:1047D0001CE0019A57897F0203B3013B6A1EB2FBBA
:1047E000F7F2B3FBF7F18A4218D37A421340A1697A
:1047F0006361ED1A00293FD10020E36865699D429D
:1048000081BF237CE56043F040032374C5F30805B2
:1048100075B1E36983420BD0E06109E0A16879B921
:104820002046FFF779FB0128014604D10226667471
:10483000304603B0F0BD013001D10126F7E7A16099
:10484000A161D7E73B446361237CED1B9A0706D542
:104850002046FFF761FB014628B905460FE02068B6
:10486000FFF700FB01464B1CE7D00129DED9019B75
:104870005B698B42DAD9A161BD426369E2D86369A1
:104880002B446361C5F30803002BB5D00198FFF7F3
:10489000B6F90028CAD000EB5520AEE71FB5044694
:1048A000019148B3002203A901A8FCF737F870B9B9
:1048B000039B019923602046FCF778F9F0B994F93D
:1048C0002B30002B0CDBA379DB0603D4052000235F
:1048D00023600FE0039BE1691878FFF7BFF9A06040
:1048E000039B2046DB88A380FFF7F0FB0428EDD074
:1048F0000028ECD104B010BD0920FBE70428E5D066
:10490000E5E713B501A90446FFF784F900B9206073
:1049100002B010BD37B50D4601A90446FFF77AF97C
:1049200018B920461DB9FFF7D1FB03B030BDFFF722
:1049300075FC10F0FB03F8D16B72A3691BB129461B
:104940002046FFF7A5F900212046FFF7F2FB0428D7
:1049500008BF0020E9E730B58FB001900D46002276
:1049600003A901A8FBF7DAFF044688B9019903A857
:10497000FCF71CF9044658B99DF93730002B0ADBC7
:1049800035B1099B68721BB1294603A8FFF780F96E
:1049900020460FB030BD0624FAE72DE9F04385B07C
:1049A00001908946164603A9002201A8FBF7B6FF2D
:1049B000054648B9039CD4E90438A8F102029342A1
:1049C000346005D8C9F80030284605B0BDE8F0834A
:1049D0002378012B19D10227064639462046FFF7D6
:1049E00041FA431C3AD001283AD000B90136039B62
:1049F00001375B69BB42F0D8039BC9F800601A79A4
:104A00001E6142F001021A71DEE7216A0746044680
:104A100006464FB903984F1CFFF78DF910BB394676
:104A20004FF40077039C3034039B1B78022B0BD18F
:104A300062782378023F53EA022308BF013602342A
:104A4000B8F10108E5D1D7E72046FFF7C2F830F00A
:104A5000704308BF01360434043FF1E70125CBE77A
:104A60000225C9E70546C7E773B501A90446FFF764
:104A7000D1F80546C0B9657CB5B9237C9A072DD518
:104A80006669E368B3420FD98EB92A46A168204609
:104A9000FFF79AFA0546A6606369E360237C43F05A
:104AA0004003237405B16574284602B070BDA16946
:104AB0002068FFF7D7F9431C01460BD001280BD023
:104AC000019B5B698342E7D9A2692046FFF77CFA24
:104AD0000546E1E70125DFE70225DDE70725E3E7F6
:104AE00070B59AB00190022203A901A8FBF716FF46
:104AF000039B049368B9019904A8FCF757F840B9DF
:104B00009DF93B30002B36DB9DF81660F20702D58D
:104B100007201AB070BD039D0B992878FFF79EF807
:104B2000F306044610D4049D0A992846FFF703F9BA
:104B30000028EED1E5220B9B1A700123EB7094B98B
:104B40000398FFF778FAE4E711900FA80F95FFF7A5
:104B5000BDFA0028DDD10FA8FFF760FB0028D7D0F1
:104B60000428D6D1DFE70246214604A8FFF72CFA35
:104B70000028E5D0CDE70620CBE72DE9F0438FB044
:104B80000190022202A901A8FBF7C8FE029B04467D
:104B90000546039300287FD1019903A8FCF706F886
:104BA0000446002800F09780042875D1294603A800
:104BB000FFF7B2F9029A054653895B020693002873
:104BC0007ED0012800F08380431C00F082801046D4
:104BD000FFF7ABF806460446002872D1029C29462E
:104BE0002046FFF70CF804F1300731464FF400720D
:104BF00080463846FEF7FDFF0B2220213846FEF79F
:104C0000F8FF102384F83B3021234FF02E0984F85D
:104C10004830482384F8466084F8493084F8476077
:104C20002A463946029884F8309004F15006FFF77E
:104C300023F820223046FFF708F8029884F85190B4
:104C40000378059A032B03D1436A934208BF0022DD
:104C50004FF001093146FFF70FF8029B5E89B0441F
:104C6000A8EB0603E6B903A8FFF702FB044640BB26
:104C700021230A9C2A462376482321466376A6757B
:104C8000E6750298FEF7F8FF1023E37201230298FD
:104C9000C370FFF7D0F9044620460FB0BDE8F0839B
:104CA0000298C36280F80390FFF71CF8044640B9ED
:104CB00001464FF400723846FEF79BFF013ECFE7F6
:104CC00007240022294603A8FFF77EF9E4E702241F
:104CD000F7E70124F5E70824DEE770B5A0B00190FE
:104CE00020A840F8801DFBF79DFD022203A901A822
:104CF000FBF714FE00286ED1039B20AC44F8583D0E
:104D000001992046FBF752FF002864D19DF85330EB
:104D100013F0A00F61D1119915220B3104A8FEF7F1
:104D200094FF214615A82C22FEF78FFF009915A8A5
:104D3000FBF73CFF48B9179A0C9B9A4203D1199A8A
:104D40000E9B9A4203D0082045E0042843D115A8C1
:104D5000FFF78EFA00283ED101261C9D13220DF18B
:104D6000120105F10D00FEF770FF9DF81030039C55
:104D700043F02003EB72E670EB7ADB061DD50C9A4C
:104D8000179B9A4219D029462078FEF767FF014603
:104D90002046FEF734FF014608B32046FEF7CBFF5E
:104DA000C8B9039890F851302E2B06D1179A00F10C
:104DB0005001FEF761FF039BDE700A9C10992046AC
:104DC000FEF7B9FF38B9E522119B1A700123E37091
:104DD0000398FFF730F920B070BD0620FBE70220F2
:104DE000F9E700474FF4801070474FF48050704748
:104DF0004FF480707047FEF7F6BB30B50024846135
:104E000041EA020414F00304C0E9023201610CD14A
:104E10004461A34203D1C0E90000002030BD4569D0
:104E200001340D6041611144F3E76FF01500F5E7BF
:104E300003460020C3E90033C3E902007047437B07
:104E4000DB0603BF8069B0FA80F04009002070479C
:104E500010B54FF02003EFF3118483F31188BFF3F3
:104E60006F8F00F03FF884F31188BFF36F8F10BD90
:104E700038B504464FF02003EFF3118583F3118812
:104E8000BFF36F8F01468068FCF71AFF637B23F046
:104E90000203637385F31188BFF36F8F0023A36050
:104EA00038BD21B9EFF3058008B9F8F72BBF81F3BE
:104EB0001188BFF36F8F7047034620B9EFF3058267
:104EC0000AB9F8F71FBF83F31188BFF36F8F7047DC
:104ED0004FF02003EFF3118083F31188BFF36F8F3E
:104EE000FFF7EABF0368984214BF184600207047D6
:104EF00050F8103C70B50446A0F11805CBB14FF046
:104F00002003EFF3118683F31188BFF36F8F2946D7
:104F100050F8100CFCF7D4FE14F80B3C23F00203FD
:104F200004F80B3C86F31188BFF36F8F002344F81D
:104F3000103C14F80B3C284623F0140304F80B3CF7
:104F4000FFF77DFF20B12846BDE87040FCF708BFA1
:104F500070BD38B54FF02003EFF3118283F3118851
:104F6000BFF36F8FFFF7BEFF044682F31188BFF3D4
:104F70006F8FC8B14FF02003EFF3118583F31188D1
:104F8000BFF36F8F01468068FCF79AFE637B23F0C6
:104F90000203637385F31188BFF36F8F002304F15D
:104FA0001800A36000F024F8204638BD3AB18A42C8
:104FB00005D3C0E90212C0E90000002070476FF07D
:104FC00015007047F7F7F8BB6FF0460070470020F8
:104FD000704710B5029C8373047300230424C373C9
:104FE0004473C0E90633C0E91333C0E9161210BD9B
:104FF00010B54FF02002EFF3118482F31188BFF354
:105000006F8F03683BB1FDF787FA002084F31188A6
:10501000BFF36F8F10BD6FF01500F7E710B54FF0BD
:105020002003EFF3118483F31188BFF36F8FFDF733
:1050300089FA84F31188BFF36F8F10BD70B50446F1
:105040000E464FF02003EFF3118583F31188BFF371
:105050006F8FFDF777FA012805DDA04203DD3146A9
:105060002046F8F7B5FD85F31188BFF36F8F70BD4B
:1050700008B5FDF71DFB08BD10B5FDF719FB4FF492
:105080007A74A0FB042304FB0133D00B40EA4340B5
:10509000D90B10BD0023C0E9061200F110024362D3
:1050A000C0E90422C0E900338362704710B50446AA
:1050B000FFF79EFF00BBE3690BB12046984704F160
:1050C00010000021FFF7C4FE0446A8B1FFF7D0FE90
:1050D000637BDB0604D1A36913B92046FCF740FECD
:1050E0004FF02003EFF3118083F31188BFF36F8F2C
:1050F000BDE81040FFF7E0BE10BD70477071FF7F44
:105100000100000000000000E9350100000000007F
:10511000E935010000000000E93501000000000051
:10512000E935010000000000E93501000000000041
:10513000D1DA000000000000E935010000000000A5
:10514000E935010000000000E93501000000000021
:10515000E935010000000000E935010039160100C1
:10516000E34D010000000000E935010000000000EF
:10517000E935010000000000E935010000000000F1
:10518000E935010000000000E935010000000000E1
:10519000E935010000000000E935010000000000D1
:1051A000E935010000000000E935010000000000C1
:1051B00025DB000000000000E935010000000000D0
:1051C000E935010000000000E935010000000000A1
:1051D000E935010000000000E93501000000000091
:1051E000E935010000000000E93501000000000081
:1051F000E935010000000000E93501000000000071
:10520000E935010000000000E93501000000000060
:10521000E935010000000000E93501000000000050
:10522000E935010000000000E93501000000000040
:10523000E935010000000000E93501000000000030
:10524000E935010000000000E93501000000000020
:10525000E935010000000000E93501000000000010
:10526000E935010000000000E93501000000000000
:10527000E935010000000000E935010000000000F0
:10528000E935010000000000E935010000000000E0
:10529000E5FE000000000000E9350100000000000C
:1052A000E935010000000000E935010000000000C0
:1052B000E935010000000000E935010000000000B0
:1052C000E935010000000000E935010000000000A0
:1052D000E935010000000000E93501000000000090
:1052E000E935010000000000E93501000000000080
:1052F000E935010000000000E93501000000000070
:10530000E935010000000000E9350100C85701003F
:1053100091C7000000000000C8570100D9C7000075
:1053200000000000C8570100A5D1000000000000E7
:105330007859010019D3000000000000C85701008F
:1053400099D90000000000008D59010099DA000091
:10535000F0540100AD59010065DB000000000000C1
:10536000C8570100C5E8000000000000C857010050
:105370000DF4000000000000C8570100CDF8000047
:10538000000000005359010041FC00005455010089
:105390004D590100350001005C550100DB60010042
:1053A000FD040100000000002E580100F906010074
:1053B000AC550100C85701009D0701000000000026
:1053C000C85701009D19010000000000C8570100E6
:1053D00091270100000000009F5901000300000018
:1053E00083580100030000000F610100030000006A
:1053F0008E5F0100030000006357010003000000FE
:1054000038570100030000009A5D0100030000000E
:1054100071620100030000008759010003000000D1
:105420007E590100030000003D5701000300000009
:10543000CD60010003000000EE60010001000000EB
:10544000A05401003C030220355801000100000077
:10545000DEE61E28EAAC45B8025B0000DEE61E2848
:105460004CBBCE8F025B000000000000000000007B
:105470000338FDD870470000000000000E580100FE
:1054800016580100000000000000000000000000AD
:105490001E58010022580100265801002A58010018
:1054A00081D10000000000000000000075D1000064
:1054B00069D1000051D100001332010044030220E1
:1054C0008005022001000000B9D50000173301005B
:1054D00091D80000F5D80000DDD20000DF350100D2
:1054E00015350100B5D9000000000000F9340100B5
:1054F00000000000000000000001000493590100BA
:1055000000000000000000000401080C995901008F
:10551000020000001855010000000000145E0100A8
:1055200006000000E0FF0F00000002201C5E0100EA
:1055300021000000E0FF0320BDFD0000193901003B
:105540004D3901007F390100173A0100D5390100BA
:1055500000000000002584400000000000B0004072
:1055600000000000FF0F0000131211FF0000FF00F9
:105570000000004000000000FD010100D93A0100D8
:10558000273B0100250501009D040100FD3A0100B3
:105590008D04010004000000813B0100A53B0100D7
:1055A000713B010089050100613B01000080004062
:1055B000010000005E61010062610100676101009D
:1055C0003C5601006A6101006E61010072610100D8
:1055D000776101005E6101006261010067610100A5
:1055E0003C5601006A6101006E61010072610100B8
:1055F00077610100A8280220FC2802200829022047
:105600005C29022074290220F5FFFFFF7C61010064
:105610008A6101009E610100AD610100B961010074
:105620000100040010004000000100020000010021
:105630000200040008001000200000005344005342
:10564000746F7261676520696E6974204552524FAC
:10565000522100556E61626C6520746F206765741D
:1056600020736563746F7220636F756E7400426C93
:105670006F636B20636F756E7420257500556E61C6
:10568000626C6520746F2067657420736563746F46
:10569000722073697A6500536563746F7220736951
:1056A0007A652025750A004D656D6F727920536902
:1056B0007A65284D42292025750A002F53443A0067
:1056C0004469736B206D6F756E7465642E0A0045B6
:1056D00072726F72206F70656E696E672064697296
:1056E000202573205B25645D0A000A4C6973746988
:1056F0006E6720646972202573202E2E2E0A005BAF
:10570000444952205D2025730A005B46494C455DA3
:10571000202573202873697A65203D20257A752914
:105720000A004572726F72206D6F756E74696E67D4
:10573000206469736B2E0A006D61696E00736F637C
:10574000006C6F6767696E67003C6C6F675F7374AE
:105750007264757020616C6C6F63206661696C6542
:10576000643E006C6F6700617267756D656E7420D2
:10577000256420696E206C6F67206D6573736167A7
:10578000652022257322206D697373696E67206C12
:105790006F675F73747264757028292E002530322C
:1057A0007820007C002563000D00206D6573736117
:1057B0006765732064726F70706564202D2D2D0DE8
:1057C0000A1B5B306D000D0A001B5B313B33316DF2
:1057D0002D2D2D20001B5B306D0025732E002573B1
:1057E0003A20005B2530386C755D20005B25303237
:1057F000643A253032643A253032642E25303364E1
:105800002C253033645D20003C25733E20001B5B5B
:10581000313B33316D001B5B313B33336D006572BF
:10582000720077726E00696E6600646267005541AF
:1058300052545F30006C6F675F6261636B656E64CA
:105840005F7561727400696E76616C696420646969
:10585000736B20696E7465726661636521210064F3
:1058600069736B20696E7465726661636520616C33
:1058700072656164792072656769737465726564C5
:105880002121006469736B00466F756E642061208E
:105890007E2575204D694220534448432063617240
:1058A000642E004D616E7566616374757265722059
:1058B00049443D2564204F454D3D272563256327F9
:1058C000204E616D653D272563256325632563258E
:1058D0006327205265766973696F6E3D307825784D
:1058E0002053657269616C3D30782578000E050B98
:1058F0008A0500004C01130202041E0000FFFFFF96
:10590000FFFFFFFFFFFFFFFFFFFFFFFFFFFFFFFFA7
:10591000FFFFFFFFFFFFFFFFFFFFFFFFFFFFFFFF97
:10592000FFFFFFFFFFFFFFFFFFFFFFFFFFFFFFFF87
:10593000FFFFFFFFFFFFFFFFFFFFFFFFFF400E2006
:105940000E0416088A10050205013600005350495E
:105950005F33004750494F5F300054696D656F7584
:1059600074207768696C652077616974696E672057
:10597000666F7220212564005344484330007364ED
:1059800068635F73706900706F77657200434C4F96
:10599000434B006866636C6B006C66636C6B006302
:1059A0006C6F636B5F636F6E74726F6C007379738F
:1059B0005F636C6F636B0072302F61313A2020306F
:1059C0007825303878202072312F61323A2020300B
:1059D0007825303878202072322F61333A202030F9
:1059E00078253038780072332F61343A20203078AF
:1059F00025303878207231322F69703A2020307883
:105A000025303878207231342F6C723A202030786B
:105A1000253038780020787073723A20203078254D
:105A2000303878004661756C74696E6720696E73F2
:105A30007472756374696F6E2061646472657373E8
:105A400020287231352F7063293A2030782530387C
:105A500078002A2A2A2A2A20425553204641554CAA
:105A600054202A2A2A2A2A002020537461636B6951
:105A70006E67206572726F720020205072656369D4
:105A80007365206461746120627573206572726F42
:105A90007200202042464152204164647265737353
:105AA0003A2030782578002020496D70726563694E
:105AB0007365206461746120627573206572726F12
:105AC00072002020496E737472756374696F6E2062
:105AD000627573206572726F72002A2A2A2A2A2040
:105AE0004D5055204641554C54202A2A2A2A2A0036
:105AF0002020537461636B696E67206572726F72E8
:105B00002028636F6E746578742061726561206D02
:105B100069676874206265206E6F742076616C69B5
:105B20006429002020556E737461636B696E672071
:105B30006572726F7200202044617461204163635A
:105B40006573732056696F6C6174696F6E002020F5
:105B50004D4D46415220416464726573733A203062
:105B6000782578002020496E737472756374696FAC
:105B70006E204163636573732056696F6C6174694D
:105B80006F6E002020466C6F6174696E672D706FB8
:105B9000696E74206C617A79207374617465207009
:105BA0007265736572766174696F6E206572726F6B
:105BB00072002A2A2A2A2A20555341474520464165
:105BC000554C54202A2A2A2A2A0020204469766922
:105BD00073696F6E206279207A65726F002020559C
:105BE0006E616C69676E6564206D656D6F7279209A
:105BF000616363657373002020537461636B206F6E
:105C0000766572666C6F772028636F6E7465787442
:105C10002061726561206E6F742076616C69642901
:105C20000020204E6F20636F70726F636573736F17
:105C30007220696E737472756374696F6E7300207D
:105C400020496C6C6567616C206C6F6164206F66C5
:105C5000204558435F52455455524E20696E746F2B
:105C6000205043002020496C6C6567616C2075737F
:105C700065206F66207468652045505352002020CF
:105C8000417474656D707420746F206578656375F8
:105C9000746520756E646566696E656420696E73EF
:105CA0007472756374696F6E0045786365707469AA
:105CB0006F6E206F6363757272656420696E205326
:105CC0006563757265205374617465002A2A2A2AF7
:105CD0002A2048415244204641554C54202A2A2A21
:105CE0002A2A002020427573206661756C74206F2B
:105CF0006E20766563746F72207461626C652072C9
:105D00006561640020204661756C74206573636171
:105D10006C6174696F6E20287365652062656C6FB5
:105D20007729002A2A2A2A2A204465627567206D6D
:105D30006F6E69746F7220657863657074696F6ED9
:105D400020286E6F7420696D706C656D656E74656A
:105D50006429202A2A2A2A2A0052657365727665E8
:105D60006420457863657074696F6E2028005370F5
:105D70007572696F757320696E746572727570746F
:105D8000202849525120002A2A2A2A2A2025732015
:105D9000256429202A2A2A2A2A006D70750050615C
:105DA00072746974696F6E2025753A2073616E692B
:105DB000747920636865636B206661696C65642E25
:105DC00000496E76616C696420756E6465726C79E9
:105DD000696E6720726567696F6E20696E646578A9
:105DE000202575004661696C656420746F20616CC4
:105DF0006C6F63617465206E6577204D505520721D
:105E00006567696F6E2025750A002D2B20233000F1
:105E1000686C7A00464C4153485F30005352414D04
:105E20005F300066735F6F70656E646972006469ED
:105E3000726563746F727920636C6F73652065722D
:105E4000726F722028256429006D6F756E74207042
:105E50006F696E74206E6F7420696E697469616C0D
:105E6000697A656421210072657175657374656472
:105E70002066696C652073797374656D206E6F742C
:105E80002072656769737465726564212100696EAB
:105E900076616C6964206D6F756E7420706F696EC9
:105EA000742121006673206F70732066756E6374B1
:105EB000696F6E73206E6F74207365742121006D9D
:105EC0006F756E7420506F696E7420616C726561BD
:105ED0006479206578697374732121006673206D7D
:105EE0006F756E74206572726F72202825642900A8
:105EF000696E76616C69642066696C65206E616D9F
:105F00006521210025733A6D6F756E7420706F697D
:105F10006E74206E6F7420666F756E64212100664A
:105F2000696C65206F70656E206572726F722028D3
:105F3000256429002F006469726563746F7279208B
:105F40006F70656E206572726F722028256429005B
:105F50002E2E006469726563746F727920726561B8
:105F600064206572726F7220282564290066616959
:105F70006C656420746F2072656769737465722044
:105F800046696C652073797374656D2121006673B1
:105F90000000FBFBFBFEFEFEF3EFF7E2EDEDEDFB99
:105FA000FBFBF4E8EA55706461746520657863650D
:105FB0006564732063757272656E742062756666BF
:105FC0006572004661696C656420746F20696E6952
:105FD0007469616C697A65206465766963653A20E5
:105FE000257300536C617665206D6F64652069735D
:105FF000206E6F7420737570706F72746564206F9B
:106000006E202573004C6F6F706261636B206D6F43
:106010006465206973206E6F7420737570706F7281
:10602000746564004F6E6C792073696E676C6520CF
:106030006C696E65206D6F6465206973207375707F
:10604000706F7274656400576F72642073697A654B
:1060500073206F74686572207468616E20382062E6
:1060600069747320617265206E6F7420737570702F
:106070006F72746564004672657175656E636965FB
:1060800073206C6F776572207468616E20313235D1
:10609000206B487A20617265206E6F742073757072
:1060A000706F7274656400435320636F6E74726F17
:1060B0006C20696E6869626974656420286E6F205F
:1060C0004750494F2064657669636529007370699C
:1060D0005F6E7266785F7370696D004E52465F4600
:1060E0004C4153485F4452565F4E414D45007561E7
:1060F00072745F6E7266785F756172746500526566
:1061000073657474696E672073797374656D006666
:106110006174616C5F6572726F7200EBFE904D533B
:10612000444F53352E30004E4F204E414D452020D8
:1061300020204641543332202020004E4F204E4133
:106140004D452020202046415420202020200022A0
:106150002A2B2C3A3B3C3D3E3F5B5D7C7F0052410D
:106160004D004E414E4400434600534432005553C7
:10617000420055534232005553423300435055209C
:10618000657863657074696F6E00556E68616E64E2
:106190006C656420696E74657272757074005374F6
:1061A00061636B206F766572666C6F77004B65720A
:1061B0006E656C206F6F7073004B65726E656C203E
:1061C00070616E696300556E6B6E6F776E206572DD
:1061D000726F7200756E6B6E6F776E003E3E3E2082
:1061E0005A455048595220464154414C204552523C
:1061F0004F522025643A202573206F6E204350555E
:10620000202564004661756C7420647572696E6740
:1062100020696E746572727570742068616E646C4A
:10622000696E670A0043757272656E7420746872D5
:106230006561643A20257020282573290076322E66
:10624000312E39392D6E637331002A2A2A20426F8C
:106250006F74696E67205A6570687972204F532099
:106260006275696C64202573202573202A2A2A0A06
:10627000006F730069646C650000000000C00000DE
:10628000000000000000000000000000000000000E
:106290001C000220000000000000000000000000C0
:1062A000992801001B2C01000000000000000000E4
:1062B0003C560100C854010000000000C138010034
:1062C000F9FB0000D1FB0000A9FB000005FB00006A
:1062D000E138010049FB0000E9FA0000BDFA0000C6
:1062E00075FA00002DFA000001FA0000B1F9000073
:1062F00091F9000039F9000055F900001DF900007E
:10630000D9F80000E738010000000000442802200E
:106310004428022000000000010000005428022050
:1063200054280220000000000100000000000000CE
:10633000000000000000000000000000000000005D
:10634000000000000000000000000000000000004D
:10635000000000000000000000C201000001030076
:10636000000000000090D003A0280220A0280220F6
:106370000C5301000000000000000000C0530100A9
:106380000000000000000000CC53010000000000ED
:106390000000000060530100000000000000000049
:1063A00048530100DC54010094030220A85301006B
:1063B00098550100902802203C5301000000000085
:1063C0000000000054530100000000000000000025
:1063D00018530100000000000000000024530100D9
:1063E00000000000000000006C53010000000000ED
:1063F000000000008453010038550100E80302202A
:106400009C530100805501000000000090530100E2
:106410007855010040280220B4530100000000001C
:106420000000000030530100000000006C03022057
:1064300078530100000000000000000074290220D1
:1064400074290220040000002C00000068260220AD
:106450000000000000000000902902209029022086
:10646000040000002800000018270220000000009F
:1064700000000000AC290220AC290220000000002E
:1064800001000000BC290220BC29022000000000FD
:08649000000000000F000000F5
:00000001FF
